     1                                  
     2                                  ; Public Domain
     3                                  
     4                                  ; test run command: *.com; .; .
     5                                  
     6                                  %include "lmacros3.mac"
     1                              <1> [list -]
    14                              <2> [list -]
    14                              <1> [list -]
     7                                  %include "eld.mac"
     1                              <1> %if 0
     2                              <1> 
     3                              <1> Extensions for lDebug macros
     4                              <1> 
     5                              <1> Copyright (C) 2008-2025 E. C. Masloch
     6                              <1> 
     7                              <1> Usage of the works is permitted provided that this
     8                              <1> instrument is retained with the works, so that any entity
     9                              <1> that uses the works is notified of this instrument.
    10                              <1> 
    11                              <1> DISCLAIMER: THE WORKS ARE WITHOUT WARRANTY.
    12                              <1> 
    13                              <1> %endif
    14                              <1> 
    15                              <1> %ifndef ELD_MAC
    16                              <1> %define ELD_MAC 1
    17                              <1> 
    18                              <1> %include "lmacros3.mac"
     1                              <2> [list -]
    19                              <1> 
    20                              <1> 		; ELD executable header
    21                              <1> 	struc ELD_HEADER
    22 00000000 ????????            <1> eldhSignature:		resb 4	; "ELD1"
    23 00000004 ??????              <1> 			resb 3	; reserved
    24 00000007 ??                  <1> 			resb 1	; 26 (Ctrl-Z)
    25 00000008 ????????            <1> eldhCodeOffset:		resd 1	; position displacement from eldhSignature
    26 0000000C ????                <1> eldhCodeImageLength:	resw 1	; amount bytes, at least 32
    27 0000000E ????                <1> eldhCodeAllocLength:	resw 1	; amount bytes, added to prior. sum < 64 KiB
    28 00000010 ????????            <1> eldhDataOffset:		resd 1
    29 00000014 ????                <1> eldhDataImageLength:	resw 1	; (zero allowed)
    30 00000016 ????                <1> eldhDataAllocLength:	resw 1	; (zero allowed)
    31 00000018 ????                <1> eldhCodeEntrypoint:	resw 1	; within code section, used as displacement
    32 0000001A ????????            <1> eldhReserved:		resb 4	; reserved
    33 0000001E ????                <1> eldhExtensionSize:	resw 1	; from eldhSignature, -> past eldhx fields in use
    34                              <1> 	endstruc
    35                              <1> 	endarea ELD_HEADER, 1
    36                              <1> 
    37                              <1> 	struc ELD_HEADERX
    38 00000000 <res 20h>           <1> eldhxHeader:		resb ELD_HEADER_size
    39 00000020 ????????            <1> eldhxDescriptionOffset:	resd 1	; zero if none, from eldhxHeader. <= 128 Bytes
    40 00000024 ????????            <1> eldhxHelpOffset:	resd 1	; zero if none, from eldhxHeader
    41 00000028 ????????            <1> eldhxLibTable:		resd 1	; zero if none, from eldhxHeader
    42 0000002C ????????            <1> eldhxDateTimeOffset:	resd 1	; zero if none, from eldhxHeader
    43                              <1> 	alignb 16
    44                              <1> 	endstruc
    45                              <1> 
    46                              <1> 	struc ELD_TRAILER_HEADER
    47 00000000 ????????????????    <1> eldthSignature:		resb 8	; "ELD1TAIL"
    48 00000008 ????????            <1> eldthHeaderOffset:	resd 1	; negative displacement from eldthSignature,
    49                              <1> 				;  add this dword to the seek offset
    50 0000000C ????                <1> eldthReserved:		resw 1	; reserved, must be initialised to zero
    51 0000000E ????                <1> eldthChecksum:		resw 1	; sum of all words in trailer header = 0
    52                              <1> 	endstruc
    53                              <1> 	endarea ELD_TRAILER_HEADER, 1
    54                              <1> 
    55                              <1> 	struc ELD_LIBTABLE
    56 00000000 ????                <1> eldltFormat:		resw 1
    57                              <1> 	; 0 = uncompressed
    58                              <1> 	; 2 = heatshrink compressed
    59                              <1> 	; 3 = lzexedat -4 compressed
    60                              <1> 	; 4 = lzexedat -4 -l compressed
    61 00000002 ????                <1> eldltAmount:		resw 1
    62 00000004 ????????            <1> eldltOffset:		resd 1	; from eldhxHeader
    63                              <1> eldltCompressedLength:		; (dword, only present if format 2, 3, or 4)
    64                              <1> 	endstruc
    65                              <1> 	endarea ELD_LIBTABLE, 1
    66                              <1> 
    67                              <1> 		; ELD instance header
    68                              <1> 	struc ELD_INSTANCE
    69 00000000 ????                <1> eldiStartCode:		resw 1	; -> this structure itself (para aligned)
    70 00000002 ????                <1> eldiEndCode:		resw 1	; -> behind memory used by instance (para aligned)
    71 00000004 ????                <1> eldiStartData:		resw 1	; -> data in data entry section (para aligned), or 0
    72 00000006 ????                <1> eldiEndData:		resw 1	; -> behind data (para aligned), or 0
    73 00000008 ????????????????    <1> eldiIdentifier:		resb 8	; blank-filled text
    74 00000010 ????                <1> eldiFlags:		resw 1	; flags
    75                              <1> eldiListing_size equ 14
    76 00000012 <res Eh>            <1> eldiListing:		resb eldiListing_size
    77                              <1> 				; ASCIZ listing file name
    78                              <1> 	endstruc
    79                              <1> 		; flags for eldiFlags:
    80                              <1> eldifResident:		equ 1
    81                              <1> 
    82                              <1> 		; ELD link info header
    83                              <1> 	struc ELD_LINKINFO
    84 00000000 ????                <1> eldlSignature:		resw 1	; 0E1D1h
    85 00000002 ????????            <1> eldlReserved:		resw 2
    86 00000006 ????                <1> eldlUseLinkHash:	resw 1
    87 00000008 ????                <1> eldlDataAmount:		resw 1
    88 0000000A ????                <1> eldlDataPrefixes:	resw 1
    89 0000000C ????                <1> eldlDataEntries:	resw 1
    90 0000000E ????                <1> eldlDataAddresses:	resw 1
    91 00000010 ????                <1> eldlCodeAmount:		resw 1
    92 00000012 ????                <1> eldlCodePrefixes:	resw 1
    93 00000014 ????                <1> eldlCodeEntries:	resw 1
    94 00000016 ????                <1> eldlCodeAddresses:	resw 1
    95                              <1> 	endstruc
    96                              <1> 
    97                              <1> 	numdef ELD_CODE_VSTART, 9001h
    98                              <1> 	numdef ELD_DATA_VSTART, 8000h
    99                              <1> 	numdef ELD_RELOC_VSTART, 8000h
   100                              <1> 
   101                              <1> 	numdef ELD_RECLAIM_HINT, 0
   102                              <1> 	strdef ELD_LISTING, ""
   103                              <1> 	numdef ELD_DATETIME, 0
   104                              <1> 
   105                              <1> %if _ELD_DATETIME
   106                              <1>  %define PUT_ELDHX_DATETIME_OFFSET at eldhxDateTimeOffset, dd DATAOFFSET + datetime - datastart
   107                              <1>  %macro PUT_ELD_DATETIME 0.nolist
   108                              <1> datetime:	asciz __UTC_DATE__,'T',__UTC_TIME__,'Z'
   109                              <1> 		asciz		; for future extension
   110                              <1>  %endmacro
   111                              <1> %else
   112                              <1>  %define PUT_ELDHX_DATETIME_OFFSET
   113                              <1>  %define PUT_ELD_DATETIME
   114                              <1> %endif
   115                              <1> 
   116                              <1> %endif
     8                                  %include "eldcall.mac"
     1                              <1> %if 0
     2                              <1> 
     3                              <1> Extensions for lDebug call macros
     4                              <1> 
     5                              <1> Copyright (C) 2008-2024 E. C. Masloch
     6                              <1> 
     7                              <1> Usage of the works is permitted provided that this
     8                              <1> instrument is retained with the works, so that any entity
     9                              <1> that uses the works is notified of this instrument.
    10                              <1> 
    11                              <1> DISCLAIMER: THE WORKS ARE WITHOUT WARRANTY.
    12                              <1> 
    13                              <1> %endif
    14                              <1> 
    15                              <1> %ifndef ELDCALL_MAC
    16                              <1> %define ELDCALL_MAC 1
    17                              <1> 
    18                              <1> %include "lmacros3.mac"
     1                              <2> [list -]
    19                              <1> %include "nasmhash.mac"
     1                              <2> 
     2                              <2> %if 0
     3                              <2> 
     4                              <2> Hashing macros
     5                              <2>  by E. C. Masloch, 2019
     6                              <2> 
     7                              <2> Usage of the works is permitted provided that this
     8                              <2> instrument is retained with the works, so that any entity
     9                              <2> that uses the works is notified of this instrument.
    10                              <2> 
    11                              <2> DISCLAIMER: THE WORKS ARE WITHOUT WARRANTY.
    12                              <2> 
    13                              <2> %endif
    14                              <2> 
    15                              <2> %ifndef __NASMHASH_MAC__
    16                              <2> %assign __NASMHASH_MAC__ 1
    17                              <2> 
    18                              <2> 
    19                              <2> 	%macro hashdef 2+.nolist
    20                              <2> %ifempty %2
    21                              <2>  %assign _%1 1
    22                              <2> %else
    23                              <2> %ifstr %2
    24                              <2>  %define %%string %2
    25                              <2> %elifid %2
    26                              <2>  %defstr %%string %2
    27                              <2> %elifnum %2
    28                              <2>  %defstr %%string %2
    29                              <2> %eliftok %2
    30                              <2>  %defstr %%string %2
    31                              <2> %else
    32                              <2>  %error Unknown input
    33                              <2> %endif
    34                              <2> %strlen %%length %%string
    35                              <2> %assign %%hash 1
    36                              <2> %assign %%index 1
    37                              <2> %rep %%length
    38                              <2>  %substr %%char %%string %%index
    39                              <2>  %assign %%hash (%%hash * 31 + %%char) & 0FFFFh
    40                              <2>  %assign %%index %%index + 1
    41                              <2> %endrep
    42                              <2> %assign _%1 %%hash
    43                              <2> %endif
    44                              <2> 	%endmacro
    45                              <2> 
    46                              <2> 
    47                              <2> %endif
    20                              <1> %include "elddata.mac"
     1                              <2> %if 0
     2                              <2> 
     3                              <2> Extensions for lDebug data relocation macros
     4                              <2> 
     5                              <2> Copyright (C) 2008-2024 E. C. Masloch
     6                              <2> 
     7                              <2> Usage of the works is permitted provided that this
     8                              <2> instrument is retained with the works, so that any entity
     9                              <2> that uses the works is notified of this instrument.
    10                              <2> 
    11                              <2> DISCLAIMER: THE WORKS ARE WITHOUT WARRANTY.
    12                              <2> 
    13                              <2> %endif
    14                              <2> 
    15                              <2> %ifndef ELDDATA_MAC
    16                              <2> %define ELDDATA_MAC 1
    17                              <2> 
    18                              <2> %include "lmacros3.mac"
     1                              <3> [list -]
    19                              <2> %include "nasmhash.mac"
     1                              <3> 
     2                              <3> %if 0
     3                              <3> 
     4                              <3> Hashing macros
     5                              <3>  by E. C. Masloch, 2019
     6                              <3> 
     7                              <3> Usage of the works is permitted provided that this
     8                              <3> instrument is retained with the works, so that any entity
     9                              <3> that uses the works is notified of this instrument.
    10                              <3> 
    11                              <3> DISCLAIMER: THE WORKS ARE WITHOUT WARRANTY.
    12                              <3> 
    13                              <3> %endif
    14                              <3> 
    15                              <3> %ifndef __NASMHASH_MAC__
    16                              <3> %assign __NASMHASH_MAC__ 1
    17                              <3> 
    18                              <3> 
    19                              <3> 	%macro hashdef 2+.nolist
    20                              <3> %ifempty %2
    21                              <3>  %assign _%1 1
    22                              <3> %else
    23                              <3> %ifstr %2
    24                              <3>  %define %%string %2
    25                              <3> %elifid %2
    26                              <3>  %defstr %%string %2
    27                              <3> %elifnum %2
    28                              <3>  %defstr %%string %2
    29                              <3> %eliftok %2
    30                              <3>  %defstr %%string %2
    31                              <3> %else
    32                              <3>  %error Unknown input
    33                              <3> %endif
    34                              <3> %strlen %%length %%string
    35                              <3> %assign %%hash 1
    36                              <3> %assign %%index 1
    37                              <3> %rep %%length
    38                              <3>  %substr %%char %%string %%index
    39                              <3>  %assign %%hash (%%hash * 31 + %%char) & 0FFFFh
    40                              <3>  %assign %%index %%index + 1
    41                              <3> %endrep
    42                              <3> %assign _%1 %%hash
    43                              <3> %endif
    44                              <3> 	%endmacro
    45                              <3> 
    46                              <3> 
    47                              <3> %endif
    20                              <2> %include "eldcheck.mac"
     1                              <3> %if 0
     2                              <3> 
     3                              <3> Extensions for lDebug relocation check macros
     4                              <3> 
     5                              <3> Copyright (C) 2008-2023 E. C. Masloch
     6                              <3> 
     7                              <3> Usage of the works is permitted provided that this
     8                              <3> instrument is retained with the works, so that any entity
     9                              <3> that uses the works is notified of this instrument.
    10                              <3> 
    11                              <3> DISCLAIMER: THE WORKS ARE WITHOUT WARRANTY.
    12                              <3> 
    13                              <3> %endif
    14                              <3> 
    15                              <3> %ifndef ELDCHECK_MAC
    16                              <3> %define ELDCHECK_MAC 1
    17                              <3> 
    18                              <3> %assign ELDSTRICT 0
    19                              <3> %assign ELDSTRICTCOUNTER 0
    20                              <3> 
    21                              <3> 	%imacro eldstrict 1.nolist
    22                              <3> %ifidni %1, on
    23                              <3>  %assign ELDSTRICT 1
    24                              <3>  [warning +error=reloc-abs]
    25                              <3>  [warning +reloc-abs]
    26                              <3> %elifidni %1, off
    27                              <3>  %assign ELDSTRICT 0
    28                              <3>  [warning -reloc-abs]
    29                              <3> %else
    30                              <3>  %error Unknown keyword
    31                              <3> %endif
    32                              <3> 	%endmacro
    33                              <3> 
    34                              <3> 	%imacro reloc 1+.nolist
    35                              <3> %if ELDSTRICT
    36                              <3>  %if ELDSTRICTCOUNTER
    37                              <3>   %error Missing relocation
    38                              <3>  %endif
    39                              <3>  [warning -reloc-abs]
    40                              <3>  %assign ELDSTRICTCOUNTER 1
    41                              <3> %endif
    42                              <3> %1
    43                              <3> 	%endmacro
    44                              <3> 
    45                              <3> 	%imacro reloc2 1+.nolist
    46                              <3> %if ELDSTRICT
    47                              <3>  %if ELDSTRICTCOUNTER
    48                              <3>   %error Missing relocation
    49                              <3>  %endif
    50                              <3>  [warning -reloc-abs]
    51                              <3>  %assign ELDSTRICTCOUNTER 2
    52                              <3> %endif
    53                              <3> %1
    54                              <3> 	%endmacro
    55                              <3> 
    56                              <3> 	%imacro eldstrictcheck 0.nolist
    57                              <3> %if ELDSTRICT
    58                              <3>  %ifn ELDSTRICTCOUNTER
    59                              <3>   %error Unexpected relocation
    60                              <3>  %else
    61                              <3>   %assign ELDSTRICTCOUNTER ELDSTRICTCOUNTER - 1
    62                              <3>   %ifn ELDSTRICTCOUNTER
    63                              <3>    [warning +reloc-abs]
    64                              <3>   %endif
    65                              <3>  %endif
    66                              <3> %endif
    67                              <3> 	%endmacro
    68                              <3> 
    69                              <3> %endif
    70                              <3> 
    21                              <2> 
    22                              <2> 
    23                              <2> %assign ELDLINKER 0
    24                              <2> 
    25                              <2> %define INTERNAL_CODE_TO_CODE_RELOCATIONS ""
    26                              <2> %define INTERNAL_CODE_TO_DATA_RELOCATIONS ""
    27                              <2> %define INTERNAL_DATA_TO_CODE_RELOCATIONS ""
    28                              <2> %define INTERNAL_DATA_TO_DATA_RELOCATIONS ""
    29                              <2> %define INTERNAL_LINKER_CODE_TO_CODE_RELOCATIONS ""
    30                              <2> %define INTERNAL_LINKER_CODE_TO_DATA_RELOCATIONS ""
    31                              <2> %define INTERNAL_LINKER_DATA_TO_CODE_RELOCATIONS ""
    32                              <2> %define INTERNAL_LINKER_DATA_TO_DATA_RELOCATIONS ""
    33                              <2> %assign ELDDATA_OPTIONAL_STATUS 0		; not any seen yet
    34                              <2> %assign ELDDATA_PMREQUIRED_STATUS 0		; not any seen yet
    35                              <2> %assign ELDDATA_NEXT_STATUS 0			; not any seen yet
    36                              <2> %assign ELDDATA_NEXT_ENTRY -1
    37                              <2> %assign ELDDATA_NEXT_SECTION -1
    38                              <2> %assign ELDDATA_NEXT_OTHER -1
    39                              <2> 
    40                              <2> 	%imacro internalcoderelocation 0-1.nolist -2
    41                              <2> %assign %%entry $ + _CURRENT_SECTION %+ FIXUP + %1
    42                              <2> %if ELDLINKER
    43                              <2>  %ifidni _CURRENT_SECTION_TYPE, DATA
    44                              <2>   %xdefine INTERNAL_LINKER_DATA_TO_CODE_RELOCATIONS INTERNAL_LINKER_DATA_TO_CODE_RELOCATIONS, %%entry
    45                              <2>  %else
    46                              <2>   %xdefine INTERNAL_LINKER_CODE_TO_CODE_RELOCATIONS INTERNAL_LINKER_CODE_TO_CODE_RELOCATIONS, %%entry
    47                              <2>  %endif
    48                              <2> %else
    49                              <2>  %ifidni _CURRENT_SECTION_TYPE, DATA
    50                              <2>   %xdefine INTERNAL_DATA_TO_CODE_RELOCATIONS INTERNAL_DATA_TO_CODE_RELOCATIONS, %%entry
    51                              <2>  %else
    52                              <2>   %xdefine INTERNAL_CODE_TO_CODE_RELOCATIONS INTERNAL_CODE_TO_CODE_RELOCATIONS, %%entry
    53                              <2>  %endif
    54                              <2> %endif
    55                              <2> 	eldstrictcheck
    56                              <2> 	%endmacro
    57                              <2> 
    58                              <2> 	%imacro internaldatarelocation 0-1.nolist -2
    59                              <2> %assign %%entry $ + _CURRENT_SECTION %+ FIXUP + %1
    60                              <2> %if ELDLINKER
    61                              <2>  %ifidni _CURRENT_SECTION_TYPE, DATA
    62                              <2>   %xdefine INTERNAL_LINKER_DATA_TO_DATA_RELOCATIONS INTERNAL_LINKER_DATA_TO_DATA_RELOCATIONS, %%entry
    63                              <2>  %else
    64                              <2>   %xdefine INTERNAL_LINKER_CODE_TO_DATA_RELOCATIONS INTERNAL_LINKER_CODE_TO_DATA_RELOCATIONS, %%entry
    65                              <2>  %endif
    66                              <2> %else
    67                              <2>  %ifidni _CURRENT_SECTION_TYPE, DATA
    68                              <2>   %xdefine INTERNAL_DATA_TO_DATA_RELOCATIONS INTERNAL_DATA_TO_DATA_RELOCATIONS, %%entry
    69                              <2>  %else
    70                              <2>   %xdefine INTERNAL_CODE_TO_DATA_RELOCATIONS INTERNAL_CODE_TO_DATA_RELOCATIONS, %%entry
    71                              <2>  %endif
    72                              <2> %endif
    73                              <2> 	eldstrictcheck
    74                              <2> 	%endmacro
    75                              <2> 
    76                              <2> ; dw INTERNAL_LINKER_CODE_TO_CODE_RELOCATIONS, 0
    77                              <2> ; dw INTERNAL_LINKER_CODE_TO_DATA_RELOCATIONS, 0
    78                              <2> ; dw INTERNAL_LINKER_DATA_TO_CODE_RELOCATIONS, -1
    79                              <2> ; dw INTERNAL_LINKER_DATA_TO_DATA_RELOCATIONS, -1
    80                              <2> ; dw INTERNAL_CODE_TO_CODE_RELOCATIONS, 0
    81                              <2> ; dw INTERNAL_CODE_TO_DATA_RELOCATIONS, 0
    82                              <2> ; dw INTERNAL_DATA_TO_CODE_RELOCATIONS, -1
    83                              <2> ; dw INTERNAL_DATA_TO_DATA_RELOCATIONS, -1
    84                              <2> 
    85                              <2> 
    86                              <2> %define LINK_DATA_RELOCATIONS ""
    87                              <2> %define LINK_LINKER_DATA_RELOCATIONS ""
    88                              <2> %define LINK_DATA_NAMES db ""
    89                              <2> %define LINK_DATA_DETECTION none, none
    90                              <2> 
    91                              <2> %define LINK_OTHER_DATA_RELOCATIONS ""
    92                              <2> %define LINK_OTHER_LINKER_DATA_RELOCATIONS ""
    93                              <2> %define LINK_OTHER_DATA_NAMES db ""
    94                              <2> %define LINK_OTHER_DATA_DETECTION none, none
    95                              <2> 
    96                              <2> %ifndef ELDOTHER
    97                              <2>  %assign ELDOTHER 0
    98                              <2> %endif
    99                              <2> %assign ELDOTHERLINK 0
   100                              <2> 
   101                              <2> 	%imacro otherlinkdatarelocation 1-3.nolist -2, required
   102                              <2> %if ELDOTHER
   103                              <2>  %assign ELDOTHERLINK 1
   104                              <2> %endif
   105                              <2> 	linkdatarelocation %1, %2, %3
   106                              <2> %assign ELDOTHERLINK 0
   107                              <2> 	%endmacro
   108                              <2> 
   109                              <2> 	%imacro linkdatarelocation 1-4.nolist -2, required, single
   110                              <2> %assign %%entry $ + _CURRENT_SECTION %+ FIXUP + %2
   111                              <2> %ifidni %3, required
   112                              <2>  %assign %%optional 0
   113                              <2> %elifidni %3, optional
   114                              <2>  %assign %%optional 100h
   115                              <2>  %if ELDDATA_OPTIONAL_STATUS == 0
   116                              <2>   %assign ELDDATA_OPTIONAL_STATUS 1
   117                              <2>  %elif ELDDATA_OPTIONAL_STATUS == 1
   118                              <2>  %else
   119                              <2>   %error Optional data link not allowed here
   120                              <2>  %endif
   121                              <2> %elifidni %3, PM required
   122                              <2>  %assign %%optional 300h
   123                              <2>  %assign ELDDATA_PMREQUIRED_STATUS 1
   124                              <2>  %if ELDDATA_OPTIONAL_STATUS == 0
   125                              <2>   %assign ELDDATA_OPTIONAL_STATUS 1
   126                              <2>  %elif ELDDATA_OPTIONAL_STATUS == 1
   127                              <2>  %else
   128                              <2>   %error Optional data link not allowed here
   129                              <2>  %endif
   130                              <2> %else
   131                              <2>  %fatal Unknown optional keyword
   132                              <2> %endif
   133                              <2> %ifidni _CURRENT_SECTION_TYPE, DATA
   134                              <2>  %assign %%DATASECTION 1
   135                              <2> %else
   136                              <2>  %assign %%DATASECTION 0
   137                              <2> %endif
   138                              <2> %ifidni %4, single
   139                              <2>  %if ELDDATA_NEXT_STATUS == 1		; after next ?
   140                              <2>   %error Unexpected single data link after next data link
   141                              <2>  %elif ELDDATA_NEXT_STATUS == 2		; after last ?
   142                              <2>   %assign ELDDATA_NEXT_STATUS 3		; note single with next/last present
   143                              <2>  %endif
   144                              <2>  %assign %%next 0
   145                              <2> %elifidni %4, next
   146                              <2>  %if ELDDATA_NEXT_STATUS == 0		; no next/last yet ?
   147                              <2>   %assign ELDDATA_NEXT_STATUS 1		; in next
   148                              <2>  %elif ELDDATA_NEXT_STATUS == 2		; after last ?
   149                              <2>   %assign ELDDATA_NEXT_STATUS 1		; in next
   150                              <2>  %elif ELDDATA_NEXT_STATUS == 3		; after single ?
   151                              <2>   %assign ELDDATA_NEXT_STATUS 1		; in next
   152                              <2>  %elif ELDDATA_NEXT_STATUS == 1		; repeated next ?
   153                              <2>   %if ELDDATA_NEXT_ENTRY != %%entry 	|| ELDDATA_NEXT_SECTION != %%DATASECTION 	|| ELDDATA_NEXT_OTHER != ELDOTHERLINK
   156                              <2>    %error Unexpected next data link
   157                              <2>   %endif
   158                              <2>  %else
   159                              <2>   %error Next data link not allowed here
   160                              <2>  %endif
   161                              <2>  %ifn %%optional
   162                              <2>   %error Next data link only valid as optional or PM required
   163                              <2>  %endif
   164                              <2>  %assign %%next 400h
   165                              <2>  %assign ELDDATA_NEXT_ENTRY %%entry
   166                              <2>  %assign ELDDATA_NEXT_SECTION %%DATASECTION
   167                              <2>  %assign ELDDATA_NEXT_OTHER ELDOTHERLINK
   168                              <2> %elifidni %4, last
   169                              <2>  %if ELDDATA_NEXT_STATUS == 0		; no next/last yet ?
   170                              <2>   %error Next last data link not allowed here
   171                              <2>  %elif ELDDATA_NEXT_STATUS == 2		; after last ?
   172                              <2>   %error Next last data link not allowed here
   173                              <2>  %elif ELDDATA_NEXT_STATUS == 3		; after single ?
   174                              <2>   %error Next last data link not allowed here
   175                              <2>  %elif ELDDATA_NEXT_STATUS == 1		; after next ?
   176                              <2>   %if ELDDATA_NEXT_ENTRY != %%entry 	|| ELDDATA_NEXT_SECTION != %%DATASECTION 	|| ELDDATA_NEXT_OTHER != ELDOTHERLINK
   179                              <2>    %error Unexpected next data link
   180                              <2>   %endif
   181                              <2>   %assign ELDDATA_NEXT_STATUS 2		; note now after last
   182                              <2>  %else
   183                              <2>   %error Next data link not allowed here
   184                              <2>  %endif
   185                              <2>  %assign %%next 800h
   186                              <2>  %assign ELDDATA_NEXT_ENTRY -1
   187                              <2>  %assign ELDDATA_NEXT_SECTION -1
   188                              <2> %else
   189                              <2>  %fatal Unknown next keyword
   190                              <2> %endif
   191                              <2> 	%if ELDOTHERLINK
   192                              <2> %if ELDLINKER
   193                              <2>  %xdefine LINK_OTHER_LINKER_DATA_RELOCATIONS LINK_OTHER_LINKER_DATA_RELOCATIONS, 1 + %%DATASECTION + %%optional + %%next, %%entry, %%name
   194                              <2> %else
   195                              <2>  %xdefine LINK_OTHER_DATA_RELOCATIONS LINK_OTHER_DATA_RELOCATIONS, 1 + %%DATASECTION + %%optional + %%next, %%entry, %%name
   196                              <2> %endif
   197                              <2> 	%else
   198                              <2> %if ELDLINKER
   199                              <2>  %xdefine LINK_LINKER_DATA_RELOCATIONS LINK_LINKER_DATA_RELOCATIONS, 1 + %%DATASECTION + %%optional + %%next, %%entry, %%name
   200                              <2> %else
   201                              <2>  %xdefine LINK_DATA_RELOCATIONS LINK_DATA_RELOCATIONS, 1 + %%DATASECTION + %%optional + %%next, %%entry, %%name
   202                              <2> %endif
   203                              <2> 	%endif
   204                              <2> %defstr %%string %1
   205                              <2> %strlen %%length %%string
   206                              <2> %if %%length > 64
   207                              <2> 	; Could be increased, but mustn't exceed 127 bytes
   208                              <2> 	;  because flag 80h is used to mark optional links
   209                              <2> 	;  that failed to be matched.
   210                              <2>  %error Too long link name: %1
   211                              <2> %endif
   212                              <2> %define LINK_DATA_CHECK %1
   213                              <2> 	%if ELDOTHERLINK
   214                              <2> 	linkdata_detect LINK_OTHER_DATA_DETECTION
   215                              <2> %if LINK_DATA_NEW
   216                              <2>  %xdefine LINK_OTHER_DATA_DETECTION LINK_OTHER_DATA_DETECTION, %1, %%name
   217                              <2> 	hashdef HASH, %%string
   218                              <2>  %xdefine LINK_OTHER_DATA_NAMES 	LINK_OTHER_DATA_NAMES, %%name:, dw _HASH, {counted %%string}
   220                              <2> %else
   221                              <2>  %%name equ LINK_DATA_DUPLICATE
   222                              <2> %endif
   223                              <2> 	%else
   224                              <2> 	linkdata_detect LINK_DATA_DETECTION
   225                              <2> %if LINK_DATA_NEW
   226                              <2>  %xdefine LINK_DATA_DETECTION LINK_DATA_DETECTION, %1, %%name
   227                              <2> 	hashdef HASH, %%string
   228                              <2>  %xdefine LINK_DATA_NAMES 	LINK_DATA_NAMES, %%name:, dw _HASH, {counted %%string}
   230                              <2> %else
   231                              <2>  %%name equ LINK_DATA_DUPLICATE
   232                              <2> %endif
   233                              <2> 	%endif
   234                              <2> 	eldstrictcheck
   235                              <2> 	%endmacro
   236                              <2> 
   237                              <2> 	%imacro linkdata_detect 2-*.nolist
   238                              <2> %assign LINK_DATA_NEW 1
   239                              <2> %rep (%0 - 2) / 2
   240                              <2>  %rotate 2
   241                              <2>  %ifidni %1, LINK_DATA_CHECK
   242                              <2>   %assign LINK_DATA_NEW 0
   243                              <2>   %xdefine LINK_DATA_DUPLICATE %2
   244                              <2>   %exitrep
   245                              <2>  %endif
   246                              <2> %endrep
   247                              <2> 	%endmacro
   248                              <2> 
   249                              <2> 	%imacro link_data_dump_names 1-*.nolist
   250                              <2> %rep %0
   251                              <2> 	%1
   252                              <2>  %rotate 1
   253                              <2> %endrep
   254                              <2> 	%endmacro
   255                              <2> 
   256                              <2> ; dw LINK_LINKER_DATA_RELOCATIONS, 0, 0
   257                              <2> ; dw LINK_DATA_RELOCATIONS, 0, 0
   258                              <2> ; link_data_dump_names ELDCALL_CODE_NAMES
   259                              <2> 
   260                              <2> %endif
    21                              <1> 
    22                              <1> %assign ELDLINKER 0
    23                              <1> 
    24                              <1> [section relocatedzero nobits vstart=0]
    25                              <1> relocatedzero:
    26                              <1> __SECT__
    27                              <1> 
    28                              <1> 	numdef HOUDINI, 1
    29                              <1> 	numdef HOUDINI_CONDITIONAL, 1
    30                              <1> 
    31                              <1> %imacro houdini 0.nolist
    32                              <1> %if _HOUDINI
    33                              <1>  %if _HOUDINI_CONDITIONAL
    34                              <1> reloc	testopt [ss:relocateddata], 100h
    35                              <1> linkdatarelocation options7, -3
    36                              <1> 	jz %%skip
    37                              <1>  %endif
    38                              <1> reloc	testopt [ss:relocateddata], 100h
    39                              <1> linkdatarelocation internalflags6, -3
    40                              <1> 	jz %%skip
    41                              <1> 	int3
    42                              <1> %%skip:
    43                              <1> %endif
    44                              <1> %endmacro
    45                              <1> 
    46                              <1> %define ELDCALL_CODE_RELOCATIONS ""
    47                              <1> %define ELDCALL_LINKER_CODE_RELOCATIONS ""
    48                              <1> %define ELDCALL_CODE_RELOCATIONS_OPTIONAL ""
    49                              <1> %define ELDCALL_LINKER_CODE_RELOCATIONS_OPTIONAL ""
    50                              <1> %define ELDCALL_CODE_NAMES db ""
    51                              <1> %define ELDCALL_CODE_DETECTION none, none
    52                              <1> %assign ELDCALL_OPTIONAL_STATUS 0		; not any seen yet
    53                              <1> %assign ELDCALL_PMREQUIRED_STATUS 0		; not any seen yet
    54                              <1> %assign ELDCALL_NEXT_STATUS 0			; not any seen yet
    55                              <1> %assign ELDCALL_NEXT_ENTRY -1
    56                              <1> 
    57                              <1> 	%imacro extcall 1-3.nolist required, single
    58                              <1> %ifidni _CURRENT_SECTION_TYPE, DATA
    59                              <1>  %error "ELD call cannot be used in ELD data block"
    60                              <1> %endif
    61                              <1> %assign %%entry $ + _CURRENT_SECTION %+ FIXUP
    62                              <1> %ifidni %2, required
    63                              <1>  %assign %%optional 0
    64                              <1> %elifidni %2, optional
    65                              <1>  %assign %%optional 100h
    66                              <1>  %if ELDCALL_OPTIONAL_STATUS == 0
    67                              <1>   %assign ELDCALL_OPTIONAL_STATUS 1
    68                              <1>  %elif ELDCALL_OPTIONAL_STATUS == 1
    69                              <1>  %else
    70                              <1>   %error Optional code link not allowed here
    71                              <1>  %endif
    72                              <1> %elifidni %2, PM required
    73                              <1>  %assign %%optional 300h
    74                              <1>  %assign ELDCALL_PMREQUIRED_STATUS 1
    75                              <1>  %if ELDCALL_OPTIONAL_STATUS == 0
    76                              <1>   %assign ELDCALL_OPTIONAL_STATUS 1
    77                              <1>  %elif ELDCALL_OPTIONAL_STATUS == 1
    78                              <1>  %else
    79                              <1>   %error Optional code link not allowed here
    80                              <1>  %endif
    81                              <1> %else
    82                              <1>  %fatal Unknown optional keyword
    83                              <1> %endif
    84                              <1> %ifidni %3, single
    85                              <1>  %if ELDCALL_NEXT_STATUS == 1		; after next ?
    86                              <1>   %error Unexpected single code link after next code link
    87                              <1>  %elif ELDCALL_NEXT_STATUS == 2		; after last ?
    88                              <1>   %assign ELDCALL_NEXT_STATUS 3		; note single with next/last present
    89                              <1>  %endif
    90                              <1>  %assign %%next 0
    91                              <1> %elifidni %3, next
    92                              <1>  %if ELDCALL_NEXT_STATUS == 0		; no next/last yet ?
    93                              <1>   %assign ELDCALL_NEXT_STATUS 1		; in next
    94                              <1>  %elif ELDCALL_NEXT_STATUS == 2		; after last ?
    95                              <1>   %assign ELDCALL_NEXT_STATUS 1		; in next
    96                              <1>  %elif ELDCALL_NEXT_STATUS == 3		; after single ?
    97                              <1>   %assign ELDCALL_NEXT_STATUS 1		; in next
    98                              <1>  %elif ELDCALL_NEXT_STATUS == 1		; repeated next ?
    99                              <1>   %if ELDCALL_NEXT_ENTRY != %%entry
   100                              <1>    %error Unexpected next code link
   101                              <1>   %endif
   102                              <1>  %else
   103                              <1>   %error Next code link not allowed here
   104                              <1>  %endif
   105                              <1>  %ifn %%optional
   106                              <1>   %error Next code link only valid as optional or PM required
   107                              <1>  %endif
   108                              <1>  %assign %%next 400h
   109                              <1>  %assign ELDCALL_NEXT_ENTRY %%entry
   110                              <1> %elifidni %3, last
   111                              <1>  %if ELDCALL_NEXT_STATUS == 0		; no next/last yet ?
   112                              <1>   %error Next last code link not allowed here
   113                              <1>  %elif ELDCALL_NEXT_STATUS == 2		; after last ?
   114                              <1>   %error Next last code link not allowed here
   115                              <1>  %elif ELDCALL_NEXT_STATUS == 3		; after single ?
   116                              <1>   %error Next last code link not allowed here
   117                              <1>  %elif ELDCALL_NEXT_STATUS == 1		; after next ?
   118                              <1>   %if ELDCALL_NEXT_ENTRY != %%entry
   119                              <1>    %error Unexpected next code link
   120                              <1>   %endif
   121                              <1>   %assign ELDCALL_NEXT_STATUS 2		; note now after last
   122                              <1>  %else
   123                              <1>   %error Next code link not allowed here
   124                              <1>  %endif
   125                              <1>  %assign %%next 800h
   126                              <1>  %assign ELDCALL_NEXT_ENTRY -1
   127                              <1>  %assign ELDCALL_NEXT_SECTION -1
   128                              <1> %else
   129                              <1>  %fatal Unknown next keyword
   130                              <1> %endif
   131                              <1> %if %%next != 400h
   132                              <1> %if 0
   133                              <1> [warning -reloc-rel-word]
   134                              <1> 	call near relocatedzero
   135                              <1> [warning +reloc-rel-word]
   136                              <1> %else
   137                              <1> 	db 0E8h
   138                              <1> reloc	dw relocatedzero
   139                              <1> 	eldstrictcheck
   140                              <1> %endif
   141                              <1> 	jmp strict short %%skipparameter
   142                              <1> 	dw 0
   143                              <1> %%skipparameter:
   144                              <1> %endif
   145                              <1> %if ELDLINKER
   146                              <1>  %xdefine ELDCALL_LINKER_CODE_RELOCATIONS ELDCALL_LINKER_CODE_RELOCATIONS, %%entry, %%name
   147                              <1>  %xdefine ELDCALL_LINKER_CODE_RELOCATIONS_OPTIONAL ELDCALL_LINKER_CODE_RELOCATIONS_OPTIONAL, 1 + %%optional + %%next, %%entry, %%name
   148                              <1> %else
   149                              <1>  %xdefine ELDCALL_CODE_RELOCATIONS ELDCALL_CODE_RELOCATIONS, %%entry, %%name
   150                              <1>  %xdefine ELDCALL_CODE_RELOCATIONS_OPTIONAL ELDCALL_CODE_RELOCATIONS_OPTIONAL, 1 + %%optional + %%next, %%entry, %%name
   151                              <1> %endif
   152                              <1> %defstr %%string %1
   153                              <1> %strlen %%length %%string
   154                              <1> %if %%length > 64
   155                              <1> 	; Could be increased, but mustn't exceed 127 bytes
   156                              <1> 	;  because flag 80h is used to mark optional links
   157                              <1> 	;  that failed to be matched.
   158                              <1>  %error Too long link name: %1
   159                              <1> %endif
   160                              <1> %define ELDCALL_CODE_CHECK %1
   161                              <1> 	linkcode_detect ELDCALL_CODE_DETECTION
   162                              <1> %if ELDCALL_CODE_NEW
   163                              <1>  %xdefine ELDCALL_CODE_DETECTION ELDCALL_CODE_DETECTION, %1, %%name
   164                              <1> 	hashdef HASH, %%string
   165                              <1> %xdefine ELDCALL_CODE_NAMES 	ELDCALL_CODE_NAMES, %%name:, dw _HASH, {counted %%string}
   167                              <1> %else
   168                              <1>  %%name equ ELDCALL_CODE_DUPLICATE
   169                              <1> %endif
   170                              <1> 	%endmacro
   171                              <1> 
   172                              <1> 	%imacro linkcode_detect 2-*.nolist
   173                              <1> %assign ELDCALL_CODE_NEW 1
   174                              <1> %rep (%0 - 2) / 2
   175                              <1>  %rotate 2
   176                              <1>  %ifidni %1, ELDCALL_CODE_CHECK
   177                              <1>   %assign ELDCALL_CODE_NEW 0
   178                              <1>   %xdefine ELDCALL_CODE_DUPLICATE %2
   179                              <1>   %exitrep
   180                              <1>  %endif
   181                              <1> %endrep
   182                              <1> 	%endmacro
   183                              <1> 
   184                              <1> 
   185                              <1> %define ELDCALL_CALLCALL_LIST none
   186                              <1> %define ELDCALL_CALLCALL_PROCESSED_PRIOR ""
   187                              <1> 
   188                              <1> 	%imacro extcallcall 1.nolist
   189                              <1> 	call %1
   190                              <1> %xdefine ELDCALL_CALLCALL_LIST ELDCALL_CALLCALL_LIST, %1
   191                              <1> 	%endmacro
   192                              <1> 
   193                              <1> %assign ELDCALLCALL_DUMPED 0
   194                              <1> 
   195                              <1> 	%imacro eldcall_dump_callcall 1-*.nolist
   196                              <1> %xdefine ELDCALL_CALLCALL_PROCESSED ELDCALL_CALLCALL_PROCESSED_PRIOR
   197                              <1>  %rep %0 - 1
   198                              <1>   %rotate 1
   199                              <1>   %define ELDCALL_CHECK %1
   200                              <1> 	eldcall_callcall_detect ELDCALL_CALLCALL_PROCESSED
   201                              <1>   %if ELDCALL_NEW
   202                              <1>    %xdefine ELDCALL_CALLCALL_PROCESSED ELDCALL_CALLCALL_PROCESSED, %1
   203                              <1> 	align 8, nop
   204                              <1> %1:
   205                              <1> 	extcall %1
   206                              <1> 	retn
   207                              <1>   %endif
   208                              <1>  %endrep
   209                              <1> %assign ELDCALLCALL_DUMPED 1
   210                              <1> %define ELDCALL_CALLCALL_LIST none
   211                              <1> 	%endmacro
   212                              <1> 
   213                              <1> 	%imacro eldcall_new_callcall 0.nolist
   214                              <1> %if ELDCALLCALL_DUMPED
   215                              <1>  %xdefine ELDCALL_CALLCALL_PROCESSED_PRIOR   ELDCALL_CALLCALL_PROCESSED_PRIOR, ELDCALL_CALLCALL_PROCESSED
   217                              <1>  %assign ELDCALLCALL_DUMPED 0
   218                              <1>  %define ELDCALL_CALLCALL_LIST none
   219                              <1> %endif
   220                              <1> 	%endmacro
   221                              <1> 
   222                              <1> 	%imacro eldcall_callcall_detect 1-*.nolist
   223                              <1> %assign ELDCALL_NEW 1
   224                              <1> %rep %0
   225                              <1>  %ifidni %1, ELDCALL_CHECK
   226                              <1>   %assign ELDCALL_NEW 0
   227                              <1>   %exitrep
   228                              <1>  %endif
   229                              <1>  %rotate 1
   230                              <1> %endrep
   231                              <1> 	%endmacro
   232                              <1> 
   233                              <1> 	%imacro eldcall_dump_names 1-*.nolist
   234                              <1> %rep %0
   235                              <1> 	%1
   236                              <1>  %rotate 1
   237                              <1> %endrep
   238                              <1> 	%endmacro
   239                              <1> 
   240                              <1> ; eldcall_dump_callcall ELDCALL_CALLCALL_LIST
   241                              <1> ; if using optional code links:
   242                              <1> ;  dw ELDCALL_LINKER_CODE_RELOCATIONS_OPTIONAL, 0
   243                              <1> ;  dw ELDCALL_CODE_RELOCATIONS_OPTIONAL, 0
   244                              <1> ; if not using optional code links:
   245                              <1> ;  dw ELDCALL_LINKER_CODE_RELOCATIONS, 0, 0
   246                              <1> ;  dw ELDCALL_CODE_RELOCATIONS, 0, 0
   247                              <1> ; eldcall_dump_names ELDCALL_CODE_NAMES
   248                              <1> 
   249                              <1> %endif
     9                                  %include "elddata.mac"
     1                              <1> %if 0
     2                              <1> 
     3                              <1> Extensions for lDebug data relocation macros
     4                              <1> 
     5                              <1> Copyright (C) 2008-2024 E. C. Masloch
     6                              <1> 
     7                              <1> Usage of the works is permitted provided that this
     8                              <1> instrument is retained with the works, so that any entity
     9                              <1> that uses the works is notified of this instrument.
    10                              <1> 
    11                              <1> DISCLAIMER: THE WORKS ARE WITHOUT WARRANTY.
    12                              <1> 
    13                              <1> %endif
    14                              <1> 
    15                              <1> %ifndef ELDDATA_MAC
    16                              <1> %define ELDDATA_MAC 1
    17                              <1> 
    18                              <1> %include "lmacros3.mac"
    19                              <1> %include "nasmhash.mac"
    20                              <1> %include "eldcheck.mac"
    21                              <1> 
    22                              <1> 
    23                              <1> %assign ELDLINKER 0
    24                              <1> 
    25                              <1> %define INTERNAL_CODE_TO_CODE_RELOCATIONS ""
    26                              <1> %define INTERNAL_CODE_TO_DATA_RELOCATIONS ""
    27                              <1> %define INTERNAL_DATA_TO_CODE_RELOCATIONS ""
    28                              <1> %define INTERNAL_DATA_TO_DATA_RELOCATIONS ""
    29                              <1> %define INTERNAL_LINKER_CODE_TO_CODE_RELOCATIONS ""
    30                              <1> %define INTERNAL_LINKER_CODE_TO_DATA_RELOCATIONS ""
    31                              <1> %define INTERNAL_LINKER_DATA_TO_CODE_RELOCATIONS ""
    32                              <1> %define INTERNAL_LINKER_DATA_TO_DATA_RELOCATIONS ""
    33                              <1> %assign ELDDATA_OPTIONAL_STATUS 0		; not any seen yet
    34                              <1> %assign ELDDATA_PMREQUIRED_STATUS 0		; not any seen yet
    35                              <1> %assign ELDDATA_NEXT_STATUS 0			; not any seen yet
    36                              <1> %assign ELDDATA_NEXT_ENTRY -1
    37                              <1> %assign ELDDATA_NEXT_SECTION -1
    38                              <1> %assign ELDDATA_NEXT_OTHER -1
    39                              <1> 
    40                              <1> 	%imacro internalcoderelocation 0-1.nolist -2
    41                              <1> %assign %%entry $ + _CURRENT_SECTION %+ FIXUP + %1
    42                              <1> %if ELDLINKER
    43                              <1>  %ifidni _CURRENT_SECTION_TYPE, DATA
    44                              <1>   %xdefine INTERNAL_LINKER_DATA_TO_CODE_RELOCATIONS INTERNAL_LINKER_DATA_TO_CODE_RELOCATIONS, %%entry
    45                              <1>  %else
    46                              <1>   %xdefine INTERNAL_LINKER_CODE_TO_CODE_RELOCATIONS INTERNAL_LINKER_CODE_TO_CODE_RELOCATIONS, %%entry
    47                              <1>  %endif
    48                              <1> %else
    49                              <1>  %ifidni _CURRENT_SECTION_TYPE, DATA
    50                              <1>   %xdefine INTERNAL_DATA_TO_CODE_RELOCATIONS INTERNAL_DATA_TO_CODE_RELOCATIONS, %%entry
    51                              <1>  %else
    52                              <1>   %xdefine INTERNAL_CODE_TO_CODE_RELOCATIONS INTERNAL_CODE_TO_CODE_RELOCATIONS, %%entry
    53                              <1>  %endif
    54                              <1> %endif
    55                              <1> 	eldstrictcheck
    56                              <1> 	%endmacro
    57                              <1> 
    58                              <1> 	%imacro internaldatarelocation 0-1.nolist -2
    59                              <1> %assign %%entry $ + _CURRENT_SECTION %+ FIXUP + %1
    60                              <1> %if ELDLINKER
    61                              <1>  %ifidni _CURRENT_SECTION_TYPE, DATA
    62                              <1>   %xdefine INTERNAL_LINKER_DATA_TO_DATA_RELOCATIONS INTERNAL_LINKER_DATA_TO_DATA_RELOCATIONS, %%entry
    63                              <1>  %else
    64                              <1>   %xdefine INTERNAL_LINKER_CODE_TO_DATA_RELOCATIONS INTERNAL_LINKER_CODE_TO_DATA_RELOCATIONS, %%entry
    65                              <1>  %endif
    66                              <1> %else
    67                              <1>  %ifidni _CURRENT_SECTION_TYPE, DATA
    68                              <1>   %xdefine INTERNAL_DATA_TO_DATA_RELOCATIONS INTERNAL_DATA_TO_DATA_RELOCATIONS, %%entry
    69                              <1>  %else
    70                              <1>   %xdefine INTERNAL_CODE_TO_DATA_RELOCATIONS INTERNAL_CODE_TO_DATA_RELOCATIONS, %%entry
    71                              <1>  %endif
    72                              <1> %endif
    73                              <1> 	eldstrictcheck
    74                              <1> 	%endmacro
    75                              <1> 
    76                              <1> ; dw INTERNAL_LINKER_CODE_TO_CODE_RELOCATIONS, 0
    77                              <1> ; dw INTERNAL_LINKER_CODE_TO_DATA_RELOCATIONS, 0
    78                              <1> ; dw INTERNAL_LINKER_DATA_TO_CODE_RELOCATIONS, -1
    79                              <1> ; dw INTERNAL_LINKER_DATA_TO_DATA_RELOCATIONS, -1
    80                              <1> ; dw INTERNAL_CODE_TO_CODE_RELOCATIONS, 0
    81                              <1> ; dw INTERNAL_CODE_TO_DATA_RELOCATIONS, 0
    82                              <1> ; dw INTERNAL_DATA_TO_CODE_RELOCATIONS, -1
    83                              <1> ; dw INTERNAL_DATA_TO_DATA_RELOCATIONS, -1
    84                              <1> 
    85                              <1> 
    86                              <1> %define LINK_DATA_RELOCATIONS ""
    87                              <1> %define LINK_LINKER_DATA_RELOCATIONS ""
    88                              <1> %define LINK_DATA_NAMES db ""
    89                              <1> %define LINK_DATA_DETECTION none, none
    90                              <1> 
    91                              <1> %define LINK_OTHER_DATA_RELOCATIONS ""
    92                              <1> %define LINK_OTHER_LINKER_DATA_RELOCATIONS ""
    93                              <1> %define LINK_OTHER_DATA_NAMES db ""
    94                              <1> %define LINK_OTHER_DATA_DETECTION none, none
    95                              <1> 
    96                              <1> %ifndef ELDOTHER
    97                              <1>  %assign ELDOTHER 0
    98                              <1> %endif
    99                              <1> %assign ELDOTHERLINK 0
   100                              <1> 
   101                              <1> 	%imacro otherlinkdatarelocation 1-3.nolist -2, required
   102                              <1> %if ELDOTHER
   103                              <1>  %assign ELDOTHERLINK 1
   104                              <1> %endif
   105                              <1> 	linkdatarelocation %1, %2, %3
   106                              <1> %assign ELDOTHERLINK 0
   107                              <1> 	%endmacro
   108                              <1> 
   109                              <1> 	%imacro linkdatarelocation 1-4.nolist -2, required, single
   110                              <1> %assign %%entry $ + _CURRENT_SECTION %+ FIXUP + %2
   111                              <1> %ifidni %3, required
   112                              <1>  %assign %%optional 0
   113                              <1> %elifidni %3, optional
   114                              <1>  %assign %%optional 100h
   115                              <1>  %if ELDDATA_OPTIONAL_STATUS == 0
   116                              <1>   %assign ELDDATA_OPTIONAL_STATUS 1
   117                              <1>  %elif ELDDATA_OPTIONAL_STATUS == 1
   118                              <1>  %else
   119                              <1>   %error Optional data link not allowed here
   120                              <1>  %endif
   121                              <1> %elifidni %3, PM required
   122                              <1>  %assign %%optional 300h
   123                              <1>  %assign ELDDATA_PMREQUIRED_STATUS 1
   124                              <1>  %if ELDDATA_OPTIONAL_STATUS == 0
   125                              <1>   %assign ELDDATA_OPTIONAL_STATUS 1
   126                              <1>  %elif ELDDATA_OPTIONAL_STATUS == 1
   127                              <1>  %else
   128                              <1>   %error Optional data link not allowed here
   129                              <1>  %endif
   130                              <1> %else
   131                              <1>  %fatal Unknown optional keyword
   132                              <1> %endif
   133                              <1> %ifidni _CURRENT_SECTION_TYPE, DATA
   134                              <1>  %assign %%DATASECTION 1
   135                              <1> %else
   136                              <1>  %assign %%DATASECTION 0
   137                              <1> %endif
   138                              <1> %ifidni %4, single
   139                              <1>  %if ELDDATA_NEXT_STATUS == 1		; after next ?
   140                              <1>   %error Unexpected single data link after next data link
   141                              <1>  %elif ELDDATA_NEXT_STATUS == 2		; after last ?
   142                              <1>   %assign ELDDATA_NEXT_STATUS 3		; note single with next/last present
   143                              <1>  %endif
   144                              <1>  %assign %%next 0
   145                              <1> %elifidni %4, next
   146                              <1>  %if ELDDATA_NEXT_STATUS == 0		; no next/last yet ?
   147                              <1>   %assign ELDDATA_NEXT_STATUS 1		; in next
   148                              <1>  %elif ELDDATA_NEXT_STATUS == 2		; after last ?
   149                              <1>   %assign ELDDATA_NEXT_STATUS 1		; in next
   150                              <1>  %elif ELDDATA_NEXT_STATUS == 3		; after single ?
   151                              <1>   %assign ELDDATA_NEXT_STATUS 1		; in next
   152                              <1>  %elif ELDDATA_NEXT_STATUS == 1		; repeated next ?
   153                              <1>   %if ELDDATA_NEXT_ENTRY != %%entry 	|| ELDDATA_NEXT_SECTION != %%DATASECTION 	|| ELDDATA_NEXT_OTHER != ELDOTHERLINK
   156                              <1>    %error Unexpected next data link
   157                              <1>   %endif
   158                              <1>  %else
   159                              <1>   %error Next data link not allowed here
   160                              <1>  %endif
   161                              <1>  %ifn %%optional
   162                              <1>   %error Next data link only valid as optional or PM required
   163                              <1>  %endif
   164                              <1>  %assign %%next 400h
   165                              <1>  %assign ELDDATA_NEXT_ENTRY %%entry
   166                              <1>  %assign ELDDATA_NEXT_SECTION %%DATASECTION
   167                              <1>  %assign ELDDATA_NEXT_OTHER ELDOTHERLINK
   168                              <1> %elifidni %4, last
   169                              <1>  %if ELDDATA_NEXT_STATUS == 0		; no next/last yet ?
   170                              <1>   %error Next last data link not allowed here
   171                              <1>  %elif ELDDATA_NEXT_STATUS == 2		; after last ?
   172                              <1>   %error Next last data link not allowed here
   173                              <1>  %elif ELDDATA_NEXT_STATUS == 3		; after single ?
   174                              <1>   %error Next last data link not allowed here
   175                              <1>  %elif ELDDATA_NEXT_STATUS == 1		; after next ?
   176                              <1>   %if ELDDATA_NEXT_ENTRY != %%entry 	|| ELDDATA_NEXT_SECTION != %%DATASECTION 	|| ELDDATA_NEXT_OTHER != ELDOTHERLINK
   179                              <1>    %error Unexpected next data link
   180                              <1>   %endif
   181                              <1>   %assign ELDDATA_NEXT_STATUS 2		; note now after last
   182                              <1>  %else
   183                              <1>   %error Next data link not allowed here
   184                              <1>  %endif
   185                              <1>  %assign %%next 800h
   186                              <1>  %assign ELDDATA_NEXT_ENTRY -1
   187                              <1>  %assign ELDDATA_NEXT_SECTION -1
   188                              <1> %else
   189                              <1>  %fatal Unknown next keyword
   190                              <1> %endif
   191                              <1> 	%if ELDOTHERLINK
   192                              <1> %if ELDLINKER
   193                              <1>  %xdefine LINK_OTHER_LINKER_DATA_RELOCATIONS LINK_OTHER_LINKER_DATA_RELOCATIONS, 1 + %%DATASECTION + %%optional + %%next, %%entry, %%name
   194                              <1> %else
   195                              <1>  %xdefine LINK_OTHER_DATA_RELOCATIONS LINK_OTHER_DATA_RELOCATIONS, 1 + %%DATASECTION + %%optional + %%next, %%entry, %%name
   196                              <1> %endif
   197                              <1> 	%else
   198                              <1> %if ELDLINKER
   199                              <1>  %xdefine LINK_LINKER_DATA_RELOCATIONS LINK_LINKER_DATA_RELOCATIONS, 1 + %%DATASECTION + %%optional + %%next, %%entry, %%name
   200                              <1> %else
   201                              <1>  %xdefine LINK_DATA_RELOCATIONS LINK_DATA_RELOCATIONS, 1 + %%DATASECTION + %%optional + %%next, %%entry, %%name
   202                              <1> %endif
   203                              <1> 	%endif
   204                              <1> %defstr %%string %1
   205                              <1> %strlen %%length %%string
   206                              <1> %if %%length > 64
   207                              <1> 	; Could be increased, but mustn't exceed 127 bytes
   208                              <1> 	;  because flag 80h is used to mark optional links
   209                              <1> 	;  that failed to be matched.
   210                              <1>  %error Too long link name: %1
   211                              <1> %endif
   212                              <1> %define LINK_DATA_CHECK %1
   213                              <1> 	%if ELDOTHERLINK
   214                              <1> 	linkdata_detect LINK_OTHER_DATA_DETECTION
   215                              <1> %if LINK_DATA_NEW
   216                              <1>  %xdefine LINK_OTHER_DATA_DETECTION LINK_OTHER_DATA_DETECTION, %1, %%name
   217                              <1> 	hashdef HASH, %%string
   218                              <1>  %xdefine LINK_OTHER_DATA_NAMES 	LINK_OTHER_DATA_NAMES, %%name:, dw _HASH, {counted %%string}
   220                              <1> %else
   221                              <1>  %%name equ LINK_DATA_DUPLICATE
   222                              <1> %endif
   223                              <1> 	%else
   224                              <1> 	linkdata_detect LINK_DATA_DETECTION
   225                              <1> %if LINK_DATA_NEW
   226                              <1>  %xdefine LINK_DATA_DETECTION LINK_DATA_DETECTION, %1, %%name
   227                              <1> 	hashdef HASH, %%string
   228                              <1>  %xdefine LINK_DATA_NAMES 	LINK_DATA_NAMES, %%name:, dw _HASH, {counted %%string}
   230                              <1> %else
   231                              <1>  %%name equ LINK_DATA_DUPLICATE
   232                              <1> %endif
   233                              <1> 	%endif
   234                              <1> 	eldstrictcheck
   235                              <1> 	%endmacro
   236                              <1> 
   237                              <1> 	%imacro linkdata_detect 2-*.nolist
   238                              <1> %assign LINK_DATA_NEW 1
   239                              <1> %rep (%0 - 2) / 2
   240                              <1>  %rotate 2
   241                              <1>  %ifidni %1, LINK_DATA_CHECK
   242                              <1>   %assign LINK_DATA_NEW 0
   243                              <1>   %xdefine LINK_DATA_DUPLICATE %2
   244                              <1>   %exitrep
   245                              <1>  %endif
   246                              <1> %endrep
   247                              <1> 	%endmacro
   248                              <1> 
   249                              <1> 	%imacro link_data_dump_names 1-*.nolist
   250                              <1> %rep %0
   251                              <1> 	%1
   252                              <1>  %rotate 1
   253                              <1> %endrep
   254                              <1> 	%endmacro
   255                              <1> 
   256                              <1> ; dw LINK_LINKER_DATA_RELOCATIONS, 0, 0
   257                              <1> ; dw LINK_DATA_RELOCATIONS, 0, 0
   258                              <1> ; link_data_dump_names ELDCALL_CODE_NAMES
   259                              <1> 
   260                              <1> %endif
    10                                  
    11                                  	numdef DEBUG, 1
    12                                  	numdef BOOT, 0
    13                                  
    14                                  %assign _CATCHINT0C 0
    15                                  %assign _CATCHINT0D 0
    16                                  %assign _CATCHINTFAULTCOND 0
    17                                  %assign _LOADER 0
    18                                  %assign _DEBUG_COND 1
    19                                  %assign _DELAY_BEFORE_BP 0
    20                                  %assign _DHIGHLIGHT 0
    21                                  %assign _GETLINEHIGHLIGHT 0
    22                                  %assign _IMMASM 0
    23                                  %assign _INPUT_FILE_BOOT 0
    24                                  %assign _INPUT_FILE_HANDLES 0
    25                                  %assign _MS_0RANGE_COMPAT 0
    26                                  %assign _PM 0
    27                                  %assign _RH 0
    28                                  %assign _SYMBOLIC 0
    29                                  %assign _VXCHG 0
    30                                  %include "options.mac"
     1                              <1> 
     2                              <1> %if 0
     3                              <1> 
     4                              <1> lDebug options and internal flags
     5                              <1> 
     6                              <1> Copyright (C) 2008-2025 E. C. Masloch
     7                              <1> 
     8                              <1> Usage of the works is permitted provided that this
     9                              <1> instrument is retained with the works, so that any entity
    10                              <1> that uses the works is notified of this instrument.
    11                              <1> 
    12                              <1> DISCLAIMER: THE WORKS ARE WITHOUT WARRANTY.
    13                              <1> 
    14                              <1> %endif
    15                              <1> 
    16                              <1> 
    17                              <1> dispregs32	equ	  1	; RX: 32-bit register display (R, T/P/G)
    18                              <1> traceints	equ	  2	; TM: trace into interrupts (T)
    19                              <1> cpdepchars	equ	  4	; allow dumping of CP-dependent characters (D, DX)
    20                              <1> fakeindos	equ	  8	; always assume InDOS flag non-zero (all)
    21                              <1> nonpagingdevice	equ	 10h	; disallow paged output with [more] prompt (all exc. P, T)
    22                              <1> 	; This option was never used anywhere:
    23                              <1> ; pagingdevice	equ	 20h	; allow paged output with [more] prompt (all exc. P, T)
    24                              <1> 				; paged output is by default on if the output device is StdOut, else off
    25                              <1> hexrn		equ	 40h	; display raw hexadecimal content of FPU registers (RN)
    26                              <1> ;novdd		equ	 80h	; don't use a registered NTVDM VDD (L, W)
    27                              <1> nondospaging	equ	100h	; paging: don't use DOS for input when waiting for a key
    28                              <1> opt1_86mnohlt	equ	200h	; (86 Mode:) HLT doesn't work, don't use it
    29                              <1> biosidles	equ	400h	; don't idle with HLT or Int2F.1680, only call BIOS Int16.00
    30                              <1> opt_usegetinput	equ	800h	; use getinput for int 21h interactive input
    31                              <1> use_si_units	equ    1000h	; in disp_*_size use SI units (kB = 1000, etc)
    32                              <1> use_jedec_units	equ    2000h	; in disp_*_size use JEDEC units (kB = 1024)
    33                              <1> enable_serial	equ    4000h	; enable serial I/O (preferred over DOS or BIOS terminal)
    34                              <1> int8_disable_serial equ	   8000h	; disable serial I/O when breaking due to intr8
    35                              <1> gg_do_not_skip_bp equ	 1_0000h	; gg: do not skip a breakpoint (bb or gg)
    36                              <1> gg_no_autorepeat equ	 2_0000h	; gg: do not auto-repeat
    37                              <1> tp_do_not_skip_bp equ	 4_0000h	; T/TP/P: do not skip a (bb) breakpoint
    38                              <1> gg_bb_hit_no_repeat equ	 8_0000h	; gg: do not auto-repeat after bb hit
    39                              <1> tp_bb_hit_no_repeat equ	10_0000h	; T/TP/P: do not auto-repeat after bb hit
    40                              <1> gg_unexpected_no_repeat equ 20_0000h	; gg: do not auto-repeat after unexpectedinterrupt
    41                              <1> tp_unexpected_no_repeat equ 40_0000h	; T/TP/P
    42                              <1> ss_no_dump:		equ 80_0000h
    43                              <1> %if _SYMBOLIC
    44                              <1> dd_no_blanks_sym:	equ 100_0000h
    45                              <1> zz_no_pm_xms:		equ 200_0000h
    46                              <1> %endif
    47                              <1> rr_disasm_no_rept:	equ 1000_0000h
    48                              <1> rr_disasm_no_show:	equ 2000_0000h
    49                              <1> opt_cmdline_quiet_input:equ 4000_0000h
    50                              <1> opt_cmdline_quiet_output:equ 8000_0000h
    51                              <1> %if _SYMBOLIC
    52                              <1> DEFAULTOPTIONS	equ zz_no_pm_xms
    53                              <1> %else
    54                              <1> DEFAULTOPTIONS	equ 0
    55                              <1> %endif
    56                              <1> 
    57                              <1> 
    58                              <1> opt2_db_header:		equ 1
    59                              <1> opt2_db_trailer:	equ 2
    60                              <1> opt2_dw_header:		equ 10h
    61                              <1> opt2_dw_trailer:	equ 20h
    62                              <1> opt2_dd_header:		equ 100h
    63                              <1> opt2_dd_trailer:	equ 200h
    64                              <1> opt2_getinput_dpmi:	equ 800h
    65                              <1> opt2_hh_compat:		equ 1000h
    66                              <1> opt2_getc_idle:		equ 2000h
    67                              <1> opt2_getc_idle_dpmi:	equ 4000h
    68                              <1> opt2_re_cancel_tpg:	equ 8000h
    69                              <1> opt2_nn_compat:		equ 1_0000h
    70                              <1> opt2_nn_capitalise:	equ 2_0000h
    71                              <1> %if _MS_0RANGE_COMPAT
    72                              <1> opt2_0range_compat:	equ 4_0000h
    73                              <1> %endif
    74                              <1> opt2_rr16_compat:	equ 8_0000h
    75                              <1> opt2_r_prompt_compat:	equ 10_0000h
    76                              <1> opt2_r_separate:	equ 20_0000h
    77                              <1> opt2_r_linebreak_always:equ 40_0000h
    78                              <1> opt2_dpminohlt:		equ 8000_0000h	; DPMI doesn't like hlt
    79                              <1> DEFAULTOPTIONS2	equ opt2_dw_header | opt2_dd_header | opt2_getc_idle_dpmi | opt2_dpminohlt
    80                              <1> 
    81                              <1> 
    82                              <1> opt3_tt_no_paging:	equ 1
    83                              <1> opt3_tp_no_paging:	equ 2
    84                              <1> opt3_pp_no_paging:	equ 4
    85                              <1> opt3_gg_no_paging:	equ 8
    86                              <1> opt3_silence_paging_set:equ 100h
    87                              <1> opt3_silence_paging_on:	equ 200h
    88                              <1> opt3_paging_rc:		equ 1000h
    89                              <1> opt3_paging_yy:		equ 2000h
    90                              <1> opt3_paging_re:		equ 4000h
    91                              <1> opt3_r_highlight_diff:	equ 10000h
    92                              <1> opt3_r_highlight_dumb:	equ 20000h
    93                              <1> opt3_r_highlight_full:	equ 40000h
    94                              <1> opt3_r_highlight_eip:	equ 80000h
    95                              <1> %if _PM
    96                              <1> opt3_ss_b_bit_set:	equ   10_0000h
    97                              <1>  %if _BREAK_INSTALLDPMI
    98                              <1> opt3_break_installdpmi:	equ   20_0000h
    99                              <1>  %endif
   100                              <1> %endif
   101                              <1> %if _DHIGHLIGHT
   102                              <1> opt3_d_highlight:	equ   80_0000h
   103                              <1> %endif
   104                              <1> %if _GETLINEHIGHLIGHT
   105                              <1> opt3_getline_highlight:	equ  100_0000h
   106                              <1> %endif
   107                              <1> opt3_no_idle_2F:	equ  200_0000h
   108                              <1> %if _DELAY_BEFORE_BP
   109                              <1> opt3_delay_before_bp:	equ  400_0000h
   110                              <1> %endif
   111                              <1> opt3_no_call_amis:	equ  800_0000h
   112                              <1> opt3_disable_autorepeat:equ 1000_0000h
   113                              <1> opt3_check_ctrlc_keyb:	equ 2000_0000h
   114                              <1> opt3_check_ctrlc_0bh:	equ 4000_0000h
   115                              <1> opt3_tsr_quit_leave_tf:	equ 8000_0000h
   116                              <1> DEFAULTOPTIONS3	equ opt3_tt_no_paging | opt3_tp_no_paging 		| opt3_pp_no_paging | opt3_gg_no_paging 		| opt3_check_ctrlc_keyb | opt3_check_ctrlc_0bh
   119                              <1> 
   120                              <1> 
   121                              <1> opt4_int_2F_hook:	equ 2
   122                              <1> opt4_int_08_hook:	equ 4
   123                              <1> opt4_int_2D_hook:	equ 8
   124                              <1> %if _CATCHINTFAULTCOND
   125                              <1> opt4_int_fault_hook:	equ 10h
   126                              <1> %endif
   127                              <1> opt4_int_serial_force:	equ 1_0000h
   128                              <1> opt4_int_2F_force:	equ 2_0000h
   129                              <1> opt4_int_08_force:	equ 4_0000h
   130                              <1> opt4_int_2D_force:	equ 8_0000h
   131                              <1> %if _CATCHINT0D
   132                              <1> opt4_int_0D_force:	equ   10_0000h
   133                              <1> %endif
   134                              <1> %if _CATCHINT0C
   135                              <1> opt4_int_0C_force:	equ   20_0000h
   136                              <1> %endif
   137                              <1> opt4_int_00_force:	equ  100_0000h
   138                              <1> opt4_int_01_force:	equ  200_0000h
   139                              <1> opt4_int_03_force:	equ  400_0000h
   140                              <1> opt4_int_06_force:	equ  800_0000h
   141                              <1> opt4_int_18_force:	equ 1000_0000h
   142                              <1> opt4_int_19_force:	equ 2000_0000h
   143                              <1> opt4_int_09_force:	equ 4000_0000h	; not used at the same time as 15h
   144                              <1> opt4_int_15_force:	equ 4000_0000h	; not used at the same time as 09h
   145                              <1> opt4_int_07_force:	equ 8000_0000h
   146                              <1> DEFAULTOPTIONS4 equ opt4_int_2F_hook
   147                              <1> 
   148                              <1> 
   149                              <1> %if _VXCHG
   150                              <1> opt6_vv_mode:		equ 1
   151                              <1> opt6_vv_keep:		equ 2
   152                              <1> opt6_vv_int16:		equ 10h
   153                              <1>  %if _VXCHG_DEFAULT_ON
   154                              <1> DEFAULTOPTIONS6 equ opt6_share_serial_irq | opt6_vv_mode
   155                              <1>  %else
   156                              <1> DEFAULTOPTIONS6 equ opt6_share_serial_irq
   157                              <1>  %endif
   158                              <1> %else
   159                              <1> DEFAULTOPTIONS6 equ opt6_share_serial_irq
   160                              <1> %endif
   161                              <1> %if _DEBUG
   162                              <1> opt6_debug_exception_late:	equ  20h
   163                              <1> opt6_debug_exception_early:	equ  40h
   164                              <1>  %if _DEBUG_COND
   165                              <1> opt6_debug_exception:	equ  80h
   166                              <1> opt6_debug_mode:	equ 100h
   167                              <1>  %endif
   168                              <1> %endif
   169                              <1> opt6_bios_output:	equ 200h
   170                              <1> opt6_flat_binary:	equ 400h
   171                              <1> opt6_big_stack:		equ 800h
   172                              <1> opt6_40_columns:	equ 1000h
   173                              <1> opt6_40_indent_odd:	equ 2000h
   174                              <1> opt6_40_dash:		equ 4000h
   175                              <1> opt6_share_serial_irq:	equ 1_0000h
   176                              <1> opt6_serial_EOI_call:	equ 2_0000h
   177                              <1> %if _RH
   178                              <1> opt6_rh_mode:		equ 10_0000h
   179                              <1> %endif
   180                              <1> %if _DEBUG
   181                              <1> opt6_debug_putrunint_early:	equ  40_0000h
   182                              <1>  %if _DEBUG_COND
   183                              <1> opt6_debug_putrunint:		equ  80_0000h
   184                              <1>  %endif
   185                              <1> %endif
   186                              <1> opt6_bios_io:		equ 100_0000h
   187                              <1> opt6_immasm_display_uu:	equ 200_0000h
   188                              <1> opt6_immasm_debug:	equ 400_0000h
   189                              <1> opt6_immasm_flag:	equ 800_0000h
   190                              <1> opt6_immasm_nobranch:	equ 1000_0000h
   191                              <1> opt6_r_flags_style2:	equ 2000_0000h
   192                              <1> opt6_r_flags_style3:	equ 4000_0000h
   193                              <1> opt6_r_linebreak_conditional:	equ 8000_0000h
   194                              <1> 
   195                              <1> 
   196                              <1> DEFAULTOPTIONS7 equ opt7_no_tsr_ll
   197                              <1> opt7_no_free_oneshot_eld:	equ 1
   198                              <1> opt7_debug_optional_link:	equ 2
   199                              <1> opt7_quiet_install:		equ 4
   200                              <1> opt7_quick_run:			equ 8
   201                              <1> opt7_houdini:			equ 100h
   202                              <1> opt7_debug_run:			equ 200h
   203                              <1> opt7_no_ensure:			equ 1000h
   204                              <1> opt7_no_tsr_ll:			equ 2000h
   205                              <1> 
   206                              <1> 
   207                              <1> oldpacket	equ	  1	; Int25/Int26 packet method available (L, W)
   208                              <1> newpacket	equ	  2	; Int21.7305 packet method available (L, W)
   209                              <1> ntpacket	equ	  4	; VDD registered and usable (L, W)
   210                              <1> pagedcommand	equ	  8	; allows paging in puts
   211                              <1> notstdinput	equ	 10h	; DEBUG's StdIn isn't a device with StdIn bit (is file or other device)
   212                              <1> inputfile	equ	 20h	; DEBUG's StdIn is a file, notstdinput also set
   213                              <1> notstdoutput	equ	 40h	; DEBUG's StdOut isn't a device with StdOut bit (is file or other device)
   214                              <1> outputfile	equ	  80h	; DEBUG's StdOut is a file, notstdoutput also set
   215                              <1> hooked2F	equ	 100h	; Int2F hooked
   216                              <1> nohook2F	equ	 200h	; don't hook Int2F.1687 (required for Win9x, DosEmu?)
   217                              <1> unused_dif1_dpminohlt equ 400h	; DPMI doesn't like hlt
   218                              <1> protectedmode	equ	 800h	; in (DPMI) protected mode
   219                              <1> debuggeeA20	equ	1000h	; state of debuggee's A20
   220                              <1> debuggerA20	equ	2000h	; state of debugger's A20 (will be on if possible)
   221                              <1> nodosloaded	equ	4000h	; No DOS loaded currently (Boot loader mode)
   222                              <1> has386		equ	8000h	; CPU is a 386
   223                              <1> usecharcounter	equ    1_0000h	; don't reset charcounter between calls to puts
   224                              <1> runningnt	equ    2_0000h	; running in NTVDM
   225                              <1> canswitchmode	equ    4_0000h	; can switch modes (auxbuff large enough, DPMI mode switch set up)
   226                              <1> modeswitched	equ    8_0000h	; switched mode (now in the mode that we weren't entered in)
   227                              <1> promptwaiting	equ   10_0000h	; puts: any more output needs to display a prompt first
   228                              <1> switchbuffer	equ   20_0000h	; mode switch needs a buffer (auxbuff)
   229                              <1> tsrmode		equ   40_0000h	; in TSR mode; DPI and DPP not valid
   230                              <1> attachedterm	equ   80_0000h	; the attached process terminated
   231                              <1> runningdosemu	equ  100_0000h	; running in dosemu
   232                              <1> ; load_is_ldp	equ  200_0000h	; boot load: partition specified as "ldp"
   233                              <1> tt_while:	equ  400_0000h	; tt: while condition specified
   234                              <1> tt_p:		equ  800_0000h	; tt: proceed past repeated string instructions
   235                              <1> tt_silent_mode:	equ 1000_0000h	; tt: run should be silent (dump at end)
   236                              <1> tt_silence:	equ 2000_0000h	; tt: silent writing (write to auxbuff instead)
   237                              <1> tt_no_bb:	equ 4000_0000h	; tt: do not use bb breakpoints
   238                              <1> tt_no_bb_first:	equ 8000_0000h	; tt: do not use bb breakpoints at first
   239                              <1> 
   240                              <1> 
   241                              <1> dif2_gg_is_first:	equ   1
   242                              <1> dif2_gg_skip_non_cseip:	equ   2
   243                              <1> dif2_gg_skip_cseip:	equ   4
   244                              <1> dif2_gg_is_gg:		equ   8
   245                              <1> dif2_gg_first_detected:	equ  10h
   246                              <1> dif2_gg_again:		equ  20h
   247                              <1> dif2_tpg_proceed_bp_set:equ  40h
   248                              <1> dif2_tpg_keep_proceed_bp: equ 80h
   249                              <1> dif2_tpg_have_bp:	equ 100h
   250                              <1> dif2_tpg_adjusted_cseip:equ 200h
   251                              <1> dif2_tpg_do_not_adjust:	equ 400h
   252                              <1> dif2_bp_failure:	equ 800h
   253                              <1> dif2_is_pp:		equ 1000h
   254                              <1> %if _SYMBOLIC
   255                              <1> dif2_createdprocess:	equ 800_0000h	; created empty debuggee process
   256                              <1> dif2_sym_req_xms:	equ 2000h
   257                              <1> dif2_sym_req_86mm:	equ 4000h
   258                              <1> dif2_sym_req_mask equ dif2_sym_req_86mm | dif2_sym_req_xms
   259                              <1> dif2_no_pm_xms:		equ 1_0000h
   260                              <1> dif2_xms_detection_done:equ 2_0000h
   261                              <1> %endif
   262                              <1> %if _INPUT_FILE_HANDLES
   263                              <1> dif2_input_file:	equ 10_0000h
   264                              <1> dif2_closed_input_file:	equ 20_0000h
   265                              <1> %endif
   266                              <1> dif2_did_getline_file:	equ 40_0000h
   267                              <1> %if _SYMBOLIC
   268                              <1> dif2_poison:		equ 80_0000h
   269                              <1> %endif
   270                              <1> dif2_boot_loaded_kernel:equ 100_0000h
   271                              <1> %if _INPUT_FILE_BOOT
   272                              <1> dif2_input_file_boot:	equ 200_0000h
   273                              <1> dif2_closed_input_file_boot:	equ 400_0000h
   274                              <1> %endif
   275                              <1> dif2_in_silence_dump:	equ 1000_0000h
   276                              <1> dif2_int31_segment:	equ 2000_0000h
   277                              <1> dif2_nn_compat:		equ 4000_0000h
   278                              <1> dif2_nn_capitalise:	equ 8000_0000h
   279                              <1> 
   280                              <1> 
   281                              <1> dif3_load_is_ldp:	equ 1	; boot load: partition specified as "ldp"
   282                              <1> dif3_load_is_sdp:	equ 2	; boot load: partition specified as "sdp"
   283                              <1> dif3_load_is_ydp:	equ 4	; boot load: partition specified as "ydp"
   284                              <1> dif3_load_is_dp:	equ dif3_load_is_ldp 				| dif3_load_is_sdp 				| dif3_load_is_ydp
   287                              <1> dif3_load_dir_dir:	equ 8
   288                              <1> dif3_input_terminal_override:	equ 10h
   289                              <1> dif3_input_serial_override:	equ 20h
   290                              <1> dif3_if_not:		equ 40h
   291                              <1> dif3_partition_changed:	equ 80h
   292                              <1> ;
   293                              <1> dif3_input_cmdline:	equ 100h; input reading from cmdline_buffer
   294                              <1> dif3_input_cmdline_closed: equ 200h
   295                              <1> dif3_at_line_end:	equ 400h
   296                              <1> dif3_quiet_input_single:equ 800h
   297                              <1> dif3_quiet_output:	equ 1000h
   298                              <1> dif3_unquiet_error:	equ 2000h
   299                              <1> dif3_unquiet_prompt:	equ 4000h
   300                              <1> dif3_unquiet:		equ dif3_unquiet_error | dif3_unquiet_prompt
   301                              <1> dif3_return_eof:	equ 8000h
   302                              <1> dif3_highlighting:	equ 1_0000h
   303                              <1> dif3_do_not_highlight:	equ 2_0000h
   304                              <1> dif3_int10_highlight:	equ 2_0000h
   305                              <1> dif3_nosymbols_1:	equ 4_0000h
   306                              <1> dif3_nosymbols_2:	equ 8_0000h
   307                              <1> %if _PM
   308                              <1> dif3_ss_b_bit_set:	equ  10_0000h
   309                              <1> %endif
   310                              <1> dif3_gotint19:		equ  20_0000h
   311                              <1> dif3_prior_pm:		equ  40_0000h
   312                              <1> %if _DELAY_BEFORE_BP
   313                              <1> dif3_delayed		equ  80_0000h
   314                              <1> %endif
   315                              <1> dif3_input_re:		equ 100_0000h	; input reading from re_buffer
   316                              <1> dif3_input_re_closed:	equ 200_0000h
   317                              <1> dif3_accept_getrange_0:	equ 400_0000h
   318                              <1> %if _INPUT_FILE_HANDLES || _INPUT_FILE_BOOT
   319                              <1> dif3_in_if:		equ 800_0000h
   320                              <1> %endif
   321                              <1> dif3_auxbuff_guarded_1:	equ 1000_0000h
   322                              <1> dif3_auxbuff_guarded_2:	equ 2000_0000h
   323                              <1> dif3_auxbuff_guarded_3:	equ 4000_0000h
   324                              <1> dif3_sss_is_reverse:	equ 8000_0000h
   325                              <1> 
   326                              <1> 
   327                              <1> dif4_int_serial_hooked:	equ 1
   328                              <1> dif4_int_2F_hooked:	equ 2
   329                              <1> dif4_int_08_hooked:	equ 4
   330                              <1> dif4_int_2D_hooked:	equ 8
   331                              <1> %if _CATCHINTFAULTCOND && _CATCHINT0D
   332                              <1> dif4_int_0D_hooked:	equ 10h
   333                              <1> %endif
   334                              <1> %if _CATCHINTFAULTCOND && _CATCHINT0C
   335                              <1> dif4_int_0C_hooked:	equ 20h
   336                              <1> %endif
   337                              <1> %if _LOADER
   338                              <1> dif4_int_18_hooked:	equ 1000h
   339                              <1> dif4_int_19_hooked:	equ 2000h
   340                              <1> %endif
   341                              <1> 
   342                              <1> 
   343                              <1> %if _VXCHG
   344                              <1> dif6_vv_mode:		equ 1
   345                              <1> %endif
   346                              <1> dif6_in_hook2F:		equ 2
   347                              <1> dif6_in_amis_hook2F:	equ 4
   348                              <1> dif6_debug_mode:	equ 100h
   349                              <1> dif6_locked:		equ 200h
   350                              <1> dif6_mcp:		equ 400h
   351                              <1> %if _RH
   352                              <1> dif6_rh_mode_was:	equ  8_0000h
   353                              <1> dif6_rh_mode:		equ 10_0000h
   354                              <1> dif6_rh_mode_2:		equ 20_0000h
   355                              <1> %endif
   356                              <1> dif6_device_mode:	equ 40_0000h
   357                              <1> dif6_cpdepchars:	equ 80_0000h
   358                              <1> %if _IMMASM
   359                              <1> dif6_immasm_no_output:	equ 100_0000h
   360                              <1> dif6_immasm:		equ 200_0000h
   361                              <1> dif6_immasm_rel8:	equ 400_0000h
   362                              <1> %endif
   363                              <1> 
   364                              <1> 
   365                              <1> disasm_lowercase	equ 1
   366                              <1> disasm_commablank	equ 2
   367                              <1> disasm_nasm		equ 4
   368                              <1> disasm_lowercase_refmem:equ 8
   369                              <1> disasm_show_short:	equ 10h
   370                              <1> disasm_show_near:	equ 20h
   371                              <1> disasm_show_far:	equ 40h
   372                              <1> disasm_nec:		equ 80h
   373                              <1> disasm_40_columns:	equ 100h
   374                              <1> disasm_no_indent:	equ 200h
   375                              <1> disasm_msdebug_mnemonofs: equ 400h
   376                              <1> disasm_a16_memref:	equ 1000h
   377                              <1> disasm_a32_memref:	equ 2000h
   378                              <1> disasm_a16_string:	equ 4000h
   379                              <1> disasm_a32_string:	equ 8000h
   380                              <1> disasm_hide_modrm:	equ 10000h
   381                              <1> disasm_asize_loop_nasm:	equ 20000h
   382                              <1> disasm_modrm_always:	equ 40000h
   383                              <1> DEFAULTASMOPTIONS equ disasm_lowercase|disasm_commablank|disasm_nasm 	| disasm_a16_memref | disasm_a32_memref 	| disasm_a16_string | disasm_a32_string
   386                              <1> 
   387                              <1> 	; serial_flags values
   388                              <1> sf_init_done:	equ 1
   389                              <1> sf_ctrl_c:	equ 2
   390                              <1> sf_double_ctrl_c:	equ 4
   391                              <1> sf_built_in_fifo:	equ 8
   392                              <1> sf_use_serial:		equ 10h
    31                                  
    32                                  %include "iniload.mac"
     1                              <1> %if 0
     2                              <1> 
     3                              <1> lDebug iniload/boot interfacing structs and macros
     4                              <1> 
     5                              <1> Copyright (C) 2008-2025 E. C. Masloch
     6                              <1> 
     7                              <1> Usage of the works is permitted provided that this
     8                              <1> instrument is retained with the works, so that any entity
     9                              <1> that uses the works is notified of this instrument.
    10                              <1> 
    11                              <1> DISCLAIMER: THE WORKS ARE WITHOUT WARRANTY.
    12                              <1> 
    13                              <1> %endif
    14                              <1> 
    15                              <1> 
    16                              <1> 	struc BS
    17 00000000 ??????              <1> bsJump:	resb 3
    18 00000003 ????????????????    <1> bsOEM:	resb 8
    19                              <1> bsBPB:
    20                              <1> 	endstruc
    21                              <1> 
    22                              <1> 	struc EBPB		;        BPB sec
    23 00000000 ????                <1> bpbBytesPerSector:	resw 1	; offset 00h 0Bh
    24 00000002 ??                  <1> bpbSectorsPerCluster:	resb 1	; offset 02h 0Dh
    25 00000003 ????                <1> bpbReservedSectors:	resw 1	; offset 03h 0Eh
    26 00000005 ??                  <1> bpbNumFATs:		resb 1	; offset 05h 10h
    27 00000006 ????                <1> bpbNumRootDirEnts:	resw 1	; offset 06h 11h -- 0 for FAT32
    28 00000008 ????                <1> bpbTotalSectors:	resw 1	; offset 08h 13h
    29 0000000A ??                  <1> bpbMediaID:		resb 1	; offset 0Ah 15h
    30 0000000B ????                <1> bpbSectorsPerFAT:	resw 1	; offset 0Bh 16h -- 0 for FAT32
    31 0000000D ????                <1> bpbCHSSectors:		resw 1	; offset 0Dh 18h
    32 0000000F ????                <1> bpbCHSHeads:		resw 1	; offset 0Fh 1Ah
    33 00000011 ????????            <1> bpbHiddenSectors:	resd 1	; offset 11h 1Ch
    34 00000015 ????????            <1> bpbTotalSectorsLarge:	resd 1	; offset 15h 20h
    35                              <1> bpbNew:				; offset 19h 24h
    36                              <1> 
    37 00000019 ????????            <1> ebpbSectorsPerFATLarge:	resd 1	; offset 19h 24h
    38 0000001D ????                <1> ebpbFSFlags:		resw 1	; offset 1Dh 28h
    39 0000001F ????                <1> ebpbFSVersion:		resw 1	; offset 1Fh 2Ah
    40 00000021 ????????            <1> ebpbRootCluster:	resd 1	; offset 21h 2Ch
    41 00000025 ????                <1> ebpbFSINFOSector:	resw 1	; offset 25h 30h
    42 00000027 ????                <1> ebpbBackupSector:	resw 1	; offset 27h 32h
    43 00000029 <res Ch>            <1> ebpbReserved:		resb 12	; offset 29h 34h
    44                              <1> ebpbNew:			; offset 35h 40h
    45                              <1> 	endstruc
    46                              <1> 
    47                              <1> 	struc BPBN		; ofs B16 S16 B32 S32
    48 00000000 ??                  <1> bpbnBootUnit:		resb 1	; 00h 19h 24h 35h 40h
    49 00000001 ??                  <1> 			resb 1	; 01h 1Ah 25h 36h 41h
    50 00000002 ??                  <1> bpbnExtBPBSignature:	resb 1	; 02h 1Bh 26h 37h 42h -- 29h for valid BPBN
    51 00000003 ????????            <1> bpbnSerialNumber:	resd 1	; 03h 1Ch 27h 38h 43h
    52 00000007 <res Bh>            <1> bpbnVolumeLabel:	resb 11	; 07h 20h 2Bh 3Ch 47h
    53 00000012 ????????????????    <1> bpbnFilesystemID:	resb 8	; 12h 2Bh 36h 47h 52h
    54                              <1> 	endstruc		; 1Ah 33h 3Eh 4Fh 5Ah
    55                              <1> 
    56                              <1> 	struc DIRENTRY
    57 00000000 ????????????????    <1> deName:		resb 8
    58 00000008 ??????              <1> deExt:		resb 3
    59 0000000B ??                  <1> deAttrib:	resb 1
    60 0000000C ??                  <1> dePlusSize:	resb 1
    61 0000000D ??????????????      <1> 		resb 7
    62 00000014 ????                <1> deClusterHigh:	resw 1
    63 00000016 ????                <1> deTime:		resw 1
    64 00000018 ????                <1> deDate:		resw 1
    65 0000001A ????                <1> deClusterLow:	resw 1
    66 0000001C ????????            <1> deSize:		resd 1
    67                              <1> 	endstruc
    68                              <1> 
    69                              <1> ATTR_READONLY	equ 1
    70                              <1> ATTR_HIDDEN	equ 2
    71                              <1> ATTR_SYSTEM	equ 4
    72                              <1> ATTR_VOLLABEL	equ 8
    73                              <1> ATTR_DIRECTORY	equ 10h
    74                              <1> ATTR_ARCHIVE	equ 20h
    75                              <1> 
    76                              <1> lsvclSignature		equ "CL"
    77                              <1> lsvclBufferLength	equ 256
    78                              <1> 
    79                              <1> 	struc LOADSTACKVARS, -10h
    80 FFFFFFF0 ????????            <1> lsvFirstCluster:	resd 1
    81 FFFFFFF4 ????????            <1> lsvFATSector:		resd 1
    82 FFFFFFF8 ????                <1> lsvFATSeg:		resw 1
    83 FFFFFFFA ????                <1> lsvLoadSeg:		resw 1
    84 FFFFFFFC ????????            <1> lsvDataStart:		resd 1
    85                              <1> 	endstruc
    86                              <1> 
    87                              <1> 	struc LOADDATA, LOADSTACKVARS - 10h
    88 FFFFFFE0 ????                <1> ldMemoryTop:	resw 1
    89 FFFFFFE2 ????                <1> ldLoadTop:	resw 1
    90 FFFFFFE4 ????                <1> ldSectorSeg:	resw 1
    91 FFFFFFE6 ??                  <1> ldFATType:	resb 1
    92                              <1> ldFlags:
    93 FFFFFFE7 ??                  <1> ldHasLBA:	resb 1
    94 FFFFFFE8 ????                <1> ldClusterSize:	resw 1
    95 FFFFFFEA ????                <1> ldParaPerSector:resw 1
    96                              <1> ldDirCluster:			; dword
    97                              <1> ldLoadingSeg:		; word
    98                              <1> ldQueryPatchValue:	; word
    99                              <1> lsvCommandLine:		; word
   100                              <1> .start:		equ $ - lsvclBufferLength
   101 FFFFFFEC ????                <1> .signature:	resw 1
   102                              <1> ldLoadUntilSeg:		; word
   103                              <1> lsvExtra:		; word
   104 FFFFFFEE ??                  <1> .partition:	resb 1	; byte
   105 FFFFFFEF ??                  <1> .flags:		resb 1	; byte
   106                              <1> 	endstruc
   107                              <1> 
   108                              <1> ldhlfPreserveLoader	equ 4
   109                              <1> 
   110                              <1> lsvefNoDataStart	equ 1
   111                              <1> lsvefPartitionNumber	equ 2
   112                              <1> lsvefPreserveLoader	equ 4
   113                              <1> 
   114                              <1> %if lsvefPreserveLoader != ldhlfPreserveLoader
   115                              <1>  %error Unexpected flag values
   116                              <1> %endif
   117                              <1> 
   118                              <1> 	struc LOADCMDLINE, LOADDATA - lsvclBufferLength
   119                              <1> ldCommandLine:
   120 FFFFFEE0 <res 100h>          <1> .start:		resb lsvclBufferLength
   121                              <1> 	endstruc
   122                              <1> 
   123                              <1> ldfHasLBA:	equ 1
   124                              <1> ldfFATInvalid:	equ 2
   125                              <1> ldfFATBuffered:	equ 4
   126                              <1> ldfDataBuffered: equ 8
   127                              <1> 
   128                              <1> 	struc LOADDATA2, LOADDATA - 10h
   129 FFFFFFD0 ????????            <1> ldRootSector:		resd 1
   130 FFFFFFD4 ????                <1> ldEntriesPerSector:	resw 1
   131                              <1> ldDataSegment:		; word
   132 FFFFFFD6 ????                <1> ldLastAvailableSector:	resw 1
   133                              <1> ldDataSector:		; dword
   134 FFFFFFD8 ????                <1> ldParasLeft:		resw 1
   135 FFFFFFDA ????                <1> ldParasDone:		resw 1
   136                              <1> 	endstruc
   137                              <1> 
   138                              <1> 	struc LOADDATA3, LOADDATA2 - 10h
   139 FFFFFFC0 ????????            <1> ldMaxCluster:		resd 1
   140 FFFFFFC4 ????????            <1> ldFileSize:		resd 1
   141 FFFFFFC8 ????????            <1> ldCurrentCluster:	resd 1
   142 FFFFFFCC ????????            <1> ldCurrentSeek:		resd 1
   143                              <1> 	endstruc
   144                              <1> 
   145                              <1> 	struc LOADERIMAGEIDENT
   146 00000000 ????????            <1> liiSignature:		resb 4		; "NLDR"
   147 00000004 ????                <1> liiVersion:		resb 2		; "00"
   148 00000006 ????                <1> liiChecksum:		resw 1		; word sum of first 8 words = 0
   149 00000008 ????                <1> liiAmountParagraphs:	resw 1
   150 0000000A ????????????        <1> liiReserved:		resw 3
   151 00000010 ????                <1> liiEntryQuerySize:	resw 1		; 0 if not supported
   152                              <1> 		; INP:	cs => NLDR image ident
   153                              <1> 		;	ip = this word field content
   154                              <1> 		;	ax = 60h
   155                              <1> 		; OUT:	ax => behind memory requested (should be >= 60h)
   156                              <1> 		; CHG:	es, ds, di, si, bx, cx, dx
   157                              <1> 		; STT:	far called, UP, EI
   158 00000012 ????                <1> liiEntryRelocate:	resw 1		; 0 if not supported
   159                              <1> 		; INP:	cs => NLDR image ident
   160                              <1> 		;	ip = this word field content
   161                              <1> 		;	ax = 60h
   162                              <1> 		; OUT:	ax => relocated NLDR segment (usually 60h)
   163                              <1> 		; CHG:	es, ds, di, si, bx, cx, dx
   164                              <1> 		; STT:	far called, UP, EI
   165 00000014 ????                <1> liiEntryDebug:		resw 1		; 0 if not supported
   166                              <1> 		; INP:	es = ds = cs = ss => relocated NLDR
   167                              <1> 		;	ip = this word field content
   168                              <1> 		;	sp = next word field content
   169                              <1> 		; STT:	running as debuggee, UP, EI
   170 00000016 ????                <1> liiStackPointer:	resw 1
   171                              <1> 	endstruc
   172                              <1> 
   173                              <1> 	struc LBAPACKET
   174 00000000 ????                <1> lpSize:		resw 1
   175 00000002 ????                <1> lpCount:	resw 1
   176 00000004 ????????            <1> lpBuffer:	resd 1
   177 00000008 ????????????????    <1> lpSector:	resq 1
   178                              <1> 	endstruc
   179                              <1> 
   180                              <1> 	struc PARTINFO
   181 00000000 ??                  <1> piBoot:		resb 1
   182 00000001 ??????              <1> piStartCHS:	resb 3
   183 00000004 ??                  <1> piType:		resb 1
   184 00000005 ??????              <1> piEndCHS:	resb 3
   185 00000008 ????????            <1> piStart:	resd 1
   186 0000000C ????????            <1> piLength:	resd 1
   187                              <1> 	endstruc
   188                              <1> 
   189                              <1> ptEmpty:		equ 0
   190                              <1> ptFAT12:		equ 1
   191                              <1> ptFAT16_16BIT_CHS:	equ 4
   192                              <1> ptExtendedCHS:		equ 5
   193                              <1> ptFAT16_CHS:		equ 6
   194                              <1> ptFAT32_CHS:		equ 0Bh
   195                              <1> ptFAT32:		equ 0Ch
   196                              <1> ptFAT16:		equ 0Eh
   197                              <1> ptExtended:		equ 0Fh
   198                              <1> ptLinux:		equ 83h
   199                              <1> ptExtendedLinux:	equ 85h
   200                              <1> 
   201                              <1> 
   202                              <1> 		; Flags of load_unit_flags
   203                              <1> lufForceCHS:		equ 1
   204                              <1> lufForceLBA:		equ 2
   205                              <1> lufForceGeometry:	equ 4
   206                              <1> luf_mask_writable equ lufForceCHS | lufForceLBA | lufForceGeometry
    33                                  
    34                                  	cpu 8086
    35                                  
    36                                  	addsection RELOCATEDDATA, nobits vstart=_ELD_RELOC_VSTART
    37                                  relocateddata:
    38                                  
    39                                  	addsection HEADER, start=0
    40                                  
    41                                  	istruc ELD_HEADERX
    42                                  at eldhxHeader
    43                                  		; ELD executable header
    44                                  	istruc ELD_HEADER
    45 00000000 454C4431                at eldhSignature,	db "ELD1"
    46 00000004 000000                  			db 0,0,0
    47 00000007 1A                      			db 26
    48 00000008 60000000                at eldhCodeOffset,	dd CODEOFFSET
    49 0000000C 1012                    at eldhCodeImageLength,	dw code_size
    50 0000000E 0000                    at eldhCodeAllocLength,	dw 0
    51 00000010 70120000                at eldhDataOffset,	dd DATAOFFSET
    52 00000014 6004                    at eldhDataImageLength,	dw data_size
    53 00000016 2002                    at eldhDataAllocLength,	dw total_data_size - data_size
    54 00000018 2008                    at eldhCodeEntrypoint,	dw linker - code
    55                                  at eldhReserved
    56 0000001A 00<rep 4h>2800          at eldhExtensionSize,	dw header_extension_end - $$
    57                                  	iend
    58 00000020 [30000000]              at eldhxDescriptionOffset,	dd description
    59 00000024 A5140000                at eldhxHelpOffset,		dd DATAOFFSET + msg.help - datastart
    60                                  PUT_ELDHX_DATETIME_OFFSET
    61                                  header_extension_end:
    62 00000028 00<rep 8h>              	iend
    63                                  
    64                                  %if _BOOT
    65                                  description:		asciz "List files from directories, boot loaded."
    66                                  %else
    67 00000030 4C69737420444F5320-     description:		asciz "List DOS files from directories."
    67 00000039 66696C65732066726F-
    67 00000042 6D206469726563746F-
    67 0000004B 726965732E00       
    68                                  %endif
    69                                  
    70 00000051 00<rep Fh>              	align 16, db 0
    71                                  
    72                                  	eldstrict on
    73                                  
    74                                  CODEOFFSET equ $ - $$
    75                                  	addsection CODE, follows=HEADER vstart=_ELD_CODE_VSTART
    76                                  %define CODEFIXUP - code + 0
    77                                  code:
    78                                  		; ELD instance header
    79                                  	istruc ELD_INSTANCE
    80                                  at eldiStartCode
    81 00000000 00<rep 2h>              at eldiEndCode
    82 00000002 00<rep 2h>              at eldiStartData
    83 00000004 00<rep 2h>              at eldiEndData
    84                                  %if _BOOT
    85                                  at eldiIdentifier,	fill 8, 32, db "BOOT DIR"
    86                                  at eldiListing,		asciz _ELD_LISTING
    87                                  %else
    88 00000006 00<rep 2h>444F5320-     at eldiIdentifier,	fill 8, 32, db "DOS DIR"
    88 0000000C 44495220           
    89 00000010 00<rep 2h>646F7364-     at eldiListing,		asciz _ELD_LISTING
    89 00000016 69722E6C737400     
    90                                  %endif
    91 0000001D 00<rep 3h>              	iend
    92                                  
    93                                  
    94                                  run:
    95 00000020 16                      	push ss
    96 00000021 07                      	pop es
    97                                  
    98                                  %if _BOOT
    99                                  run_boot:
   100                                  reloc	testopt [relocateddata], nodosloaded
   101                                  linkdatarelocation internalflags, -3
   102                                  	jz error
   103                                  	extcallcall yy_boot_parse_name2
   104                                  	call parse_verbose
   105                                  reloc	mov word [pathname_start], bx
   106                                  internaldatarelocation
   107                                  
   108                                  	push bx
   109                                  	mov di, bx
   110                                  	call find_dir
   111                                  	pop bx
   112                                  	mov dx, di
   113                                   %if 0
   114                                  	db __TEST_IMM8			; (skip inc)
   115                                  @@:
   116                                  	inc di
   117                                  	cmp byte [di], 0
   118                                  	je boot_no_wild
   119                                  	cmp byte [di], '?'
   120                                  	je boot_wild
   121                                  	cmp byte [di], '*'
   122                                  	jne @B
   123                                  
   124                                  boot_no_wild:
   125                                  boot_wild:
   126                                   %endif
   127                                  reloc	mov word [wild_pattern], dx
   128                                  internaldatarelocation
   129                                  
   130                                  	extcallcall yy_boot_init_dir2
   131                                  
   132                                  	mov di, word [bp + bsBPB + bpbBytesPerSector]
   133                                  					; di = sector size
   134                                  					; = start of available auxbuff
   135                                  	cmp byte [bp + ldFATType], 12	; FAT12 ?
   136                                  	jne @F				; no -->
   137                                  	cmp di, 8192			; already enough for a full FAT ?
   138                                  	jae @F				; yes -->
   139                                  	add di, di			; reserve straddling sector
   140                                  @@:
   141                                  %else
   142                                  run_dos:
   143 00000022 E84307                  	extcallcall InDOS
   144 00000025 E84807                  	extcallcall yy_dos_parse_name
   145 00000028 E83905                  	call parse_verbose
   146                                  
   147                                  	houdini
   148 0000002B 891E[7004]              reloc	mov word [pathname_start], bx
   149                                  internaldatarelocation
   150 0000002F 53                      	push bx
   151                                  
   152 00000030 B42F                    	mov ah, 2Fh			; get DTA
   153 00000032 E84307                  	extcallcall ispm
   154 00000035 750F                    	jnz .rm
   155                                  
   156                                  subcpu 286
   157 00000037 6A00                    	push word 0
   158 00000039 6A21                    	push word 21h
   159 0000003B E8[0000]EB020000        	extcall intcall_ext_return_es, PM required	; must NOT be extcallcall
   160 00000042 5A                      	pop dx				; discard interrupt number
   161 00000043 5A                      	pop dx				; get es
   162                                  subcpureset
   163 00000044 EB04                    	jmp @F
   164                                  .rm:
   165 00000046 CD21                    	int 21h
   166 00000048 8CC2                    	mov dx, es
   167                                  @@:
   168                                  
   169 0000004A 891E[6004]              reloc	mov word [originaldta], bx
   170                                  internaldatarelocation
   171 0000004E 8916[6204]              reloc	mov word [originaldta + 2], dx
   172                                  internaldatarelocation
   173                                  
   174 00000052 A1[0000]                reloc	mov ax, word [relocateddata]
   175                                  linkdatarelocation ext_inject_handler
   176 00000055 A3[6404]                reloc	mov word [originalinject], ax
   177                                  internaldatarelocation
   178 00000058 C706[0000][BE06]        reloc2	mov word [relocateddata], inject
   179                                  linkdatarelocation ext_inject_handler, -4
   180                                  internalcoderelocation
   181 0000005E E8B306                  	call get_es_ext
   182 00000061 26800E[1000]01          reloc	setopt [es:code + eldiFlags], eldifResident
   183                                  internalcoderelocation -3	; mark block as resident
   184 00000067 16                      	 push ss
   185 00000068 07                      	 pop es
   186                                  
   187                                  	houdini
   188 00000069 BA[7804]                reloc	mov dx, dta
   189                                  internaldatarelocation
   190 0000006C B41A                    	mov ah, 1Ah		; set DTA
   191 0000006E E80F07                  	extcallcall _doscall
   192                                  
   193 00000071 5A                      	pop dx
   194                                  %endif
   195                                  
   196 00000072 D006[0900]              reloc	rol byte [sort], 1
   197                                  internaldatarelocation
   198 00000076 7352                    	jnc .no_sort_buffer
   199                                  
   200 00000078 A1[0000]                reloc	mov ax, word [relocateddata]
   201                                  linkdatarelocation extdata_size
   202 0000007B 2B06[0000]              reloc	sub ax, word [relocateddata]
   203                                  linkdatarelocation extdata_used
   204 0000007F 8B1E[0000]              reloc	mov bx, word [relocateddata]
   205                                  linkdatarelocation auxbuff_current_size
   206 00000083 83C008                  	add ax, (uinit_data_end_2 - buffer_end)
   207                                  %if _BOOT
   208                                  	sub bx, di
   209                                  	jbe .use_sort_buffer_eld_data_block
   210                                  %endif
   211 00000086 39D8                    	cmp ax, bx
   212 00000088 7307                    	jae .use_sort_buffer_eld_data_block
   213                                  
   214                                  %ifn _BOOT
   215 0000008A F606[0300]70            reloc	testopt [relocateddata], dif3_auxbuff_guarded_1 		| dif3_auxbuff_guarded_2 		| dif3_auxbuff_guarded_3
   218                                  linkdatarelocation internalflags3, -3
   219 0000008F 741C                    	jz .use_sort_buffer_auxbuff
   220                                  %else
   221                                  	jmp .use_sort_buffer_auxbuff
   222                                  %endif
   223                                  
   224                                  .use_sort_buffer_eld_data_block:
   225 00000091 83E808                  	sub ax, (uinit_data_end_2 - buffer_end)
   226 00000094 E87D06                  	call get_es_ext
   227 00000097 260106[0600]            reloc	add word [es:code + eldiEndData], ax
   228                                  internalcoderelocation		; adjust size
   229 0000009C 0106[0000]              reloc	add word [relocateddata], ax
   230                                  linkdatarelocation extdata_used	; adjust size
   231 000000A0 26A1[0600]              reloc	mov ax, word [es:code + eldiEndData]
   232                                  internalcoderelocation		; -> end of sort buffer
   233 000000A4 16                      	push ss
   234 000000A5 07                      	pop es
   235                                  
   236 000000A6 BF[7806]                reloc	mov di, buffer_end	; -> start of sort buffer
   237                                  internaldatarelocation
   238 000000A9 8CD6                    	mov si, ss		; => sort buffer
   239 000000AB EB0A                    	jmp .sort_buffer_common
   240                                  
   241                                  .use_sort_buffer_auxbuff:
   242 000000AD 93                      	xchg ax, bx		; ax -> end of sort buffer
   243                                  %ifn _BOOT
   244 000000AE 31FF                    	xor di, di		; di -> start of sort buffer
   245                                  %endif
   246 000000B0 8B36[0000]              reloc	mov si, word [relocateddata]
   247                                  linkdatarelocation auxbuff_segorsel	; => sort buffer
   248                                  %ifn _BOOT
   249 000000B4 E8D106                  	extcallcall guard_auxbuff
   250                                  %endif
   251                                  
   252                                  		; INP:	si:di -> buffer
   253                                  		;	si:ax -> behind buffer
   254                                  .sort_buffer_common:
   255 000000B7 8936[6604]              reloc	mov word [sortsegsel], si
   256                                  internaldatarelocation
   257 000000BB 893E[6804]              reloc	mov word [sortstartoffset], di
   258                                  internaldatarelocation
   259 000000BF 893E[6C04]              reloc	mov word [sort_last], di
   260                                  internaldatarelocation
   261 000000C3 893E[6E04]              reloc	mov word [sort_next], di
   262                                  internaldatarelocation
   263 000000C7 A3[6A04]                reloc	mov word [sortendoffset], ax
   264                                  internaldatarelocation
   265                                  
   266                                  .no_sort_buffer:
   267                                  
   268                                  %ifn _BOOT
   269 000000CA E85304                  	call findfirst
   270 000000CD 7303E98001              	jc .notfound
   271 000000D2 BF[0000]                reloc	mov di, relocateddata
   272                                  linkdatarelocation line_out
   273                                  
   274                                  .loop:
   275                                  %else
   276                                  boot_scan:
   277                                  reloc	mov byte [relocateddata], 0
   278                                  linkdatarelocation load_check_dir_attr, -3
   279                                  reloc	mov si, word [relocateddata]
   280                                  linkdatarelocation load_yyname_input
   281                                  	cmp byte [si], '/'
   282                                  	jne @F
   283                                  	inc si
   284                                  @@:
   285                                  	cmp byte [si], 0
   286                                  	jne @F
   287                                  	extcall ..@yy_filename_empty
   288                                  @@:
   289                                  	 push ss
   290                                  	 pop es
   291                                  	call boot_parse_name
   292                                  	cmp al, '/'
   293                                  	jne @F
   294                                  reloc	mov byte [relocateddata], ATTR_DIRECTORY
   295                                  linkdatarelocation load_check_dir_attr, -3
   296                                  reloc	mov word [relocateddata], si
   297                                  linkdatarelocation load_yyname_next
   298                                  @@:
   299                                  
   300                                  	mov di, -1
   301                                  	mov si, di
   302                                  	mov [bp + lsvFATSector], di
   303                                  	mov [bp + lsvFATSector + 2], si
   304                                  
   305                                  	xor ax, ax
   306                                  	xor dx, dx
   307                                  
   308                                  scan_dir_yyname_loop:
   309                                  	mov word [bp + ldDirCluster], ax
   310                                  	mov word [bp + ldDirCluster + 2], dx
   311                                  
   312                                  	push ss
   313                                  	pop es
   314                                  reloc	mov bx, relocateddata
   315                                  linkdatarelocation load_yy_direntry
   316                                  
   317                                  reloc2	mov word [relocateddata], relocateddata
   318                                  linkdatarelocation handle_scan_dir_not_found, -4
   319                                  ;linkdatarelocation near_transfer_ext_entry
   320                                  linkdatarelocation dmycmd
   321                                  	extcall scan_dir_aux
   322                                  	jc end_of_directory
   323                                  
   324                                  reloc	cmp byte [relocateddata], ATTR_DIRECTORY
   325                                  linkdatarelocation load_check_dir_attr, -3
   326                                  	jne got_single_yyentry
   327                                  
   328                                  	push si
   329                                  	push di
   330                                  reloc	mov byte [relocateddata], 0
   331                                  linkdatarelocation load_check_dir_attr, -3
   332                                  reloc	mov si, word [relocateddata]
   333                                  linkdatarelocation load_yyname_next
   334                                  	cmp byte [si], 0
   335                                  	jne @F
   336                                  	extcall ..@yy_filename_empty
   337                                  @@:
   338                                  	push es
   339                                  	 push ss
   340                                  	 pop es
   341                                  	call boot_parse_name
   342                                  	pop es
   343                                  	cmp al, '/'
   344                                  	jne @F
   345                                  reloc	mov byte [relocateddata], ATTR_DIRECTORY
   346                                  linkdatarelocation load_check_dir_attr, -3
   347                                  reloc	mov word [relocateddata], si
   348                                  linkdatarelocation load_yyname_next
   349                                  @@:
   350                                  	pop di
   351                                  	pop si
   352                                  
   353                                  	xor dx, dx
   354                                  	mov ax, [es:bx + deClusterLow]
   355                                  				; = first cluster (not FAT32)
   356                                  	cmp byte [bp + ldFATType], 32
   357                                  	jne @F
   358                                  	mov dx, [es:bx + deClusterHigh]
   359                                  				; dx:ax = first cluster (FAT32)
   360                                  @@:
   361                                  
   362                                  	jmp scan_dir_yyname_loop
   363                                  
   364                                  boot_parse_name:
   365                                  reloc	cmp word [wild_pattern], si
   366                                  internaldatarelocation
   367                                  	je @F
   368                                  	extcallcall boot_parse_fn	; get next pathname
   369                                  
   370                                  reloc2	mov word [relocateddata], relocateddata
   371                                  linkdatarelocation handle_scan_dir_entry, -4
   372                                  linkdatarelocation scan_dir_entry
   373                                  
   374                                  	retn
   375                                  
   376                                  @@:
   377                                  	extcallcall boot_parse_fn	; get next pathname
   378                                  
   379                                  reloc2	mov word [relocateddata], match_wildcard
   380                                  linkdatarelocation near_transfer_ext_address, -4
   381                                  internalcoderelocation
   382                                  reloc2	mov word [relocateddata], relocateddata
   383                                  linkdatarelocation handle_scan_dir_entry, -4
   384                                  linkdatarelocation near_transfer_ext_entry
   385                                  
   386                                  	push ax
   387                                  reloc	mov di, relocateddata
   388                                  linkdatarelocation load_kernel_name
   389                                  	mov cx, 8
   390                                  	call .handle_asterisk		; handle in basename
   391                                  	mov cl, 3
   392                                  	call .handle_asterisk		; handle in extension
   393                                  	pop ax
   394                                  	retn
   395                                  
   396                                  .handle_asterisk:
   397                                  	mov al, '*'
   398                                  	repne scasb			; scan for asterisk
   399                                  	jne @F				; not found -->
   400                                  	mov al, '?'			; fill with question marks
   401                                  	dec di				; -> at the asterisk
   402                                  	inc cx				; = how many bytes remain
   403                                  	rep stosb			; fill this field
   404                                  @@:
   405                                  	retn
   406                                  
   407                                  
   408                                  		; INP:	es:di -> DIRENTRY
   409                                  		;	dx:ax - 1 = sector
   410                                  		;	cx, si in use
   411                                  		; OUT:	CY if end of directory
   412                                  		;	NC if to continue,
   413                                  		;	 ZR if match
   414                                  		;	 NZ if mismatch
   415                                  		; CHG:	bx
   416                                  match_wildcard:
   417                                  	cmp byte [es:di], 0
   418                                  	stc
   419                                  	je .ret
   420                                  	mov bl, byte [es:di + deAttrib]
   421                                  	test bl, ATTR_VOLLABEL
   422                                  	jnz .ret_NC		; skip volume labels (and LFNs) --> (NZ)
   423                                  	push si
   424                                  	push di
   425                                  	push cx
   426                                  reloc	mov si, relocateddata	; ds:si-> name to match
   427                                  linkdatarelocation load_kernel_name
   428                                  	mov cx, 11		; length of padded 8.3 FAT filename
   429                                  @@:
   430                                  	repe cmpsb		; check entry
   431                                  	je @F			; match -->
   432                                  	cmp byte [si - 1], '?'	; wildcard ?
   433                                  	je @B			; yes --> (ZR)
   434                                  				; no (NZ)
   435                                  @@:
   436                                  	pop cx
   437                                  	pop di
   438                                  	pop si
   439                                  	jne .ret_NC
   440                                  
   441                                  	push si
   442                                  	push es
   443                                  	push di
   444                                  	push dx
   445                                  	push ax
   446                                  	push cx
   447                                  
   448                                  	mov cx, DIRENTRY_size
   449                                  	push ds
   450                                  	 push es
   451                                  	 pop ds
   452                                  	mov si, di		; ds:si -> entry in directory buffer
   453                                  	push ss
   454                                  	pop es
   455                                  reloc	mov di, relocateddata	; es:di -> destination for entry
   456                                  linkdatarelocation load_yy_direntry
   457                                  	push di
   458                                  	rep movsb
   459                                  	pop si
   460                                  	pop ds
   461                                  
   462                                  reloc	mov di, pathnamebuffer - 1
   463                                  internaldatarelocation		; di -> buffer
   464                                  	mov al, 0
   465                                  	stosb
   466                                  	push di
   467                                  	mov cl, 8
   468                                  	cmp byte [si], 05h
   469                                  	jne @F
   470                                  	mov al, 0E5h
   471                                  	stosb
   472                                  	dec cx
   473                                  	inc si
   474                                  @@:
   475                                  	rep movsb
   476                                  	mov cl, 9
   477                                  	db __TEST_IMM8
   478                                  @@:
   479                                  	dec di
   480                                  	cmp byte [di - 1], 32
   481                                  	loope @B
   482                                  
   483                                  	cmp byte [di - 1], '.'
   484                                  	jne @F
   485                                  	cmp word [si], 2020h
   486                                  	jne @F
   487                                  	cmp byte [si + 2], 32
   488                                  	je .dotname
   489                                  @@:
   490                                  
   491                                  	mov al, '.'
   492                                  	stosb
   493                                  	mov cl, 3
   494                                  	rep movsb
   495                                  	mov cl, 4
   496                                  	db __TEST_IMM8
   497                                  @@:
   498                                  	dec di
   499                                  	cmp byte [di - 1], 32
   500                                  	loope @B
   501                                  	cmp byte [di - 1], '.'
   502                                  	jne @F
   503                                  	dec di
   504                                  @@:
   505                                  .dotname:
   506                                  	mov al, 0
   507                                  	stosb
   508                                  
   509                                  	 push ss
   510                                  	 pop es
   511                                  	pop dx
   512                                  
   513                                  		; get attrib byte
   514                                  reloc	mov al, byte [relocateddata + deAttrib]
   515                                  linkdatarelocation load_yy_direntry
   516                                  reloc	mov byte [finddata.attrib], al
   517                                  internaldatarelocation
   518                                  
   519                                  		; get time and date
   520                                  reloc	mov ax, word [relocateddata + deTime]
   521                                  linkdatarelocation load_yy_direntry
   522                                  reloc	mov word [finddata.time], ax
   523                                  internaldatarelocation
   524                                  reloc	mov ax, word [relocateddata + deDate]
   525                                  linkdatarelocation load_yy_direntry
   526                                  reloc	mov word [finddata.date], ax
   527                                  internaldatarelocation
   528                                  
   529                                  		; get size low
   530                                  reloc	mov ax, word [relocateddata + deSize]
   531                                  linkdatarelocation load_yy_direntry
   532                                  reloc	mov word [finddata.sizelow], ax
   533                                  internaldatarelocation
   534                                  reloc	mov ax, word [relocateddata + deSize + 2]
   535                                  linkdatarelocation load_yy_direntry
   536                                  reloc	mov word [finddata.sizelow + 2], ax
   537                                  internaldatarelocation
   538                                  
   539                                  		; zero unused fields
   540                                  	xor ax, ax
   541                                  reloc	mov word [finddata.sizehigh + 2], ax
   542                                  internaldatarelocation
   543                                  reloc	mov byte [finddata.shortname], al
   544                                  internaldatarelocation
   545                                  
   546                                  		; get FAT+ high 6 size bits
   547                                  reloc	mov al, byte [relocateddata + dePlusSize]
   548                                  linkdatarelocation load_yy_direntry
   549                                  	mov ah, al
   550                                  	and ax, 0E007h
   551                                  	shr ah, 1
   552                                  	shr ah, 1
   553                                  	or al, ah
   554                                  	mov ah, 0
   555                                  reloc	mov word [finddata.sizehigh], ax
   556                                  internaldatarelocation
   557                                  
   558                                  reloc	call near [matchfunction]
   559                                  internaldatarelocation		; NZ to continue search, ZR to end
   560                                  
   561                                  	pop cx
   562                                  	pop ax
   563                                  	pop dx
   564                                  	pop di
   565                                  	pop es
   566                                  	pop si			; restore registers
   567                                  
   568                                  %if 0
   569                                  	pushf
   570                                  	sub ax, 1
   571                                  	sbb dx, 0
   572                                  reloc	mov bx, [relocateddata]
   573                                  linkdatarelocation load_adr_dirbuf_segment
   574                                  	extcall read_sector	; restore sector
   575                                  	popf
   576                                  %endif
   577                                  
   578                                  .ret_NC:
   579                                  	clc
   580                                  .ret:
   581                                  	extcall near_transfer_ext_return, required ; must NOT be extcallcall
   582                                  
   583                                  
   584                                  got_single_yyentry:
   585                                  end_of_directory:
   586                                  reloc2	cmp word [matchfunction], display_ZR
   587                                  internaldatarelocation -4
   588                                  internalcoderelocation
   589                                  	jne ..@boot_scan_end
   590                                  	retn
   591                                  
   592                                  sort_or_display:
   593                                  %endif
   594 000000D5 D006[0900]              reloc	rol byte [sort], 1
   595                                  internaldatarelocation
   596 000000D9 7203E94101              	jnc .display
   597                                  
   598 000000DE E83C02                  	call populate_finddata
   599 000000E1 7503E93C01              	je .next
   600                                  
   601                                  %ifn _BOOT
   602 000000E6 D006[0A00]              reloc	rol byte [sortlfn], 1
   603                                  internaldatarelocation
   604 000000EA 7303                    	jnc @F
   605                                  
   606 000000EC BE[D004]                reloc	mov si, finddata.fullname
   607                                  internaldatarelocation
   608                                  @@:
   609                                  %endif
   610                                  
   611 000000EF 89F7                    	mov di, si
   612 000000F1 B000                    	mov al, 0
   613 000000F3 B90002                  	mov cx, 512
   614 000000F6 F2AE                    	repne scasb
   615 000000F8 7403E96401              	jne .error
   616                                  
   617 000000FD 89F9                    	mov cx, di
   618 000000FF 29F1                    	sub cx, si		; = length including NUL
   619                                  
   620 00000101 8B3E[6C04]              reloc	mov di, word [sort_last]
   621                                  internaldatarelocation
   622 00000105 89F8                    	mov ax, di
   623 00000107 01C8                    	add ax, cx
   624 00000109 7303E96301              	jc .toofull
   625 0000010E 0306[0000]              reloc	add ax, word [meta]
   626                                  internaldatarelocation
   627 00000112 7303E95A01              	jc .toofull
   628 00000117 3B06[6A04]              reloc	cmp ax, word [sortendoffset]
   629                                  internaldatarelocation
   630 0000011B 7603E95101              	ja .toofull
   631                                  
   632 00000120 8E06[6604]              reloc	mov es, word [sortsegsel]
   633                                  internaldatarelocation
   634 00000124 8B3E[6804]              reloc	mov di, word [sortstartoffset]
   635                                  internaldatarelocation
   636 00000128 89F2                    	mov dx, si
   637                                  
   638                                  .sort:
   639 0000012A 3B3E[6C04]              reloc	cmp di, word [sort_last]
   640                                  internaldatarelocation
   641 0000012E 7203E9DD00              	jae .sort_insert_last
   642                                  
   643 00000133 89FB                    	mov bx, di
   644                                  
   645 00000135 D006[0B00]              reloc	rol byte [dirfirst], 1
   646                                  internaldatarelocation
   647 00000139 730E                    	jnc .notdirfirst
   648 0000013B A0[A404]                reloc	mov al, byte [finddata.attrib]
   649                                  internaldatarelocation
   650 0000013E 268A25                  	mov ah, byte [es:di]
   651 00000141 251010                  	and ax, (ATTR_DIRECTORY << 8) | ATTR_DIRECTORY
   652 00000144 38E0                    	cmp al, ah
   653 00000146 755F                    	jne ..@compare_normal
   654 00000148 47                      	inc di
   655                                  .notdirfirst:
   656                                  
   657 00000149 D006[0C00]              reloc	rol byte [date], 1
   658                                  internaldatarelocation
   659 0000014D 7311                    	jnc .notdate
   660 0000014F A1[BA04]                reloc	mov ax, word [finddata.date]
   661                                  internaldatarelocation
   662 00000152 263B4502                	cmp ax, word [es:di + 2]
   663 00000156 7547                    	jne .sort_compare
   664 00000158 A1[B804]                reloc	mov ax, word [finddata.time]
   665                                  internaldatarelocation
   666 0000015B 263B05                  	cmp ax, word [es:di]
   667 0000015E 753F                    	jne .sort_compare
   668                                  	; scasw
   669                                  	; scasw
   670                                  .notdate:
   671                                  
   672 00000160 D006[0D00]              reloc	rol byte [size], 1
   673                                  internaldatarelocation
   674 00000164 731A                    	jnc .notsize
   675 00000166 A0[E605]                reloc	mov al, byte [size40bit + 4]
   676                                  internaldatarelocation
   677 00000169 263A4504                	cmp al, byte [es:di + 4]
   678 0000016D 7530                    	jne .sort_compare
   679 0000016F A1[E405]                reloc	mov ax, word [size40bit + 2]
   680                                  internaldatarelocation
   681 00000172 263B4502                	cmp ax, word [es:di + 2]
   682 00000176 7527                    	jne .sort_compare
   683 00000178 A1[E205]                reloc	mov ax, word [size40bit]
   684                                  internaldatarelocation
   685 0000017B 263B05                  	cmp ax, word [es:di]
   686 0000017E 751F                    	jne .sort_compare
   687                                  	; add di, 5
   688                                  .notsize:
   689                                  
   690 00000180 89DF                    	mov di, bx
   691 00000182 033E[0000]              reloc	add di, word [meta]
   692                                  internaldatarelocation
   693 00000186 89D6                    	mov si, dx
   694 00000188 B001                    	mov al, 1
   695                                  @@:
   696 0000018A 3C00                    	cmp al, 0
   697 0000018C 741B                    	je .sort_insert_skip_bx
   698 0000018E AC                      	lodsb
   699 0000018F 268A25                  	mov ah, byte [es:di]
   700 00000192 47                      	inc di
   701 00000193 E8FA05                  	extcallcall uppercase
   702 00000196 86C4                    	xchg al, ah
   703 00000198 E8F505                  	extcallcall uppercase
   704 0000019B 38E0                    	cmp al, ah
   705 0000019D 74EB                    	je @B
   706                                  .sort_compare:
   707 0000019F FF26[0200]              reloc	jmp near [compare]
   708                                  internaldatarelocation
   709                                  
   710                                  ..@compare_reverse:
   711 000001A3 7216                    	jb .sort_insert_before_bx
   712 000001A5 EB02                    	jmp .sort_insert_skip_bx
   713                                  
   714                                  ..@compare_normal:
   715 000001A7 7712                    	ja .sort_insert_before_bx
   716                                  .sort_insert_skip_bx:
   717 000001A9 51                      	push cx
   718 000001AA 89DF                    	mov di, bx
   719 000001AC 033E[0000]              reloc	add di, word [meta]
   720                                  internaldatarelocation
   721 000001B0 B000                    	mov al, 0
   722 000001B2 B90002                  	mov cx, 512
   723 000001B5 F2AE                    	repne scasb
   724 000001B7 59                      	pop cx
   725 000001B8 E96FFF                  	jmp .sort
   726                                  
   727                                  .sort_insert_before_bx:
   728                                  	houdini
   729 000001BB 8B3E[6C04]              reloc	mov di, word [sort_last]	; -> after last
   730                                  internaldatarelocation
   731 000001BF 89FE                    	mov si, di			; -> behind source
   732 000001C1 01CF                    	add di, cx			; -> behind target
   733 000001C3 033E[0000]              reloc	add di, word [meta]
   734                                  internaldatarelocation
   735 000001C7 51                      	push cx
   736 000001C8 89F1                    	mov cx, si			; -> behind source
   737 000001CA 29D9                    	sub cx, bx			; behind source minus start source
   738                                  					;  = length of source
   739 000001CC FD                      	std
   740 000001CD A6                      	cmpsb				; -> last bytes
   741                                  @@:
   742 000001CE 26A4                    	es movsb
   743 000001D0 E2FC                    	loop @B				; move up trailer
   744 000001D2 FC                      	cld
   745 000001D3 59                      	pop cx
   746 000001D4 010E[6C04]              reloc	add word [sort_last], cx
   747                                  internaldatarelocation
   748 000001D8 8B3E[0000]              reloc	mov di, word [meta]
   749                                  internaldatarelocation
   750 000001DC 013E[6C04]              reloc	add word [sort_last], di
   751                                  internaldatarelocation
   752 000001E0 89DF                    	mov di, bx
   753 000001E2 E80200                  	call .store_with_meta
   754 000001E5 EB34                    	jmp .sort_inserted
   755                                  
   756                                  .store_with_meta:
   757 000001E7 D006[0B00]              reloc	rol byte [dirfirst], 1
   758                                  internaldatarelocation
   759 000001EB 7304                    	jnc @F
   760 000001ED A0[A404]                reloc	mov al, byte [finddata.attrib]
   761                                  internaldatarelocation
   762 000001F0 AA                      	stosb
   763                                  @@:
   764                                  
   765 000001F1 D006[0D00]              reloc	rol byte [size], 1
   766                                  internaldatarelocation
   767 000001F5 7306                    	jnc @F
   768 000001F7 BE[E205]                reloc	mov si, size40bit
   769                                  internaldatarelocation
   770 000001FA A5                      	movsw
   771 000001FB A5                      	movsw
   772 000001FC A4                      	movsb
   773                                  @@:
   774                                  
   775 000001FD D006[0C00]              reloc	rol byte [date], 1
   776                                  internaldatarelocation
   777 00000201 7308                    	jnc @F
   778 00000203 A1[B804]                reloc	mov ax, word [finddata.time]
   779                                  internaldatarelocation
   780 00000206 AB                      	stosw
   781 00000207 A1[BA04]                reloc	mov ax, word [finddata.date]
   782                                  internaldatarelocation
   783 0000020A AB                      	stosw
   784                                  @@:
   785                                  
   786 0000020B 89D6                    	mov si, dx			; -> to insert, cx = length
   787 0000020D F3A4                    	rep movsb			; store new entry
   788 0000020F C3                      	retn
   789                                  
   790                                  .sort_insert_last:
   791 00000210 8B3E[6C04]              reloc	mov di, word [sort_last]	; -> after last
   792                                  internaldatarelocation
   793 00000214 E8D0FF                  	call .store_with_meta
   794 00000217 893E[6C04]              reloc	mov word [sort_last], di	; update -> after last
   795                                  internaldatarelocation
   796                                  
   797                                  .sort_inserted:
   798 0000021B 16                      	push ss
   799 0000021C 07                      	pop es
   800                                  
   801 0000021D EB03                    	jmp @F
   802                                  
   803                                  .display:
   804 0000021F E89701                  	call display_single
   805                                  @@:
   806                                  
   807                                  .next:
   808                                  %if _BOOT
   809                                  	test sp, sp		; NZ (continue search)
   810                                  	retn
   811                                  %else
   812 00000222 A1[7404]                reloc	mov ax, word [findnext_function_number]
   813                                  internaldatarelocation
   814 00000225 8B1E[7604]              reloc	mov bx, word [findhandle]
   815                                  internaldatarelocation
   816 00000229 57                      	push di
   817 0000022A BE0100                  	mov si, 1
   818 0000022D BF[A404]                reloc	mov di, finddata
   819                                  internaldatarelocation
   820 00000230 F9                      	stc
   821 00000231 E84C05                  	extcallcall _doscall
   822 00000234 5F                      	pop di
   823 00000235 7203E99BFE              	jnc .loop
   824                                  %endif
   825                                  
   826                                  %if _BOOT
   827                                  ..@boot_scan_end:
   828                                  %endif
   829                                  
   830 0000023A D006[0400]              reloc	rol byte [found], 1
   831                                  internaldatarelocation
   832 0000023E 7312                    	jnc .notfound
   833 00000240 D006[0900]              reloc	rol byte [sort], 1
   834                                  internaldatarelocation
   835 00000244 7233                    	jc sorted
   836 00000246 D006[0700]              reloc	rol byte [wide], 1
   837                                  internaldatarelocation
   838 0000024A 7303                    	jnc @F
   839                                  
   840                                  %if _BOOT
   841                                  reloc	mov di, [widecurrent]
   842                                  internaldatarelocation
   843                                  %endif
   844                                  
   845 0000024C E84905                  	extcallcall trimputs
   846                                  @@:
   847 0000024F E84E05                  	extcallcall cmd3
   848                                  
   849                                  
   850                                  .notfound:
   851 00000252 BA[2302]                reloc	mov dx, msg.notfound
   852                                  internaldatarelocation
   853 00000255 B8220E                  	mov ax, 0E22h
   854                                  @@:
   855 00000258 E84D05                  	extcallcall setrc
   856 0000025B E85205                  	extcallcall putsz
   857 0000025E E83F05                  	extcallcall cmd3
   858                                  
   859                                  .error:
   860 00000261 BA[9F01]                reloc	mov dx, msg.error
   861                                  internaldatarelocation
   862 00000264 B8230E                  	mov ax, 0E23h
   863 00000267 EBEF                    	jmp @B
   864                                  
   865                                  .error2:
   866 00000269 BA[C601]                reloc	mov dx, msg.error2
   867                                  internaldatarelocation
   868 0000026C B8240E                  	mov ax, 0E24h
   869 0000026F EBE7                    	jmp @B
   870                                  
   871                                  .toofull:
   872 00000271 BA[E801]                reloc	mov dx, msg.toofull
   873                                  internaldatarelocation
   874 00000274 B8250E                  	mov ax, 0E25h
   875 00000277 EBDF                    	jmp @B
   876                                  
   877                                  
   878                                  sorted:
   879                                  	houdini
   880                                  %ifn _BOOT
   881 00000279 E88304                  	call findclose
   882                                  %endif
   883                                  
   884 0000027C 8B3E[7004]              reloc	mov di, word [pathname_start]
   885                                  internaldatarelocation
   886                                  
   887                                  .find_dir:
   888 00000280 89FB                    	mov bx, di		; bx -> start of path
   889 00000282 B9FFFF                  	mov cx, -1
   890 00000285 B000                    	mov al, 0
   891 00000287 F2AE                    	repne scasb
   892 00000289 4F                      	dec di
   893                                  @@:
   894 0000028A 39DF                    	cmp di, bx
   895 0000028C 7611                    	jbe .di
   896 0000028E 4F                      	dec di
   897 0000028F 803D2F                  	cmp byte [di], '/'
   898 00000292 740A                    	je .di_plus_one
   899 00000294 803D5C                  	cmp byte [di], '\'
   900 00000297 7405                    	je .di_plus_one
   901 00000299 803D3A                  	cmp byte [di], ':'
   902 0000029C 75EC                    	jne @B
   903                                  .di_plus_one:
   904 0000029E 47                      	inc di
   905                                  .di:				; di -> end of path
   906 0000029F 89F9                    	mov cx, di
   907 000002A1 29D9                    	sub cx, bx		; = length of path
   908                                  
   909 000002A3 890E[7204]              reloc	mov word [pathname_length], cx
   910                                  internaldatarelocation
   911                                  
   912 000002A7 BF[0000]                reloc	mov di, relocateddata
   913                                  linkdatarelocation line_out
   914                                  
   915                                  .loop:
   916 000002AA 57                      	push di
   917 000002AB 8B1E[7204]              reloc	mov bx, word [pathname_length]
   918                                  internaldatarelocation
   919 000002AF 8B36[7004]              reloc	mov si, word [pathname_start]
   920                                  internaldatarelocation
   921 000002B3 89D9                    	mov cx, bx
   922 000002B5 81F90002                	cmp cx, buffer_end - buffer
   923 000002B9 73A6                    	jae .error
   924                                  
   925 000002BB BF[7804]                reloc	mov di, buffer
   926                                  internaldatarelocation
   927 000002BE F3A4                    	rep movsb
   928 000002C0 89FA                    	mov dx, di
   929                                  
   930 000002C2 8B3E[6E04]              reloc	mov di, word [sort_next]
   931                                  internaldatarelocation
   932 000002C6 3B3E[6C04]              reloc	cmp di, word [sort_last]
   933                                  internaldatarelocation
   934 000002CA 7344                    	jae .end
   935 000002CC 033E[0000]              reloc	add di, word [meta]
   936                                  internaldatarelocation
   937 000002D0 89FE                    	mov si, di
   938                                  
   939 000002D2 8E06[6604]              reloc	mov es, word [sortsegsel]
   940                                  internaldatarelocation
   941 000002D6 B000                    	mov al, 0
   942 000002D8 B90002                  	mov cx, 512
   943 000002DB F2AE                    	repne scasb
   944 000002DD 7582                    	jne .error
   945 000002DF 89F9                    	mov cx, di
   946 000002E1 29F1                    	sub cx, si
   947                                  
   948 000002E3 01CB                    	add bx, cx
   949 000002E5 81FB0002                	cmp bx, buffer_end - !!_BOOT - buffer
   950 000002E9 7603E973FF              	ja .error
   951                                  
   952 000002EE 89D7                    	mov di, dx
   953                                  %if _BOOT
   954                                  reloc	cmp di, strict word buffer
   955                                  internaldatarelocation
   956                                  	je .slash
   957                                  	cmp byte [di - 1], '/'
   958                                  	je .notslash
   959                                  	cmp byte [di - 1], '\'
   960                                  	je .notslash
   961                                  .slash:
   962                                  	mov byte [di], '/'
   963                                  	inc di
   964                                  .notslash:
   965                                  reloc	mov word [wild_pattern], di
   966                                  internaldatarelocation
   967                                  %endif
   968 000002F0 06                      	 push es
   969 000002F1 1E                      	 push ds
   970 000002F2 07                      	 pop es
   971 000002F3 1F                      	 pop ds				; swap
   972 000002F4 F3A4                    	rep movsb
   973 000002F6 16                      	 push ss
   974 000002F7 1F                      	 pop ds				; reset
   975 000002F8 8936[6E04]              reloc	mov word [sort_next], si
   976                                  internaldatarelocation
   977                                  
   978 000002FC BA[7804]                reloc	mov dx, buffer
   979                                  internaldatarelocation
   980                                  %if _BOOT
   981                                  	pop di
   982                                  
   983                                  	mov bx, dx
   984                                  reloc	clropt [relocateddata], dif3_auxbuff_guarded_1
   985                                  linkdatarelocation internalflags3, -3
   986                                  	extcallcall yy_boot_init_dir2
   987                                  
   988                                  reloc2	mov word [matchfunction], display_ZR
   989                                  internaldatarelocation -4
   990                                  internalcoderelocation
   991                                  
   992                                  	call boot_scan
   993                                  
   994                                  	jmp .loop
   995                                  
   996                                  .error equ sort_or_display.error
   997                                  .error2 equ sort_or_display.error2
   998                                  %else
   999 000002FF E81E02                  	call findfirst
  1000 00000302 7303E962FF              	jc .error2
  1001                                  
  1002 00000307 E8F503                  	call findclose
  1003 0000030A 5F                      	pop di
  1004 0000030B E8AB00                  	call display_single
  1005 0000030E EB9A                    	jmp .loop
  1006                                  
  1007                                  .error equ run_dos.error
  1008                                  .error2 equ run_dos.error2
  1009                                  %endif
  1010                                  
  1011                                  .end:
  1012 00000310 5F                      	pop di
  1013 00000311 D006[0700]              reloc	rol byte [wide], 1
  1014                                  internaldatarelocation
  1015 00000315 7303                    	jnc @F
  1016                                  
  1017                                  %if _BOOT
  1018                                  reloc	mov di, [widecurrent]
  1019                                  internaldatarelocation
  1020                                  %endif
  1021                                  
  1022 00000317 E87E04                  	extcallcall trimputs
  1023                                  @@:
  1024 0000031A E88304                  	extcallcall cmd3
  1025                                  
  1026                                  
  1027                                  populate_finddata:
  1028                                  %ifn _BOOT
  1029 0000031D 803E[7504]71            reloc	cmp byte [findnext_function_number + 1], 71h
  1030                                  internaldatarelocation -3
  1031 00000322 7436                    	je .have_lfn
  1032                                  
  1033 00000324 A0[8D04]                reloc	mov al, byte [dta.attrib]
  1034                                  internaldatarelocation
  1035 00000327 A2[A404]                reloc	mov byte [finddata.attrib], al
  1036                                  internaldatarelocation
  1037                                  
  1038 0000032A A1[8E04]                reloc	mov ax, word [dta.time]
  1039                                  internaldatarelocation
  1040 0000032D A3[B804]                reloc	mov word [finddata.time], ax
  1041                                  internaldatarelocation
  1042                                  
  1043 00000330 A1[9004]                reloc	mov ax, word [dta.date]
  1044                                  internaldatarelocation
  1045 00000333 A3[BA04]                reloc	mov word [finddata.date], ax
  1046                                  internaldatarelocation
  1047                                  
  1048 00000336 A1[9204]                reloc	mov ax, word [dta.size]
  1049                                  internaldatarelocation
  1050 00000339 A3[C404]                reloc	mov word [finddata.sizelow], ax
  1051                                  internaldatarelocation
  1052                                  
  1053 0000033C A1[9404]                reloc	mov ax, word [dta.size + 2]
  1054                                  internaldatarelocation
  1055 0000033F A3[C604]                reloc	mov word [finddata.sizelow + 2], ax
  1056                                  internaldatarelocation
  1057                                  
  1058 00000342 31C0                    	xor ax, ax
  1059 00000344 A3[C004]                reloc	mov word [finddata.sizehigh], ax
  1060                                  internaldatarelocation
  1061 00000347 A3[C204]                reloc	mov word [finddata.sizehigh + 2], ax
  1062                                  internaldatarelocation
  1063                                  
  1064 0000034A 57                      	push di
  1065 0000034B BE[9604]                reloc	mov si, dta.name
  1066                                  internaldatarelocation
  1067 0000034E BF[D004]                reloc	mov di, finddata.fullname
  1068                                  internaldatarelocation
  1069 00000351 B90700                  	mov cx, words(14)
  1070 00000354 F3A5                    	rep movsw
  1071 00000356 5F                      	pop di
  1072                                  
  1073 00000357 A2[D405]                reloc	mov byte [finddata.shortname], al
  1074                                  internaldatarelocation
  1075                                  
  1076                                  .have_lfn:
  1077                                  %endif
  1078                                  
  1079 0000035A 57                      	push di
  1080 0000035B BF[E205]                reloc	mov di, size40bit
  1081                                  internaldatarelocation
  1082 0000035E F606[A404]10            reloc	test byte [finddata.attrib], ATTR_DIRECTORY
  1083                                  internaldatarelocation -3
  1084 00000363 740E                    	jz @F
  1085 00000365 31C0                    	xor ax, ax
  1086 00000367 A3[C404]                reloc	mov word [finddata.sizelow], ax
  1087                                  internaldatarelocation
  1088 0000036A A3[C604]                reloc	mov word [finddata.sizelow + 2], ax
  1089                                  internaldatarelocation
  1090 0000036D A3[C004]                reloc	mov word [finddata.sizehigh], ax
  1091                                  internaldatarelocation
  1092 00000370 A3[C204]                reloc	mov word [finddata.sizehigh + 2], ax
  1093                                  internaldatarelocation
  1094                                  @@:
  1095 00000373 833E[C204]00            reloc	cmp word [finddata.sizehigh + 2], strict byte 0
  1096                                  internaldatarelocation -3
  1097 00000378 7516                    	jne .sizelarge
  1098 0000037A 813E[C004]0001          reloc	cmp word [finddata.sizehigh], 256
  1099                                  internaldatarelocation -4
  1100 00000380 730E                    	jae .sizelarge
  1101 00000382 A1[C404]                reloc	mov ax, word [finddata.sizelow]
  1102                                  internaldatarelocation
  1103 00000385 AB                      	stosw
  1104 00000386 A1[C604]                reloc	mov ax, word [finddata.sizelow + 2]
  1105                                  internaldatarelocation
  1106 00000389 AB                      	stosw
  1107 0000038A A0[C004]                reloc	mov al, byte [finddata.sizehigh]
  1108                                  internaldatarelocation
  1109 0000038D AA                      	stosb
  1110 0000038E EB06                    	jmp @F
  1111                                  
  1112                                  .sizelarge:
  1113 00000390 B8FFFF                  	mov ax, 0FFFFh
  1114 00000393 AB                      	stosw
  1115 00000394 AB                      	stosw
  1116 00000395 AA                      	stosb
  1117                                  @@:
  1118 00000396 5F                      	pop di
  1119                                  
  1120 00000397 BE[D405]                reloc	mov si, finddata.shortname
  1121                                  internaldatarelocation
  1122 0000039A 803C00                  	cmp byte [si], 0
  1123 0000039D 7503                    	jne @F
  1124 0000039F BE[D004]                reloc	mov si, finddata.fullname
  1125                                  internaldatarelocation
  1126                                  @@:
  1127                                  
  1128 000003A2 803C2E                  	cmp byte [si], '.'	; dot ?
  1129 000003A5 750A                    	jne @F			; no --> NZ
  1130 000003A7 837C012E                	cmp word [si + 1], "."	; dot and NUL ?
  1131 000003AB 7404                    	je .next		; dotdot, skip --> ZR
  1132 000003AD 807C0100                	cmp byte [si + 1], 0	; NUL ?
  1133                                  	; je .next		; dot, skip --> ZR
  1134                                  .next:
  1135                                  @@:
  1136 000003B1 7405                    	je @F
  1137 000003B3 800E[0400]FF            reloc	or byte [found], -1
  1138                                  internaldatarelocation -3	; NZ
  1139                                  @@:
  1140 000003B8 C3                      	retn
  1141                                  
  1142                                  
  1143                                  %if _BOOT
  1144                                  display_ZR:
  1145                                  %endif
  1146                                  display_single:
  1147 000003B9 E861FF                  	call populate_finddata
  1148 000003BC 7503E95E01              	je .next
  1149                                  
  1150 000003C1 D006[0700]              reloc	rol byte [wide], 1
  1151                                  internaldatarelocation
  1152 000003C5 7338                    	jnc .notwide
  1153                                  
  1154                                  .wide:
  1155                                  	houdini
  1156                                  %if _BOOT
  1157                                  reloc	mov di, [widecurrent]
  1158                                  internaldatarelocation
  1159                                  %endif
  1160                                  
  1161 000003C7 FE06[0800]              reloc	inc byte [widecounter]
  1162                                  internaldatarelocation
  1163 000003CB 803E[0800]06            reloc	cmp byte [widecounter], 6
  1164                                  internaldatarelocation -3
  1165 000003D0 720B                    	jb @F
  1166 000003D2 E8C303                  	extcallcall trimputs
  1167 000003D5 BF[0000]                reloc	mov di, relocateddata
  1168                                  linkdatarelocation line_out
  1169 000003D8 C606[0800]01            reloc	mov byte [widecounter], 1
  1170                                  internaldatarelocation -3
  1171                                  @@:
  1172                                  
  1173 000003DD B420                    	mov ah, 32
  1174 000003DF B90F00                  	mov cx, 15		; width of column: 8 + 1 + 3 + 2 + 1
  1175 000003E2 F606[A404]10            reloc	test byte [finddata.attrib], ATTR_DIRECTORY
  1176                                  internaldatarelocation -3
  1177 000003E7 7405                    	jz @FF			; skip brackets and first iter stosb -->
  1178 000003E9 B85B5D                  	mov ax, "[]"		; use brackets
  1179 000003EC 49                      	dec cx			; decrement remaining width
  1180                                  @@:
  1181 000003ED AA                      	stosb			; dir first iter: store opening square bracket
  1182                                  				; file first iter: skipped
  1183                                  				; subsequent iter: store text byte
  1184                                  @@:
  1185 000003EE AC                      	lodsb			; load from name
  1186 000003EF 84C0                    	test al, al		; got a NUL ? do not loop if so
  1187 000003F1 E0FA                    	loopnz @BB		; decrements width once per text byte
  1188                                  				;  and finally once more for the NUL
  1189 000003F3 88E0                    	mov al, ah		; get blank or closing square bracket
  1190 000003F5 AA                      	stosb			; store blank or closing square bracket
  1191                                  				; (this store does not decrement the width)
  1192 000003F6 B020                    	mov al, 32		; pad with blanks
  1193 000003F8 E301                    	jcxz @F			; (error?) only once -->
  1194 000003FA F3                      	rep
  1195                                  @@:
  1196 000003FB AA                      	stosb			; store separator blanks
  1197                                  
  1198                                  %if _BOOT
  1199                                  reloc	mov [widecurrent], di
  1200                                  internaldatarelocation
  1201                                  %endif
  1202 000003FC E92001                  	jmp .next
  1203                                  
  1204                                  
  1205                                  .notwide:
  1206 000003FF BF[0000]                reloc	mov di, relocateddata
  1207                                  linkdatarelocation line_out
  1208 00000402 B90800                  	mov cx, 8
  1209                                  
  1210                                  @@:
  1211 00000405 AC                      	lodsb
  1212 00000406 3C2E                    	cmp al, '.'
  1213 00000408 740D                    	je @F
  1214 0000040A 3C00                    	cmp al, 0
  1215 0000040C 741A                    	je .no_ext
  1216 0000040E AA                      	stosb
  1217 0000040F E2F4                    	loop @B
  1218 00000411 AC                      	lodsb
  1219 00000412 3C2E                    	cmp al, '.'
  1220 00000414 7401                    	je @F
  1221 00000416 4E                      	dec si			; doesn't fit, nothing sensible here
  1222                                  
  1223                                  @@:
  1224 00000417 41                      	inc cx
  1225 00000418 B020                    	mov al, 32
  1226 0000041A F3AA                    	rep stosb
  1227                                  
  1228 0000041C B103                    	mov cl, 3
  1229                                  @@:
  1230 0000041E AC                      	lodsb
  1231 0000041F 3C00                    	cmp al, 0
  1232 00000421 7408                    	je @F
  1233 00000423 AA                      	stosb
  1234 00000424 E2F8                    	loop @B
  1235 00000426 EB03                    	jmp @F
  1236                                  
  1237                                  .no_ext:
  1238 00000428 83C104                  	add cx, 1 + 3
  1239                                  
  1240                                  @@:
  1241 0000042B 41                      	inc cx
  1242 0000042C 41                      	inc cx
  1243 0000042D B020                    	mov al, 32
  1244 0000042F F3AA                    	rep stosb
  1245                                  
  1246                                  
  1247 00000431 8A1E[A404]              reloc	mov bl, byte [finddata.attrib]
  1248                                  internaldatarelocation
  1249                                  
  1250 00000435 B02D                    	mov al, '-'
  1251 00000437 F6C320                  	test bl, ATTR_ARCHIVE
  1252 0000043A 7402                    	jz @F
  1253 0000043C B041                    	mov al, 'A'
  1254                                  @@:
  1255 0000043E AA                      	stosb
  1256 0000043F B02D                    	mov al, '-'
  1257 00000441 F6C302                  	test bl, ATTR_HIDDEN
  1258 00000444 7402                    	jz @F
  1259 00000446 B048                    	mov al, 'H'
  1260                                  @@:
  1261 00000448 AA                      	stosb
  1262 00000449 B02D                    	mov al, '-'
  1263 0000044B F6C301                  	test bl, ATTR_READONLY
  1264 0000044E 7402                    	jz @F
  1265 00000450 B052                    	mov al, 'R'
  1266                                  @@:
  1267 00000452 AA                      	stosb
  1268 00000453 B02D                    	mov al, '-'
  1269 00000455 F6C304                  	test bl, ATTR_SYSTEM
  1270 00000458 7402                    	jz @F
  1271 0000045A B053                    	mov al, 'S'
  1272                                  @@:
  1273 0000045C AA                      	stosb
  1274 0000045D B82020                  	mov ax, 2020h
  1275 00000460 AB                      	stosw
  1276                                  
  1277 00000461 F6C310                  	test bl, ATTR_DIRECTORY
  1278 00000464 7408                    	jz @F
  1279 00000466 BE[1102]                reloc	mov si, msg.dirinsteadsize
  1280                                  internaldatarelocation
  1281                                  .nosize:
  1282 00000469 E84C03                  	extcallcall copy_single_counted_string
  1283 0000046C EB1F                    	jmp @FF
  1284                                  
  1285                                  @@:
  1286 0000046E 833E[C204]00            reloc	cmp word [finddata.sizehigh + 2], strict byte 0
  1287                                  internaldatarelocation -3
  1288 00000473 7405                    	je .sizefits
  1289                                  
  1290 00000475 BE[1A02]                reloc	mov si, msg.sizetoolarge
  1291                                  internaldatarelocation
  1292 00000478 EBEF                    	jmp .nosize
  1293                                  
  1294                                  .sizefits:
  1295 0000047A 8B36[C004]              reloc	mov si, word [finddata.sizehigh] 	; from FAT+ upper size bits
  1296                                  internaldatarelocation
  1297 0000047E 8B16[C604]              reloc	mov dx, word [finddata.sizelow + 2]
  1298                                  internaldatarelocation
  1299 00000482 A1[C404]                reloc	mov ax, word [finddata.sizelow]
  1300                                  internaldatarelocation
  1301 00000485 31C9                    	xor cx, cx
  1302 00000487 BB0800                  	mov bx, 4+4
  1303 0000048A E83303                  	extcallcall disp_dxax_times_cx_width_bx_size.store
  1304                                  
  1305                                  @@:
  1306 0000048D B82020                  	mov ax, 2020h
  1307 00000490 AB                      	stosw
  1308 00000491 8B1E[BA04]              reloc	mov bx, word [finddata.date]
  1309                                  internaldatarelocation
  1310 00000495 8B36[B804]              reloc	mov si, word [finddata.time]
  1311                                  internaldatarelocation
  1312                                  
  1313 00000499 31D2                    	xor dx, dx
  1314 0000049B 85DB                    	test bx, bx
  1315 0000049D 750A                    	jnz @F
  1316 0000049F B82020                  	mov ax, 2020h
  1317 000004A2 B90500                  	mov cx, 5
  1318 000004A5 F3AB                    	rep stosw
  1319 000004A7 EB2B                    	jmp .nodate
  1320                                  
  1321                                  @@:
  1322 000004A9 89D8                    	mov ax, bx
  1323 000004AB B90900                  	mov cx, 9
  1324 000004AE D3E8                    	shr ax, cl
  1325 000004B0 05BC07                  	add ax, 1980
  1326 000004B3 B104                    	mov cl, 4
  1327 000004B5 E81003                  	extcallcall dec_dword_minwidth
  1328 000004B8 B02D                    	mov al, '-'
  1329 000004BA AA                      	stosb
  1330 000004BB 89D8                    	mov ax, bx
  1331 000004BD B105                    	mov cl, 5
  1332 000004BF D3E8                    	shr ax, cl
  1333 000004C1 83E00F                  	and ax, 15
  1334 000004C4 B102                    	mov cl, 2
  1335 000004C6 E8FF02                  	extcallcall dec_dword_minwidth
  1336 000004C9 B02D                    	mov al, '-'
  1337 000004CB AA                      	stosb
  1338 000004CC 89D8                    	mov ax, bx
  1339 000004CE 83E01F                  	and ax, 31
  1340 000004D1 E8F402                  	extcallcall dec_dword_minwidth
  1341                                  .nodate:
  1342 000004D4 B020                    	mov al, 32
  1343 000004D6 AA                      	stosb
  1344 000004D7 89F0                    	mov ax, si
  1345 000004D9 B10B                    	mov cl, 11
  1346 000004DB D3E8                    	shr ax, cl
  1347 000004DD B102                    	mov cl, 2
  1348 000004DF E8E602                  	extcallcall dec_dword_minwidth
  1349 000004E2 B03A                    	mov al, ':'
  1350 000004E4 AA                      	stosb
  1351 000004E5 89F0                    	mov ax, si
  1352 000004E7 B105                    	mov cl, 5
  1353 000004E9 D3E8                    	shr ax, cl
  1354 000004EB 83E03F                  	and ax, 63
  1355 000004EE B102                    	mov cl, 2
  1356 000004F0 E8D502                  	extcallcall dec_dword_minwidth
  1357 000004F3 B03A                    	mov al, ':'
  1358 000004F5 AA                      	stosb
  1359 000004F6 89F0                    	mov ax, si
  1360 000004F8 83E01F                  	and ax, 31
  1361 000004FB D1E0                    	shl ax, 1
  1362 000004FD E8C802                  	extcallcall dec_dword_minwidth
  1363                                  
  1364 00000500 803E[D405]00            reloc	cmp byte [finddata.shortname], 0
  1365                                  internaldatarelocation -3
  1366 00000505 7415                    	je @F
  1367 00000507 B82020                  	mov ax, 2020h
  1368 0000050A AB                      	stosw
  1369 0000050B E8C202                  	extcallcall putsline
  1370 0000050E BA[D004]                reloc	mov dx, finddata.fullname
  1371                                  internaldatarelocation
  1372 00000511 E89C02                  	extcallcall putsz
  1373 00000514 BA[3202]                reloc	mov dx, msg.linebreak
  1374                                  internaldatarelocation
  1375 00000517 E89602                  	extcallcall putsz
  1376 0000051A EB03                    	jmp .next
  1377                                  
  1378                                  @@:
  1379 0000051C E8B902                  	extcallcall putsline_crlf
  1380                                  
  1381                                  .next:
  1382                                  %if _BOOT
  1383                                  	cmp al, al		; ZR
  1384                                  %endif
  1385 0000051F C3                      	retn
  1386                                  
  1387                                  
  1388                                  %ifn _BOOT
  1389                                  findfirst:
  1390 00000520 C706[7404]4F71          reloc	mov word [findnext_function_number], 714Fh
  1391                                  internaldatarelocation -4
  1392 00000526 B84E71                  	mov ax, 714Eh
  1393 00000529 B91600                  	mov cx, 16h		; find all files and directories
  1394 0000052C BE0100                  	mov si, 1
  1395 0000052F BF[A404]                reloc	mov di, finddata
  1396                                  internaldatarelocation
  1397 00000532 D006[0600]              reloc	rol byte [prefersfn], 1
  1398                                  internaldatarelocation
  1399 00000536 721B                    	jc .sfn_try
  1400 00000538 F9                      	stc
  1401 00000539 E84402                  	extcallcall _doscall
  1402 0000053C 730C                    	jnc .lfn_found
  1403 0000053E 83F801                  	cmp ax, 1
  1404 00000541 7410                    	je .sfn_try
  1405 00000543 3D0071                  	cmp ax, 7100h
  1406 00000546 740B                    	je .sfn_try
  1407 00000548 F9                      	stc	; CY
  1408 00000549 C3                      	retn
  1409                                  
  1410                                  .lfn_found:
  1411 0000054A A3[7604]                reloc	mov word [findhandle], ax
  1412                                  internaldatarelocation
  1413 0000054D C606[0500]FF            reloc	mov byte [findhandle_set], 0FFh
  1414                                  internaldatarelocation -3
  1415                                  		; NC
  1416 00000552 C3                      	retn
  1417                                  
  1418                                  .sfn_try:
  1419 00000553 C706[7404]004F          reloc	mov word [findnext_function_number], 4F00h
  1420                                  internaldatarelocation -4
  1421 00000559 B8004E                  	mov ax, 4E00h
  1422 0000055C B91600                  	mov cx, 16h		; find all files and directories
  1423 0000055F E81E02                  	extcallcall _doscall
  1424                                  		; CY if not found
  1425 00000562 C3                      	retn
  1426                                  %endif
  1427                                  
  1428                                  
  1429                                  %if _BOOT
  1430                                  find_dir:
  1431                                  	mov bx, di		; bx -> start of path
  1432                                  	mov cx, -1
  1433                                  	mov al, 0
  1434                                  	repne scasb
  1435                                  	dec di
  1436                                  @@:
  1437                                  	cmp di, bx
  1438                                  	jbe .di
  1439                                  	dec di
  1440                                  	cmp byte [di], '/'
  1441                                  	je .di_plus_one
  1442                                  	cmp byte [di], '\'
  1443                                  	je .di_plus_one
  1444                                  	cmp byte [di], ':'
  1445                                  	jne @B
  1446                                  .di_plus_one:
  1447                                  	inc di
  1448                                  .di:				; di -> end of path
  1449                                  	retn
  1450                                  %endif
  1451                                  
  1452                                  
  1453                                  parse_verbose.loop:
  1454 00000563 AC                      	lodsb
  1455                                  parse_verbose:
  1456 00000564 E87902                  	extcallcall skipcomm0
  1457 00000567 E87E02                  	extcallcall iseol?
  1458 0000056A 7526                    	jne .parse
  1459                                  
  1460                                  .meta:
  1461 0000056C D006[0C00]              reloc	rol byte [date], 1
  1462                                  internaldatarelocation
  1463 00000570 730A                    	jnc @F
  1464 00000572 C606[0D00]00            reloc	mov byte [size], 0
  1465                                  internaldatarelocation -3
  1466 00000577 8006[0000]04            reloc	add byte [meta], 4
  1467                                  internaldatarelocation -3
  1468                                  @@:
  1469                                  
  1470 0000057C D006[0D00]              reloc	rol byte [size], 1
  1471                                  internaldatarelocation
  1472 00000580 7305                    	jnc @F
  1473 00000582 8006[0000]05            reloc	add byte [meta], 5
  1474                                  internaldatarelocation -3
  1475                                  @@:
  1476                                  
  1477 00000587 D006[0B00]              reloc	rol byte [dirfirst], 1
  1478                                  internaldatarelocation
  1479 0000058B 7304                    	jnc @F
  1480 0000058D FE06[0000]              reloc	inc byte [meta]
  1481                                  internaldatarelocation
  1482                                  @@:
  1483 00000591 C3                      	retn
  1484                                  
  1485                                  .parse:
  1486 00000592 4E                      	dec si
  1487                                  %ifn _BOOT
  1488 00000593 BA[0E00]                reloc	mov dx, msg.string_sfn
  1489                                  internaldatarelocation
  1490 00000596 E85702                  	extcallcall isstring?
  1491 00000599 7507                    	jne @F
  1492 0000059B C606[0600]FF            reloc	mov byte [prefersfn], 0FFh
  1493                                  internaldatarelocation -3
  1494 000005A0 EBC1                    	jmp .loop
  1495                                  
  1496                                  @@:
  1497                                  %endif
  1498 000005A2 BA[1200]                reloc	mov dx, msg.string_wide
  1499                                  internaldatarelocation
  1500 000005A5 E84802                  	extcallcall isstring?
  1501 000005A8 7507                    	jne @F
  1502 000005AA C606[0700]FF            reloc	mov byte [wide], 0FFh
  1503                                  internaldatarelocation -3
  1504 000005AF EBB2                    	jmp .loop
  1505                                  
  1506                                  @@:
  1507 000005B1 BA[1700]                reloc	mov dx, msg.string_sort
  1508                                  internaldatarelocation
  1509 000005B4 E83902                  	extcallcall isstring?
  1510 000005B7 7507                    	jne @F
  1511                                  .loop_sort:
  1512 000005B9 C606[0900]FF            reloc	mov byte [sort], 0FFh
  1513                                  internaldatarelocation -3
  1514 000005BE EBA3                    	jmp .loop
  1515                                  @@:
  1516 000005C0 BA[1C00]                reloc	mov dx, msg.string_dirfirst
  1517                                  internaldatarelocation
  1518 000005C3 E82A02                  	extcallcall isstring?
  1519 000005C6 7507                    	jne @F
  1520 000005C8 C606[0B00]FF            reloc	mov byte [dirfirst], 0FFh
  1521                                  internaldatarelocation -3
  1522 000005CD EB94                    	jmp .loop
  1523                                  
  1524                                  @@:
  1525 000005CF BA[2500]                reloc	mov dx, msg.string_date
  1526                                  internaldatarelocation
  1527 000005D2 E81B02                  	extcallcall isstring?
  1528 000005D5 7507                    	jne @F
  1529 000005D7 C606[0C00]FF            reloc	mov byte [date], 0FFh
  1530                                  internaldatarelocation -3
  1531 000005DC EB85                    	jmp .loop
  1532                                  @@:
  1533 000005DE BA[2A00]                reloc	mov dx, msg.string_size
  1534                                  internaldatarelocation
  1535 000005E1 E80C02                  	extcallcall isstring?
  1536 000005E4 7508                    	jne @F
  1537 000005E6 C606[0D00]FF            reloc	mov byte [size], 0FFh
  1538                                  internaldatarelocation -3
  1539 000005EB E975FF                  	jmp .loop
  1540                                  
  1541                                  @@:
  1542 000005EE BA[2F00]                reloc	mov dx, msg.string_reverse
  1543                                  internaldatarelocation
  1544 000005F1 E8FC01                  	extcallcall isstring?
  1545 000005F4 7509                    	jne @F
  1546 000005F6 C706[0200][A301]        reloc2	mov word [compare], ..@compare_reverse
  1547                                  internaldatarelocation -4
  1548                                  internalcoderelocation
  1549 000005FC E964FF                  	jmp .loop
  1550                                  
  1551                                  @@:
  1552                                  %ifn _BOOT
  1553 000005FF BA[3700]                reloc	mov dx, msg.string_sortlfn
  1554                                  internaldatarelocation
  1555 00000602 E8EB01                  	extcallcall isstring?
  1556 00000605 7507                    	jne @F
  1557 00000607 C606[0A00]FF            reloc	mov byte [sortlfn], 0FFh
  1558                                  internaldatarelocation -3
  1559 0000060C EBAB                    	jmp .loop_sort
  1560                                  
  1561                                  @@:
  1562 0000060E BA[3F00]                reloc	mov dx, msg.string_sortsfn
  1563                                  internaldatarelocation
  1564 00000611 E8DC01                  	extcallcall isstring?
  1565 00000614 7507                    	jne @F
  1566 00000616 C606[0A00]00            reloc	mov byte [sortlfn], 0
  1567                                  internaldatarelocation -3
  1568 0000061B EB9C                    	jmp .loop_sort
  1569                                  
  1570                                  @@:
  1571                                  %endif
  1572                                  %if _DEBUG
  1573 0000061D BA[4700]                reloc	mov dx, msg.string_sortdebug
  1574                                  internaldatarelocation
  1575 00000620 E8CD01                  	extcallcall isstring?
  1576 00000623 7403                    	je @F
  1577                                  %endif
  1578 00000625 E8D001                  	extcallcall error
  1579                                  
  1580                                  %if _DEBUG
  1581                                  @@:
  1582 00000628 AC                      	lodsb
  1583 00000629 E8D401                  	extcallcall chkeol
  1584                                  
  1585 0000062C E83DFF                  	call .meta
  1586                                  
  1587                                  %if _BOOT
  1588                                  	extcallcall yy_boot_init_dir2
  1589                                  
  1590                                  	mov dx, word [bp + bsBPB + bpbBytesPerSector]
  1591                                  					; di = sector size
  1592                                  					; = start of available auxbuff
  1593                                  	cmp byte [bp + ldFATType], 12	; FAT12 ?
  1594                                  	jne @F				; no -->
  1595                                  	cmp dx, 8192			; already enough for a full FAT ?
  1596                                  	jae @F				; yes -->
  1597                                  	add dx, dx			; reserve straddling sector
  1598                                  @@:
  1599                                  %endif
  1600                                  
  1601 0000062F BF[0000]                reloc	mov di, relocateddata
  1602                                  linkdatarelocation line_out
  1603                                  
  1604 00000632 BE[5100]                reloc	mov si, msg.debug.1
  1605                                  internaldatarelocation
  1606 00000635 E88001                  	extcallcall copy_single_counted_string
  1607                                  
  1608 00000638 8CD0                    	mov ax, ss
  1609 0000063A E8CB01                  	extcallcall hexword
  1610 0000063D B03A                    	mov al, ':'
  1611 0000063F AA                      	stosb
  1612 00000640 B8[7806]                reloc	mov ax, buffer_end
  1613                                  internaldatarelocation
  1614 00000643 E8C201                  	extcallcall hexword
  1615                                  
  1616 00000646 A1[0000]                reloc	mov ax, word [relocateddata]
  1617                                  linkdatarelocation extdata_size
  1618 00000649 2B06[0000]              reloc	sub ax, word [relocateddata]
  1619                                  linkdatarelocation extdata_used
  1620 0000064D 8B1E[0000]              reloc	mov bx, word [relocateddata]
  1621                                  linkdatarelocation auxbuff_current_size
  1622                                  %if _BOOT
  1623                                  	sub bx, dx
  1624                                  	push dx
  1625                                  %endif
  1626                                  
  1627 00000651 BE[6B00]                reloc	mov si, msg.debug.2
  1628                                  internaldatarelocation
  1629 00000654 E86101                  	extcallcall copy_single_counted_string
  1630                                  
  1631 00000657 83C008                  	add ax, (uinit_data_end_2 - buffer_end)
  1632 0000065A E84500                  	call display_buffer_size
  1633                                  
  1634 0000065D BE[7E00]                reloc	mov si, msg.debug.3
  1635                                  internaldatarelocation
  1636 00000660 E85501                  	extcallcall copy_single_counted_string
  1637                                  
  1638 00000663 BA[DD00]                reloc	mov dx, msg.debug.larger_data_block
  1639                                  internaldatarelocation
  1640                                  
  1641 00000666 39D8                    	cmp ax, bx
  1642 00000668 730D                    	jae .use_sort_buffer_eld_data_block
  1643                                  
  1644 0000066A BA[1D01]                reloc	mov dx, msg.debug.smaller_data_block
  1645                                  internaldatarelocation
  1646                                  
  1647                                  %ifn _BOOT
  1648 0000066D F606[0300]70            reloc	testopt [relocateddata], dif3_auxbuff_guarded_1 		| dif3_auxbuff_guarded_2 		| dif3_auxbuff_guarded_3
  1651                                  linkdatarelocation internalflags3, -3
  1652 00000672 7403                    	jz .use_sort_buffer_auxbuff
  1653                                  
  1654 00000674 BA[5B01]                reloc	mov dx, msg.debug.smaller_data_block_forced
  1655                                  internaldatarelocation
  1656                                  %endif
  1657                                  
  1658                                  .use_sort_buffer_eld_data_block:
  1659                                  .use_sort_buffer_auxbuff:
  1660                                  
  1661 00000677 A1[0000]                reloc	mov ax, word [relocateddata]
  1662                                  linkdatarelocation auxbuff_segorsel	; => sort buffer
  1663 0000067A E88B01                  	extcallcall hexword
  1664                                  
  1665                                  %if _BOOT
  1666                                  	mov al, ':'
  1667                                  	stosb
  1668                                  	pop ax
  1669                                  	extcallcall hexword
  1670                                  %endif
  1671                                  
  1672 0000067D 93                      	xchg ax, bx
  1673 0000067E BE[A100]                reloc	mov si, msg.debug.5
  1674                                  internaldatarelocation
  1675 00000681 E83401                  	extcallcall copy_single_counted_string
  1676 00000684 E81B00                  	call display_buffer_size
  1677                                  
  1678 00000687 BE[AE00]                reloc	mov si, msg.debug.6.available
  1679                                  internaldatarelocation
  1680                                  
  1681 0000068A F606[0300]70            reloc	testopt [relocateddata], dif3_auxbuff_guarded_1 		| dif3_auxbuff_guarded_2 		| dif3_auxbuff_guarded_3
  1684                                  linkdatarelocation internalflags3, -3
  1685 0000068F 7403                    	jz @F
  1686                                  
  1687 00000691 BE[C700]                reloc	mov si, msg.debug.6.inuse
  1688                                  internaldatarelocation
  1689                                  @@:
  1690                                  
  1691 00000694 E82101                  	extcallcall copy_single_counted_string
  1692 00000697 52                      	push dx
  1693 00000698 E83D01                  	extcallcall putsline_crlf
  1694 0000069B 5A                      	pop dx
  1695                                  
  1696 0000069C E81101                  	extcallcall putsz
  1697 0000069F E8FE00                  	extcallcall cmd3
  1698                                  
  1699                                  
  1700                                  display_buffer_size:
  1701 000006A2 E86B01                  	extcallcall decword
  1702 000006A5 BE[7300]                reloc	mov si, msg.debug.bytes
  1703                                  internaldatarelocation
  1704 000006A8 E80D01                  	extcallcall copy_single_counted_string
  1705 000006AB 50                      	push ax
  1706 000006AC 52                      	push dx
  1707 000006AD 31D2                    	xor dx, dx
  1708 000006AF BE0D00                  	mov si, 8 + 1 + 3 + 1		; ASCIZ SFN maximum length
  1709 000006B2 0336[0000]              reloc	add si, word [meta]
  1710                                  internaldatarelocation
  1711 000006B6 F7F6                    	div si
  1712 000006B8 E85501                  	extcallcall decword
  1713 000006BB 5A                      	pop dx
  1714 000006BC 58                      	pop ax
  1715 000006BD C3                      	retn
  1716                                  %endif
  1717                                  
  1718                                  
  1719                                  %ifn _BOOT
  1720                                  inject:
  1721 000006BE 8B16[6004]              reloc	mov dx, word [originaldta]	; dx -> original DTA
  1722                                  internaldatarelocation
  1723 000006C2 B41A                    	mov ah, 1Ah			; set DTA (restoring)
  1724 000006C4 E8B100                  	extcallcall ispm
  1725 000006C7 7511                    	jnz .rm
  1726                                  
  1727                                  subcpu 286
  1728 000006C9 FF36[6204]              reloc	push word [originaldta + 2]
  1729                                  internaldatarelocation			; ds => original DTA (86M segment)
  1730 000006CD 6A21                    	push word 21h
  1731 000006CF E8[0000]EB020000        	extcall intcall_ext_return_es, PM required	; must NOT be extcallcall
  1732 000006D6 5A                      	pop dx				; discard interrupt number
  1733 000006D7 5A                      	pop dx				; discard es
  1734                                  subcpureset
  1735 000006D8 EB08                    	jmp @F
  1736                                  .rm:
  1737 000006DA 8E1E[6204]              reloc	mov ds, word [originaldta + 2]	; ds => original DTA
  1738                                  internaldatarelocation
  1739 000006DE CD21                    	int 21h
  1740 000006E0 16                      	 push ss
  1741 000006E1 1F                      	 pop ds
  1742                                  @@:
  1743                                  
  1744 000006E2 E81A00                  	call findclose
  1745                                  
  1746 000006E5 8B0E[6404]              reloc	mov cx, word [originalinject]
  1747                                  internaldatarelocation
  1748 000006E9 E82800                  	call get_es_ext
  1749 000006EC 268026[1000]FE          reloc	clropt [es:code + eldiFlags], eldifResident
  1750                                  internalcoderelocation -3		; mark block as no longer resident
  1751 000006F2 16                      	 push ss
  1752 000006F3 07                      	 pop es
  1753 000006F4 E302                    	jcxz @F
  1754 000006F6 FFE1                    	jmp cx
  1755                                  
  1756                                  @@:
  1757 000006F8 E8[0000]EB020000        	extcall cmd3_not_inject
  1758                                  
  1759                                  
  1760                                  findclose:
  1761 000006FF 8B1E[7604]              reloc	mov bx, word [findhandle]	; bx = find handle, if any
  1762                                  internaldatarelocation
  1763 00000703 D006[0500]              reloc	rol byte [findhandle_set], 1	; find handle set ?
  1764                                  internaldatarelocation
  1765 00000707 730A                    	jnc @F				; no -->
  1766 00000709 F616[0500]              reloc	not byte [findhandle_set]
  1767                                  internaldatarelocation
  1768 0000070D B8A171                  	mov ax, 71A1h
  1769 00000710 E86D00                  	extcallcall _doscall		; LFN find close
  1770                                  @@:
  1771 00000713 C3                      	retn
  1772                                  %endif
  1773                                  
  1774                                  
  1775                                  get_es_ext:
  1776 00000714 8E06[0000]              reloc	mov es, word [relocateddata]
  1777                                  linkdatarelocation extdssel
  1778 00000718 E85D00                  	extcallcall ispm
  1779 0000071B 7404                    	jz @F
  1780 0000071D 8E06[0000]              reloc	mov es, word [relocateddata]
  1781                                  linkdatarelocation extseg
  1782                                  @@:
  1783 00000721 C3                      	retn
  1784                                  
  1785                                  
  1786                                  start:
  1787 00000722 8CC3                    	mov bx, es
  1788 00000724 16                      	 push ss
  1789 00000725 07                      	 pop es
  1790 00000726 E8EF00                  	extcallcall skipcomma
  1791 00000729 E8BC00                  	extcallcall iseol?
  1792 0000072C 7409                    	je .help
  1793 0000072E E8EFF8                  	call run
  1794                                  @@:
  1795 00000731 E80B00                  	call uninstall_oneshot
  1796 00000734 31C0                    	xor ax, ax
  1797 00000736 CB                      	retf
  1798                                  
  1799                                  .help:
  1800 00000737 BA[3502]                reloc	mov dx, msg.help
  1801                                  internaldatarelocation
  1802 0000073A E87300                  	extcallcall putsz
  1803 0000073D EBF2                    	jmp @B
  1804                                  
  1805                                  
  1806                                  uninstall_oneshot:
  1807 0000073F 36F606[0000]01          reloc	testopt [ss:relocateddata], 1
  1808                                  linkdatarelocation options7, -3
  1809 00000745 751A                    	jnz @F
  1810                                  
  1811 00000747 2EA1[0200]              reloc	mov ax, word [cs:code + eldiEndCode]
  1812                                  internalcoderelocation
  1813 0000074B 2E2B06[0000]            reloc	sub ax, word [cs:code + eldiStartCode]
  1814                                  internalcoderelocation
  1815 00000750 2906[0000]              reloc	sub word [relocateddata], ax
  1816                                  linkdatarelocation extseg_used
  1817                                  
  1818 00000754 2EA1[0600]              reloc	mov ax, word [cs:code + eldiEndData]
  1819                                  internalcoderelocation
  1820 00000758 2E2B06[0400]            reloc	sub ax, word [cs:code + eldiStartData]
  1821                                  internalcoderelocation
  1822 0000075D 2906[0000]              reloc	sub word [relocateddata], ax
  1823                                  linkdatarelocation extdata_used
  1824                                  @@:
  1825 00000761 C3                      	retn
  1826                                  
  1827                                  
  1828                                  DATAOFFSET equ CODEOFFSET + code_size
  1829                                  	addsection DATA, follows=CODE vstart=_ELD_DATA_VSTART
  1830                                  %define DATAFIXUP - datastart + 0
  1831                                  datastart:
  1832                                  PUT_ELD_DATETIME
  1833                                  
  1834                                  %if _BOOT
  1835                                  reloc matchfunction:	dw sort_or_display
  1836                                  internalcoderelocation
  1837                                  reloc widecurrent:	dw relocateddata
  1838                                  linkdatarelocation line_out
  1839                                  %endif
  1840 00000000 0000                    meta:			dw 0
  1841 00000002 [A701]                  reloc compare:		dw ..@compare_normal
  1842                                  internalcoderelocation
  1843 00000004 00                      found:			db 0
  1844                                  %ifn _BOOT
  1845 00000005 00                      findhandle_set:		db 0
  1846 00000006 00                      prefersfn:		db 0
  1847                                  %endif
  1848 00000007 00                      wide:			db 0
  1849 00000008 00                      widecounter:		db 0
  1850 00000009 00                      sort:			db 0
  1851                                  %ifn _BOOT
  1852 0000000A 00                      sortlfn:		db 0
  1853                                  %endif
  1854 0000000B 00                      dirfirst:		db 0
  1855 0000000C 00                      date:			db 0
  1856 0000000D 00                      size:			db 0
  1857                                  
  1858                                  msg:
  1859                                  %ifn _BOOT
  1860 0000000E 53464E00                .string_sfn:		asciz "SFN"
  1861                                  %endif
  1862 00000012 5749444500              .string_wide:		asciz "WIDE"
  1863 00000017 534F525400              .string_sort:		asciz "SORT"
  1864 0000001C 444952464952535400      .string_dirfirst:	asciz "DIRFIRST"
  1865 00000025 4441544500              .string_date:		asciz "DATE"
  1866 0000002A 53495A4500              .string_size:		asciz "SIZE"
  1867 0000002F 5245564552534500        .string_reverse:	asciz "REVERSE"
  1868                                  %ifn _BOOT
  1869 00000037 534F52544C464E00        .string_sortlfn:	asciz "SORTLFN"
  1870 0000003F 534F525453464E00        .string_sortsfn:	asciz "SORTSFN"
  1871                                  %endif
  1872                                  %if _DEBUG
  1873 00000047 534F52544445425547-     .string_sortdebug:	asciz "SORTDEBUG"
  1873 00000050 00                 
  1874 00000051 19454C442064617461-     .debug.1:			counted "ELD data block buffer at "
  1874 0000005A 20626C6F636B206275-
  1874 00000063 6666657220617420   
  1875 0000006B 072C2073697A6520        .debug.2:			counted ", size "
  1876 00000073 0A2062797465732C20-     .debug.bytes:			counted " bytes, >="
  1876 0000007C 3E3D               
  1877 0000007E 222053464E20656E74-     .debug.3:			counted " SFN entries",13,10,"Auxiliary buffer at "
  1877 00000087 726965730D0A417578-
  1877 00000090 696C69617279206275-
  1877 00000099 6666657220617420   
  1878                                  %if _BOOT
  1879                                  .debug.5 equ .debug.2
  1880                                  %else
  1881 000000A1 0C3A303030302C2073-     .debug.5:			counted ":0000, size "
  1881 000000AA 697A6520           
  1882                                  %endif
  1883 000000AE 182053464E20656E74-     .debug.6.available:		counted " SFN entries (available)"
  1883 000000B7 726965732028617661-
  1883 000000C0 696C61626C6529     
  1884 000000C7 152053464E20656E74-     .debug.6.inuse:			counted " SFN entries (in use)"
  1884 000000D0 726965732028696E20-
  1884 000000D9 75736529           
  1885 000000DD 4461746120626C6F63-     .debug.larger_data_block:	asciz "Data block chosen because it is larger (above-or-equal size).",13,10
  1885 000000E6 6B2063686F73656E20-
  1885 000000EF 626563617573652069-
  1885 000000F8 74206973206C617267-
  1885 00000101 6572202861626F7665-
  1885 0000010A 2D6F722D657175616C-
  1885 00000113 2073697A65292E0D0A-
  1885 0000011C 00                 
  1886 0000011D 417578696C69617279-     .debug.smaller_data_block:	asciz "Auxiliary buffer chosen because it is larger and available.",13,10
  1886 00000126 206275666665722063-
  1886 0000012F 686F73656E20626563-
  1886 00000138 617573652069742069-
  1886 00000141 73206C617267657220-
  1886 0000014A 616E6420617661696C-
  1886 00000153 61626C652E0D0A00   
  1887                                   %ifn _BOOT
  1888 0000015B 536D616C6C65722064-     .debug.smaller_data_block_forced:asciz "Smaller data block chosen because auxiliary buffer not available.",13,10
  1888 00000164 61746120626C6F636B-
  1888 0000016D 2063686F73656E2062-
  1888 00000176 656361757365206175-
  1888 0000017F 78696C696172792062-
  1888 00000188 7566666572206E6F74-
  1888 00000191 20617661696C61626C-
  1888 0000019A 652E0D0A00         
  1889                                   %endif
  1890                                  %endif
  1891 0000019F 546F6F206C6F6E6720-     .error:			asciz "Too long short name, internal error!",13,10
  1891 000001A8 73686F7274206E616D-
  1891 000001B1 652C20696E7465726E-
  1891 000001BA 616C206572726F7221-
  1891 000001C3 0D0A00             
  1892 000001C6 46696C65206E6F7420-     .error2:		asciz "File not found, internal error!",13,10
  1892 000001CF 666F756E642C20696E-
  1892 000001D8 7465726E616C206572-
  1892 000001E1 726F72210D0A00     
  1893 000001E8 46696C656E616D6573-     .toofull:		asciz "Filenames list does not fit in buffer!",13,10
  1893 000001F1 206C69737420646F65-
  1893 000001FA 73206E6F7420666974-
  1893 00000203 20696E206275666665-
  1893 0000020C 72210D0A00         
  1894 00000211 082020205B4449525D      .dirinsteadsize:	countedb "   [DIR]"
  1895 0000021A 083E32353620546942      .sizetoolarge:		countedb ">256 TiB"
  1896 00000223 46696C65206E6F7420-     .notfound:		db "File not found."
  1896 0000022C 666F756E642E       
  1897 00000232 0D0A00                  .linebreak:		asciz 13,10
  1898 00000235 52756E207769746820-     .help:		db "Run with a pathname as parameter.",13,10
  1898 0000023E 6120706174686E616D-
  1898 00000247 652061732070617261-
  1898 00000250 6D657465722E0D0A   
  1899 00000258 4C61737420636F6D70-     		db "Last component may include wildcards.",13,10
  1899 00000261 6F6E656E74206D6179-
  1899 0000026A 20696E636C75646520-
  1899 00000273 77696C646361726473-
  1899 0000027C 2E0D0A             
  1900 0000027F 0D0A                    		db 13,10
  1901 00000281 416674657220746865-     		db "After the pathname, keywords may follow:",13,10
  1901 0000028A 20706174686E616D65-
  1901 00000293 2C206B6579776F7264-
  1901 0000029C 73206D617920666F6C-
  1901 000002A5 6C6F773A0D0A       
  1902                                  %ifn _BOOT
  1903 000002AB 0953464E0955736520-     		db 9,"SFN",9,"Use DOS SFN search even if LFN available",13,10
  1903 000002B4 444F532053464E2073-
  1903 000002BD 656172636820657665-
  1903 000002C6 6E206966204C464E20-
  1903 000002CF 617661696C61626C65-
  1903 000002D8 0D0A               
  1904 000002DA 095749444509446973-     		db 9,"WIDE",9,"Display in wide mode, up to 5 SFNs per line",13,10
  1904 000002E3 706C617920696E2077-
  1904 000002EC 696465206D6F64652C-
  1904 000002F5 20757020746F203520-
  1904 000002FE 53464E732070657220-
  1904 00000307 6C696E650D0A       
  1905 0000030D 09534F525409536F72-     		db 9,"SORT",9,"Sort filenames, default is SFNs. Must fit in buffer!",13,10
  1905 00000316 742066696C656E616D-
  1905 0000031F 65732C206465666175-
  1905 00000328 6C742069732053464E-
  1905 00000331 732E204D7573742066-
  1905 0000033A 697420696E20627566-
  1905 00000343 666572210D0A       
  1906 00000349 09534F525453464E09-     		db 9,"SORTSFN",9,"Same as SORT, but explicitly sort SFNs",13,10
  1906 00000352 53616D652061732053-
  1906 0000035B 4F52542C2062757420-
  1906 00000364 6578706C696369746C-
  1906 0000036D 7920736F7274205346-
  1906 00000376 4E730D0A           
  1907 0000037A 09534F52544C464E09-     		db 9,"SORTLFN",9,"Sort filenames using their LFNs",13,10
  1907 00000383 536F72742066696C65-
  1907 0000038C 6E616D657320757369-
  1907 00000395 6E6720746865697220-
  1907 0000039E 4C464E730D0A       
  1908                                  %else
  1909                                  		db 9,"WIDE",9,"Display in wide mode, up to 5 SFNs per line",13,10
  1910                                  		db 9,"SORT",9,"Sort filenames. Must fit in buffer!",13,10
  1911                                  %endif
  1912 000003A4 094441544509576865-     		db 9,"DATE",9,"When sorting, sort by date first",13,10
  1912 000003AD 6E20736F7274696E67-
  1912 000003B6 2C20736F7274206279-
  1912 000003BF 206461746520666972-
  1912 000003C8 73740D0A           
  1913 000003CC 0953495A4509576865-     		db 9,"SIZE",9,"When sorting, sort by size first",13,10
  1913 000003D5 6E20736F7274696E67-
  1913 000003DE 2C20736F7274206279-
  1913 000003E7 2073697A6520666972-
  1913 000003F0 73740D0A           
  1914 000003F4 095245564552534509-     		db 9,"REVERSE",9,"When sorting, reverse name/DATE/SIZE sort order",13,10
  1914 000003FD 5768656E20736F7274-
  1914 00000406 696E672C2072657665-
  1914 0000040F 727365206E616D652F-
  1914 00000418 444154452F53495A45-
  1914 00000421 20736F7274206F7264-
  1914 0000042A 65720D0A           
  1915 0000042E 094449524649525354-     		db 9,"DIRFIRST",9,"When sorting, sort directories first",13,10
  1915 00000437 095768656E20736F72-
  1915 00000440 74696E672C20736F72-
  1915 00000449 74206469726563746F-
  1915 00000452 726965732066697273-
  1915 0000045B 740D0A             
  1916 0000045E 00                      		asciz
  1917                                  
  1918                                  uinit_data: equ $
  1919                                  
  1920 0000045F 00                      	align 16, db 0
  1921                                  data_size equ $ - datastart
  1922                                  
  1923                                  	absolute uinit_data
  1924                                  
  1925 0000045F ??                      	alignb 2
  1926                                  %if _BOOT
  1927                                  wild_pattern:	resw 1
  1928                                  %else
  1929 00000460 ????????                originaldta:	resd 1
  1930 00000464 ????                    originalinject:	resw 1
  1931                                  %endif
  1932                                  
  1933 00000466 ????                    sortsegsel:	resw 1
  1934 00000468 ????                    sortstartoffset:resw 1
  1935 0000046A ????                    sortendoffset:	resw 1
  1936 0000046C ????                    sort_last:	resw 1
  1937 0000046E ????                    sort_next:	resw 1
  1938                                  
  1939 00000470 ????                    pathname_start:	resw 1
  1940 00000472 ????                    pathname_length:resw 1
  1941                                  %ifn _BOOT
  1942                                  findnext_function_number:
  1943 00000474 ????                    		resw 1
  1944 00000476 ????                    findhandle:	resw 1
  1945                                  %endif
  1946                                  
  1947                                  buffer:
  1948                                  %ifn _BOOT
  1949 00000478 <res 15h>               dta:		resb 15h
  1950 0000048D ??                      .attrib:	resb 1
  1951 0000048E ????                    .time:		resw 1
  1952 00000490 ????                    .date:		resw 1
  1953 00000492 ????????                .size:		resd 1
  1954 00000496 <res Dh>                .name:		resb 13
  1955                                  %endif
  1956                                  
  1957 000004A3 ??                      	alignb 2
  1958                                  finddata:
  1959 000004A4 ????????                .attrib:	resd 1
  1960 000004A8 <res 10h>               		resq 2
  1961 000004B8 ????                    .time:		resw 1
  1962 000004BA ????                    .date:		resw 1
  1963 000004BC ????????                		resd 1
  1964 000004C0 ????????                .sizehigh:	resd 1
  1965 000004C4 ????????                .sizelow:	resd 1
  1966 000004C8 ????????????????        		resb 8
  1967                                  pathnamebuffer equ $
  1968 000004D0 <res 104h>              .fullname:	resb 260
  1969 000005D4 <res Eh>                .shortname:	resb 14
  1970 000005E2 ??????????              size40bit:	resb 5
  1971                                  
  1972 000005E7 <res 9h>                	alignb 16
  1973                                  uinit_data_end_1:
  1974                                  
  1975                                  	absolute buffer
  1976 00000478 <res 200h>              		resb 512
  1977                                  buffer_end:
  1978                                  
  1979 00000678 ????????????????        	alignb 16
  1980                                  uinit_data_end_2:
  1981                                  
  1982                                  %if uinit_data_end_2 > uinit_data_end_1
  1983                                   uinit_data_end equ uinit_data_end_2
  1984                                  %else
  1985                                   uinit_data_end equ uinit_data_end_1
  1986                                  %endif
  1987                                  
  1988                                  
  1989                                  total_data_size equ uinit_data_end - datastart
  1990                                  %assign _DATA_SIZE total_data_size
  1991                                  
  1992                                  	usesection CODE
  1993                                  
  1994                                  %include "eldlink.asm"
     1                              <1> %if 0
     2                              <1> 
     3                              <1> Extensions for lDebug linker
     4                              <1> 
     5                              <1> Copyright (C) 2008-2025 E. C. Masloch
     6                              <1> 
     7                              <1> Usage of the works is permitted provided that this
     8                              <1> instrument is retained with the works, so that any entity
     9                              <1> that uses the works is notified of this instrument.
    10                              <1> 
    11                              <1> DISCLAIMER: THE WORKS ARE WITHOUT WARRANTY.
    12                              <1> 
    13                              <1> %endif
    14                              <1> 
    15                              <1> %include "lmacros3.mac"
     1                              <2> [list -]
    16                              <1> %include "eld.mac"
     1                              <2> %if 0
     2                              <2> 
     3                              <2> Extensions for lDebug macros
     4                              <2> 
     5                              <2> Copyright (C) 2008-2025 E. C. Masloch
     6                              <2> 
     7                              <2> Usage of the works is permitted provided that this
     8                              <2> instrument is retained with the works, so that any entity
     9                              <2> that uses the works is notified of this instrument.
    10                              <2> 
    11                              <2> DISCLAIMER: THE WORKS ARE WITHOUT WARRANTY.
    12                              <2> 
    13                              <2> %endif
    14                              <2> 
    15                              <2> %ifndef ELD_MAC
    16                              <2> %define ELD_MAC 1
    17                              <2> 
    18                              <2> %include "lmacros3.mac"
    19                              <2> 
    20                              <2> 		; ELD executable header
    21                              <2> 	struc ELD_HEADER
    22                              <2> eldhSignature:		resb 4	; "ELD1"
    23                              <2> 			resb 3	; reserved
    24                              <2> 			resb 1	; 26 (Ctrl-Z)
    25                              <2> eldhCodeOffset:		resd 1	; position displacement from eldhSignature
    26                              <2> eldhCodeImageLength:	resw 1	; amount bytes, at least 32
    27                              <2> eldhCodeAllocLength:	resw 1	; amount bytes, added to prior. sum < 64 KiB
    28                              <2> eldhDataOffset:		resd 1
    29                              <2> eldhDataImageLength:	resw 1	; (zero allowed)
    30                              <2> eldhDataAllocLength:	resw 1	; (zero allowed)
    31                              <2> eldhCodeEntrypoint:	resw 1	; within code section, used as displacement
    32                              <2> eldhReserved:		resb 4	; reserved
    33                              <2> eldhExtensionSize:	resw 1	; from eldhSignature, -> past eldhx fields in use
    34                              <2> 	endstruc
    35                              <2> 	endarea ELD_HEADER, 1
    36                              <2> 
    37                              <2> 	struc ELD_HEADERX
    38                              <2> eldhxHeader:		resb ELD_HEADER_size
    39                              <2> eldhxDescriptionOffset:	resd 1	; zero if none, from eldhxHeader. <= 128 Bytes
    40                              <2> eldhxHelpOffset:	resd 1	; zero if none, from eldhxHeader
    41                              <2> eldhxLibTable:		resd 1	; zero if none, from eldhxHeader
    42                              <2> eldhxDateTimeOffset:	resd 1	; zero if none, from eldhxHeader
    43                              <2> 	alignb 16
    44                              <2> 	endstruc
    45                              <2> 
    46                              <2> 	struc ELD_TRAILER_HEADER
    47                              <2> eldthSignature:		resb 8	; "ELD1TAIL"
    48                              <2> eldthHeaderOffset:	resd 1	; negative displacement from eldthSignature,
    49                              <2> 				;  add this dword to the seek offset
    50                              <2> eldthReserved:		resw 1	; reserved, must be initialised to zero
    51                              <2> eldthChecksum:		resw 1	; sum of all words in trailer header = 0
    52                              <2> 	endstruc
    53                              <2> 	endarea ELD_TRAILER_HEADER, 1
    54                              <2> 
    55                              <2> 	struc ELD_LIBTABLE
    56                              <2> eldltFormat:		resw 1
    57                              <2> 	; 0 = uncompressed
    58                              <2> 	; 2 = heatshrink compressed
    59                              <2> 	; 3 = lzexedat -4 compressed
    60                              <2> 	; 4 = lzexedat -4 -l compressed
    61                              <2> eldltAmount:		resw 1
    62                              <2> eldltOffset:		resd 1	; from eldhxHeader
    63                              <2> eldltCompressedLength:		; (dword, only present if format 2, 3, or 4)
    64                              <2> 	endstruc
    65                              <2> 	endarea ELD_LIBTABLE, 1
    66                              <2> 
    67                              <2> 		; ELD instance header
    68                              <2> 	struc ELD_INSTANCE
    69                              <2> eldiStartCode:		resw 1	; -> this structure itself (para aligned)
    70                              <2> eldiEndCode:		resw 1	; -> behind memory used by instance (para aligned)
    71                              <2> eldiStartData:		resw 1	; -> data in data entry section (para aligned), or 0
    72                              <2> eldiEndData:		resw 1	; -> behind data (para aligned), or 0
    73                              <2> eldiIdentifier:		resb 8	; blank-filled text
    74                              <2> eldiFlags:		resw 1	; flags
    75                              <2> eldiListing_size equ 14
    76                              <2> eldiListing:		resb eldiListing_size
    77                              <2> 				; ASCIZ listing file name
    78                              <2> 	endstruc
    79                              <2> 		; flags for eldiFlags:
    80                              <2> eldifResident:		equ 1
    81                              <2> 
    82                              <2> 		; ELD link info header
    83                              <2> 	struc ELD_LINKINFO
    84                              <2> eldlSignature:		resw 1	; 0E1D1h
    85                              <2> eldlReserved:		resw 2
    86                              <2> eldlUseLinkHash:	resw 1
    87                              <2> eldlDataAmount:		resw 1
    88                              <2> eldlDataPrefixes:	resw 1
    89                              <2> eldlDataEntries:	resw 1
    90                              <2> eldlDataAddresses:	resw 1
    91                              <2> eldlCodeAmount:		resw 1
    92                              <2> eldlCodePrefixes:	resw 1
    93                              <2> eldlCodeEntries:	resw 1
    94                              <2> eldlCodeAddresses:	resw 1
    95                              <2> 	endstruc
    96                              <2> 
    97                              <2> 	numdef ELD_CODE_VSTART, 9001h
    98                              <2> 	numdef ELD_DATA_VSTART, 8000h
    99                              <2> 	numdef ELD_RELOC_VSTART, 8000h
   100                              <2> 
   101                              <2> 	numdef ELD_RECLAIM_HINT, 0
   102                              <2> 	strdef ELD_LISTING, ""
   103                              <2> 	numdef ELD_DATETIME, 0
   104                              <2> 
   105                              <2> %if _ELD_DATETIME
   106                              <2>  %define PUT_ELDHX_DATETIME_OFFSET at eldhxDateTimeOffset, dd DATAOFFSET + datetime - datastart
   107                              <2>  %macro PUT_ELD_DATETIME 0.nolist
   108                              <2> datetime:	asciz __UTC_DATE__,'T',__UTC_TIME__,'Z'
   109                              <2> 		asciz		; for future extension
   110                              <2>  %endmacro
   111                              <2> %else
   112                              <2>  %define PUT_ELDHX_DATETIME_OFFSET
   113                              <2>  %define PUT_ELD_DATETIME
   114                              <2> %endif
   115                              <2> 
   116                              <2> %endif
    17                              <1> 
    18                              <1> 	cpu 8086
    19                              <1> 
    20                              <1> %if ELDSTRICT
    21                              <1>  %if ELDSTRICTCOUNTER
    22                              <1>   %error Missing relocation
    23                              <1>  %endif
    24                              <1> %endif
    25                              <1> 	eldstrict off		; linker does some relocations
    26                              <1> 
    27                              <1> %ifn ELDCALLCALL_DUMPED
    28 00000762 90<rep 6h>E8[0000]- <1> 	eldcall_dump_callcall ELDCALL_CALLCALL_LIST
    28 0000076B EB020000C3E8[0000]- <1>
    28 00000773 EB020000C3E8[0000]- <1>
    28 0000077B EB020000C3E8[0000]- <1>
    28 00000783 EB020000C3E8[0000]- <1>
    28 0000078B EB020000C3E8[0000]- <1>
    28 00000793 EB020000C3E8[0000]- <1>
    28 0000079B EB020000C3E8[0000]- <1>
    28 000007A3 EB020000C3E8[0000]- <1>
    28 000007AB EB020000C3E8[0000]- <1>
    28 000007B3 EB020000C3E8[0000]- <1>
    28 000007BB EB020000C3E8[0000]- <1>
    28 000007C3 EB020000C3E8[0000]- <1>
    28 000007CB EB020000C3E8[0000]- <1>
    28 000007D3 EB020000C3E8[0000]- <1>
    28 000007DB EB020000C3E8[0000]- <1>
    28 000007E3 EB020000C3E8[0000]- <1>
    28 000007EB EB020000C3E8[0000]- <1>
    28 000007F3 EB020000C3E8[0000]- <1>
    28 000007FB EB020000C3E8[0000]- <1>
    28 00000803 EB020000C3E8[0000]- <1>
    28 0000080B EB020000C3E8[0000]- <1>
    28 00000813 EB020000C3E8[0000]- <1>
    28 0000081B EB020000C3          <1>
    29                              <1> %endif
    30                              <1> 
    31                              <1> 	numdef ELD_IDENTICALISE, 0
    32                              <1> 	numdef ELD_DEBUG, 0
    33                              <1> 	numdef ELD_LINKER_PASSES, 1
    34                              <1> 	strdef LISTING, _ELD_LISTING
    35                              <1> 	numdef ELDCALL_OPTIONAL, ELDCALL_OPTIONAL_STATUS
    36                              <1> 	numdef ELDDATA_OPTIONAL, ELDDATA_OPTIONAL_STATUS
    37                              <1> 	numdef ELDDATA_NEXT, ELDDATA_NEXT_STATUS
    38                              <1> 	numdef ELDCALL_NEXT, ELDCALL_NEXT_STATUS
    39                              <1> %if _ELD_IDENTICALISE
    40                              <1>  ;%assign _ELDCALL_OPTIONAL 1
    41                              <1> %endif
    42                              <1> %ifn _ELDCALL_OPTIONAL
    43                              <1> %assign ELDCALL_OPTIONAL_STATUS 2		; not allowed
    44                              <1> %endif
    45                              <1> ;%ifn _ELDDATA_OPTIONAL
    46                              <1> ;%assign ELDDATA_OPTIONAL_STATUS 2		; not allowed
    47                              <1> ;%endif
    48                              <1> 	gendef MAP, ""
    49                              <1> 
    50                              <1> %ifnidni _MAP, ""
    51                              <1>  [map all _MAP]
    52                              <1> %endif
    53                              <1> 
    54                              <1> 
    55                              <1> endresident: equ ($ + _CURRENT_SECTION %+ FIXUP + 15) & ~15
    56                              <1> 
    57                              <1> %if _ELD_LINKER_PASSES
    58                              <1> %assign ELDLINKER 1
    59                              <1> 
    60                              <1> 	struc LINKTABLE
    61 00000000 ????????            <1> ltCodeToCode:	resw 2
    62 00000004 ????????            <1> ltCodeToData:	resw 2
    63 00000008 ????????            <1> ltDataToCode:	resw 2
    64 0000000C ????????            <1> ltDataToData:	resw 2
    65 00000010 ????????            <1> ltLinkData:	resw 2
    66 00000014 ????????            <1> ltLinkCode:	resw 2
    67                              <1> 	endstruc
    68                              <1> %endif
    69                              <1> 
    70                              <1> 
    71                              <1> 		; INP:	es:dx -> loaded initial ELD image
    72                              <1> 		;	 ELD instance structure filled
    73                              <1> 		;	es => ELD code area
    74                              <1> 		;	ds:di -> link info
    75                              <1> 		;	ss:bx -> loaded initial data
    76                              <1> 		;	ss:si -> command line tail
    77                              <1> 		;	cs:ip -> entrypoint
    78                              <1> 		;	ss:sp -> far return address for current mode
    79                              <1> 		; STT:	UP, EI
    80                              <1> linker:
    81                              <1> 		; The first 15 Bytes of the linker should be
    82                              <1> 		;  the same regardless of the linker options
    83                              <1> 		;  used (debug, passes, vstart). This allows
    84                              <1> 		;  the eldcomp ELD to match even if up to 15
    85                              <1> 		;  Bytes of the linker are trailing in the
    86                              <1> 		;  resident part of the ELD.
    87                              <1> 	lframe
    88                              <1>  %if ELDOTHER
    89                              <1> 	lvar dword, linkinfo_other
    90                              <1> 	lvar word, use_hash_other
    91                              <1>  %endif
    92 00000820 5589E5              <1> 	lenter
    93                              <1> 	lvar dword, instance
    94 00000823 06                  <1> 	 push es
    95 00000824 52                  <1> 	 push dx		; -> start of where we're loaded in ELD cs
    96                              <1> 	lvar word, targetsection_low_optional_high
    97 00000825 50                  <1> 	 push ax		; placeholder
    98                              <1> 	lequ ?targetsection_low_optional_high, targetsection
    99                              <1> 	lequ ?targetsection_low_optional_high + 1, optional
   100                              <1> 	lvar dword, linkinfo
   101 00000826 1E                  <1> 	 push ds
   102 00000827 57                  <1> 	 push di		; -> link info (in debugger ss or message seg)
   103                              <1> 	lvar dword, nextreloc
   104 00000828 06                  <1> 	 push es		; => ELD cs
   105 00000829 52                  <1> 	 push dx		; placeholder
   106                              <1> 	lvar dword, entry
   107 0000082A 06                  <1> 	 push es		; => ELD cs
   108 0000082B 50                  <1> 	 push ax		; placeholder
   109 0000082C 31C0                <1> 	xor ax, ax
   110 0000082E 813DD1E1            <1> 	cmp word [di + eldlSignature], 0E1D1h
   111                              <1> %if ($ - linker) < 16
   112                              <1>  %error Expected invariant first paragraph of linker
   113                              <1> %endif
   114 00000832 7403                <1> 	je @F
   115                              <1> .error_j1:
   116 00000834 E92C03              <1> 	jmp .error		; signature mismatch -->
   117                              <1> @@:
   118 00000837 837D0601            <1> 	cmp word [di + eldlUseLinkHash], 1
   119 0000083B 77F7                <1> 	ja .error_j1		; unknown use link hash number -->
   120 0000083D 7201                <1> 	jb @F
   121                              <1> %if _ELDDATA_NEXT || _ELDCALL_NEXT
   122                              <1> 	dec al			; = -1 if hash used
   123                              <1> %else
   124 0000083F 48                  <1> 	dec ax
   125                              <1> %endif
   126                              <1> @@:
   127                              <1> 	lvar word, use_hash_low_skip_last_high
   128 00000840 50                  <1> 	 push ax		; = -1 if hash used, else 0
   129                              <1> 	lequ ?use_hash_low_skip_last_high, use_hash
   130                              <1> 	lequ ?use_hash_low_skip_last_high + 1, skip_last
   131                              <1> %if _ELD_IDENTICALISE && _ELD_LINKER_PASSES
   132                              <1> 	mov ax, linktable - code
   133                              <1> 	lvar word, lt
   134                              <1> 	 push ax		; -> link tables (a single reference)
   135                              <1> %endif
   136                              <1> %if _ELD_LINKER_PASSES || ELDOTHER || _ELDDATA_OPTIONAL || _ELDCALL_OPTIONAL
   137 00000841 31C0                <1> 	xor ax, ax
   138                              <1>  %if _ELD_LINKER_PASSES
   139                              <1> 	lvar word, pass
   140 00000843 50                  <1> 	 push ax		; = 0 for linker itself, = 2 for application
   141                              <1> 	lvar word, amounterrors
   142 00000844 50                  <1> 	 push ax		; how many distinct errors encountered in pass 2
   143                              <1>  %endif
   144                              <1>  %if _ELD_LINKER_PASSES || _ELDDATA_OPTIONAL || _ELDCALL_OPTIONAL
   145                              <1> 	lvar word, name
   146 00000845 50                  <1> 	 push ax		; -> name currently being sought (in our table)
   147                              <1>  %endif
   148                              <1>  %if ELDOTHER
   149                              <1> 	lvar word, other
   150                              <1> 	 push ax		; byte: 0 = own data links, -1 = other data links
   151                              <1>  %endif
   152                              <1>  %if _ELDDATA_OPTIONAL || _ELDCALL_OPTIONAL
   153                              <1> 	lvar word, optionalmissing
   154 00000846 50                  <1> 	 push ax
   155                              <1>  %endif
   156                              <1> %endif
   157 00000847 56                  <1> 	push si			; -> command line tail
   158 00000848 53                  <1> 	push bx			; -> data block in ELD data area (segment ss)
   159                              <1> 
   160                              <1> 			; simple: add instance base (dx) to code
   161 00000849 06                  <1> 	push es
   162 0000084A 1F                  <1> 	pop ds			; ds = es => ELD cs
   163                              <1> %if _ELD_LINKER_PASSES
   164                              <1> .pass:
   165 0000084B 8B5EEA              <1> 	mov bx, word [bp + ?pass]	; 0 or 2
   166 0000084E 01D3                <1> 	add bx, dx		; -> start of the ELD instance in cs, +0 or +2
   167                              <1>  %if _ELD_IDENTICALISE
   168                              <1> 	add bx, word [bp + ?lt]	; add in single reference to linktable
   169                              <1> 	mov si, word [ltCodeToCode + bx]
   170                              <1>  %else
   171 00000850 8BB7760C            <1> 	mov si, word [linktable - code + ltCodeToCode + bx]
   172                              <1>  %endif
   173                              <1> %else
   174                              <1> 	mov si, internalcodetocoderelocations - code
   175                              <1> %endif		 		; si -> table for code to code (linker or app)
   176 00000854 01D6                <1> 	add si, dx		; relocate the table pointer itself
   177                              <1> @@:
   178 00000856 AD                  <1> 	lodsw
   179 00000857 85C0                <1> 	test ax, ax		; was last ?
   180 00000859 740B                <1> 	jz @F			; yes -->
   181 0000085B 93                  <1> 	xchg bx, ax		; bx = entry
   182 0000085C 01D3                <1> 	add bx, dx		; relocate the entry itself
   183                              <1> %if _ELD_CODE_VSTART
   184 0000085E 812F[0000]          <1> 	sub word [bx], code	; undo adjustment
   185                              <1> %endif
   186 00000862 0117                <1> 	add word [bx], dx	; relocate word referenced by entry
   187 00000864 EBF0                <1> 	jmp @B
   188                              <1> 
   189                              <1> @@:
   190                              <1> 			; next, add heap data base (on stack) to code
   191                              <1> %if _ELD_LINKER_PASSES
   192 00000866 8B5EEA              <1> 	mov bx, word [bp + ?pass]	; 0 or 2
   193 00000869 01D3                <1> 	add bx, dx		; -> start of the ELD instance in cs, +0 or +2
   194                              <1>  %if _ELD_IDENTICALISE
   195                              <1> 	add bx, word [bp + ?lt]	; add in single reference to linktable
   196                              <1> 	mov si, word [ltCodeToData + bx]
   197                              <1>  %else
   198 0000086B 8BB77A0C            <1> 	mov si, word [linktable - code + ltCodeToData + bx]
   199                              <1>  %endif
   200                              <1> %else
   201                              <1> 	mov si, internalcodetodatarelocations - code
   202                              <1> %endif				; si -> table for code to data (linker or app)
   203 0000086F 01D6                <1> 	add si, dx		; relocate the table pointer itself
   204                              <1> @@:
   205 00000871 AD                  <1> 	lodsw
   206 00000872 85C0                <1> 	test ax, ax		; was last ?
   207 00000874 740C                <1> 	jz @F			; yes -->
   208 00000876 93                  <1> 	xchg bx, ax		; bx = entry
   209 00000877 01D3                <1> 	add bx, dx		; relocate the entry itself
   210                              <1> 		; ! access the offset of the data area block, topmost on stack
   211 00000879 58                  <1> 	pop ax			; ax -> heap data
   212 0000087A 50                  <1> 	push ax
   213                              <1> %if _ELD_DATA_VSTART
   214 0000087B 2D[0000]            <1> 	sub ax, datastart	; undo adjustment
   215                              <1> %endif
   216 0000087E 0107                <1> 	add word [bx], ax	; relocate word referenced by entry
   217 00000880 EBEF                <1> 	jmp @B
   218                              <1> 
   219                              <1> @@:
   220                              <1> 
   221                              <1> 			; add instance base (dx) to data
   222                              <1> %if _ELD_LINKER_PASSES
   223 00000882 8B5EEA              <1> 	mov bx, word [bp + ?pass]
   224 00000885 01D3                <1> 	add bx, dx
   225                              <1>  %if _ELD_IDENTICALISE
   226                              <1> 	add bx, word [bp + ?lt]
   227                              <1> 	mov si, word [ltDataToCode + bx]
   228                              <1>  %else
   229 00000887 8BB77E0C            <1> 	mov si, word [linktable - code + ltDataToCode + bx]
   230                              <1>  %endif
   231                              <1> %else
   232                              <1> 	mov si, internaldatatocoderelocations - code
   233                              <1> %endif
   234 0000088B 01D6                <1> 	add si, dx
   235                              <1> @@:
   236 0000088D AD                  <1> 	lodsw
   237 0000088E 83F8FF              <1> 	cmp ax, -1		; was last ?
   238 00000891 740F                <1> 	je @F			; yes -->
   239 00000893 93                  <1> 	xchg bx, ax		; bx = entry
   240                              <1> 		; ! access the offset of the data area block, topmost on stack
   241 00000894 58                  <1> 	pop ax
   242 00000895 50                  <1> 	push ax
   243 00000896 01C3                <1> 	add bx, ax		; relocate the entry itself
   244                              <1> %if _ELD_CODE_VSTART
   245 00000898 36812F[0000]        <1> 	sub word [ss:bx], code	; undo adjustment
   246                              <1> %endif
   247 0000089D 360117              <1> 	add word [ss:bx], dx	; relocate word referenced by entry
   248 000008A0 EBEB                <1> 	jmp @B
   249                              <1> 
   250                              <1> @@:
   251                              <1> 			; next, add heap data base (on stack) to data
   252                              <1> %if _ELD_LINKER_PASSES
   253 000008A2 8B5EEA              <1> 	mov bx, word [bp + ?pass]
   254 000008A5 01D3                <1> 	add bx, dx
   255                              <1>  %if _ELD_IDENTICALISE
   256                              <1> 	add bx, word [bp + ?lt]
   257                              <1> 	mov si, word [ltDataToData + bx]
   258                              <1>  %else
   259 000008A7 8BB7820C            <1> 	mov si, word [linktable - code + ltDataToData + bx]
   260                              <1>  %endif
   261                              <1> %else
   262                              <1> 	mov si, internaldatatodatarelocations - code
   263                              <1> %endif
   264 000008AB 01D6                <1> 	add si, dx
   265                              <1> @@:
   266 000008AD AD                  <1> 	lodsw
   267 000008AE 83F8FF              <1> 	cmp ax, -1		; was last ?
   268 000008B1 740D                <1> 	je @F			; yes -->
   269 000008B3 93                  <1> 	xchg bx, ax		; bx = entry
   270                              <1> 		; ! access the offset of the data area block, topmost on stack
   271 000008B4 58                  <1> 	pop ax			; ax -> heap data
   272 000008B5 50                  <1> 	push ax
   273 000008B6 01C3                <1> 	add bx, ax		; relocate the entry itself
   274                              <1> %if _ELD_DATA_VSTART
   275 000008B8 2D[0000]            <1> 	sub ax, datastart	; undo adjustment
   276                              <1> %endif
   277 000008BB 360107              <1> 	add word [ss:bx], ax	; relocate word referenced by entry
   278 000008BE EBED                <1> 	jmp @B
   279                              <1> 
   280                              <1> @@:
   281 000008C0 8B56FC              <1> 	mov dx, word [bp + ?instance]
   282                              <1> 				; reset (why??) -> ELD instance in ELD cs
   283                              <1> %if _ELD_LINKER_PASSES
   284 000008C3 8B5EEA              <1> 	mov bx, word [bp + ?pass]
   285 000008C6 01D3                <1> 	add bx, dx
   286                              <1>  %if _ELD_IDENTICALISE
   287                              <1> 	add bx, word [bp + ?lt]
   288                              <1> 	add dx, word [ltLinkData + bx]
   289                              <1>  %else
   290 000008C8 0397860C            <1> 	add dx, word [linktable - code + ltLinkData + bx]
   291                              <1>  %endif
   292                              <1> %else
   293                              <1> 	add dx, linkerdatarelocations - code
   294                              <1> %endif
   295                              <1> .otherloop:
   296 000008CC 8956F2              <1> 	mov word [bp + ?nextreloc], dx
   297                              <1> 				; -> data link relocation table
   298                              <1> 
   299                              <1> .datarelocloop:		; must be done before further relocs
   300 000008CF C576F2              <1> 	lds si, [bp + ?nextreloc]
   301 000008D2 AD                  <1> 	lodsw			; ax = section indicator
   302 000008D3 85C0                <1> 	test ax, ax		; end of table ?
   303 000008D5 7503E96601          <1> 	jz .donedatareloc
   304 000008DA 48                  <1> 	dec ax			; al = 1 if data, 0 if code (NB ah may != 0)
   305                              <1> 		; ! access the offset of the data area block, topmost on stack
   306 000008DB 5B                  <1> 	pop bx
   307 000008DC 53                  <1> 	push bx			; bx -> ELD data block
   308 000008DD 8946FA              <1> 	mov word [bp + ?targetsection_low_optional_high], ax
   309 000008E0 84C0                <1> 	test al, al		; data ?
   310 000008E2 AD                  <1> 	lodsw
   311 000008E3 7504                <1> 	jnz @F			; yes -->
   312 000008E5 0346FC              <1> 	add ax, word [bp + ?instance]
   313                              <1> 				; relocate entry into code
   314 000008E8 A9                  <1> 	db __TEST_IMM16		; (skip add)
   315                              <1> @@:
   316 000008E9 01D8                <1> 	add ax, bx		; relocate entry into data
   317 000008EB 8946EE              <1> 	mov word [bp + ?entry], ax
   318                              <1> 				; save away -> where to patch
   319 000008EE AD                  <1> 	lodsw			; get unrelocated -> name
   320 000008EF 8976F2              <1> 	mov word [bp + ?nextreloc], si
   321                              <1> 				; update -> behind relocation table entry
   322                              <1> %if _ELDDATA_NEXT
   323                              <1> 	rol byte [bp + ?skip_last], 1	; skipping ?
   324                              <1> 	jnc @F				; no -->
   325                              <1> 	test byte [bp + ?optional], 8	; is it a last relocation ?
   326                              <1> 	jz .datarelocloop		; no, leave skip_last set -->
   327                              <1> 	not byte [bp + ?skip_last]	; disable skip_last
   328                              <1> 	jmp .datarelocloop
   329                              <1> @@:
   330                              <1> %endif
   331 000008F2 E81001              <1> 	call .build_match	; get ax = scan value, si -> counted string,
   332                              <1> 				;  dl = original value at byte [si]
   333                              <1> 				; NC if symbol already not found before
   334                              <1> 				; CY if to search for the symbol
   335                              <1> %if _ELD_LINKER_PASSES
   336 000008F5 73D8                <1> 	jnc .datarelocloop	; if duplicate of a not found symbol -->
   337                              <1> %endif
   338 000008F7 C45EF6              <1> 	les bx, [bp + ?linkinfo]
   339                              <1> %if ELDOTHER
   340                              <1> 	rol byte [bp + ?other], 1
   341                              <1> 	jnc @F
   342                              <1> 	les bx, [bp + ?linkinfo_other]
   343                              <1> @@:
   344                              <1> %endif				; es:bx -> link info table of the ELD host
   345 000008FA 268B4F08            <1> 	mov cx, word [es:bx + eldlDataAmount]	; amount data link info
   346 000008FE 268B7F0A            <1> 	mov di, word [es:bx + eldlDataPrefixes]	; -> prefixes or hashes
   347                              <1> .datarelocfind:
   348 00000902 83F901              <1> 	cmp cx, 1			; NZ if cx == 0
   349 00000905 F2AF                <1> 	repne scasw			; scan initial
   350                              <1> %if _ELDDATA_OPTIONAL
   351                              <1> 	jne .datanotfound_may_be_optional
   352                              <1> %else
   353 00000907 7403E98900          <1> 	jne .datanotfound
   354                              <1> %endif
   355 0000090C 57                  <1> 	push di
   356 0000090D 51                  <1> 	push cx
   357 0000090E 56                  <1> 	push si
   358 0000090F 262B7F0A            <1> 	sub di, word [es:bx + eldlDataPrefixes]	; = double index, 1-based
   359 00000913 4F                  <1> 	dec di
   360 00000914 4F                  <1> 	dec di				; 0-based
   361 00000915 26037F0C            <1> 	add di, word [es:bx + eldlDataEntries]	; -> entry
   362 00000919 268B3D              <1> 	mov di, [es:di]			; -> counted suffix/string
   363 0000091C B500                <1> 	mov ch, 0
   364 0000091E 8A0C                <1> 	mov cl, byte [si]		; cx = length
   365 00000920 41                  <1> 	inc cx
   366                              <1> 	; cmp al, al			; ZR if length is zero
   367 00000921 F3A6                <1> 	repe cmpsb			; match ?
   368 00000923 5E                  <1> 	pop si
   369 00000924 59                  <1> 	pop cx
   370 00000925 5F                  <1> 	pop di
   371 00000926 75DA                <1> 	jne .datarelocfind		; if not found this time,
   372                              <1> 					;  scan for next initial -->
   373 00000928 8814                <1> 	mov byte [si], dl		; restore the original byte at counter
   374 0000092A 262B7F0A            <1> 	sub di, word [es:bx + eldlDataPrefixes]	; = double index, 1-based
   375 0000092E 4F                  <1> 	dec di
   376 0000092F 4F                  <1> 	dec di				; 0-based
   377 00000930 26037F0E            <1> 	add di, word [es:bx + eldlDataAddresses]	; -> address (offset)
   378 00000934 268B05              <1> 	mov ax, word [es:di]		; get link data from the table
   379 00000937 E80700              <1> 	call .address_data_reloc
   380                              <1> %if _ELD_RELOC_VSTART
   381 0000093A 2D[0000]            <1> 	sub ax, relocateddata		; *not* a relocation
   382                              <1> %endif
   383 0000093D 0104                <1> 	add word [si], ax		; relocate
   384                              <1> %if _ELDDATA_NEXT
   385                              <1> 	test byte [bp + ?optional], 4	; is it a next relocation ?
   386                              <1> 	jz .datarelocloop
   387                              <1> 	mov byte [bp + ?skip_last], -1	; skip subsequent next/last relocs
   388                              <1> %endif
   389 0000093F EB8E                <1> 	jmp .datarelocloop
   390                              <1> 
   391                              <1> .address_data_reloc:
   392 00000941 C576EE              <1> 	lds si, [bp + ?entry]		; -> entry if in ELD code instance
   393 00000944 807EFA00            <1> 	cmp byte [bp + ?targetsection], 0
   394                              <1> 					; relocation in code ?
   395 00000948 7402                <1> 	je @F				; yes -->
   396 0000094A 16                  <1> 	push ss
   397 0000094B 1F                  <1> 	pop ds				; => our ELD data block
   398                              <1> @@:
   399 0000094C C3                  <1> 	retn
   400                              <1> 
   401                              <1> %if _ELDDATA_OPTIONAL
   402                              <1> .datanotfound_may_be_optional:
   403                              <1> 	mov byte [si], dl		; restore the original byte at counter
   404                              <1> %if _ELDDATA_NEXT
   405                              <1> 	test byte [bp + ?optional], 3	; is it an optional relocation ?
   406                              <1> %else
   407                              <1> 	cmp byte [bp + ?optional], 0	; is it an optional relocation ?
   408                              <1> %endif
   409                              <1> %if _ELD_DEBUG
   410                              <1> 	jnz @F
   411                              <1>  %ifn _ELD_LINKER_PASSES
   412                              <1> 	mov si, 0			; (invalid link)
   413                              <1> linkdatarelocation internalflags6
   414                              <1> 	test si, si
   415                              <1> 	jz .datanotfound
   416                              <1> 	mov si, 0			; (invalid link)
   417                              <1> linkdatarelocation options7
   418                              <1> 	test si, si
   419                              <1> 	jz .datanotfound
   420                              <1>  %else
   421                              <1> 	cmp byte [bp + ?pass], 0
   422                              <1> 	je .datanotfound
   423                              <1>  %endif
   424                              <1> 	houdini				; (the above conditions are for this)
   425                              <1> 	jmp .datanotfound
   426                              <1> @@:
   427                              <1> %else
   428                              <1> 	jz .datanotfound		; no, handle as an error -->
   429                              <1> %endif
   430                              <1> 
   431                              <1> %if ELDDATA_PMREQUIRED_STATUS
   432                              <1> 	mov si, relocateddata
   433                              <1> linkdatarelocation build_option_PM
   434                              <1> 	test si, si			; is it a PM build ?
   435                              <1> 	jz @F				; no --> (treat PM required as optional)
   436                              <1> 	test byte [bp + ?optional], 2	; optional status is PM required ?
   437                              <1> 	jnz .datanotfound		; yes, handle as an error -->
   438                              <1> @@:
   439                              <1> %endif
   440                              <1> 
   441                              <1> %if _ELD_LINKER_PASSES
   442                              <1> %if _ELDDATA_OPTIONAL || _ELDCALL_OPTIONAL
   443                              <1> 	rol byte [bp + ?optionalmissing], 1
   444                              <1> 	jnc .optionaldatamissingmsg
   445                              <1> 	mov si, [bp + ?name]
   446                              <1> 	or byte [si], 80h
   447                              <1> 	not byte [bp + ?optionalmissing]
   448                              <1> 	jmp @F
   449                              <1> .optionaldatamissingmsg:
   450                              <1> %endif
   451                              <1> 	testopt [ss:relocateddata], 2	; debug optional link ?
   452                              <1> linkdatarelocation options7, -3
   453                              <1> 	jz @F				; no -->
   454                              <1> %if _ELDDATA_OPTIONAL || _ELDCALL_OPTIONAL
   455                              <1> 	mov byte [bp + ?optionalmissing + 1], -1
   456                              <1> %endif
   457                              <1> 	mov si, lmsg.warning_data_optional
   458                              <1> internalcoderelocation
   459                              <1> 	call .notfound			; display a warning
   460                              <1> %if _ELDDATA_OPTIONAL || _ELDCALL_OPTIONAL
   461                              <1> 	not byte [bp + ?optionalmissing + 1]
   462                              <1> %endif
   463                              <1> @@:
   464                              <1> %endif
   465                              <1> %if _ELDDATA_NEXT
   466                              <1> 	test byte [bp + ?optional], 4	; is it a next relocation ?
   467                              <1> 	jnz .datarelocloop
   468                              <1> %endif
   469                              <1> 	call .address_data_reloc
   470                              <1> 	and word [si], 0		; indicate optional data link failed
   471                              <1> 	jmp .datarelocloop
   472                              <1> %endif
   473                              <1> 
   474                              <1> 
   475                              <1> %if _ELDCALL_OPTIONAL
   476                              <1> .codenotfound_may_be_optional:
   477 0000094D 8814                <1> 	mov byte [si], dl		; restore the original byte at counter
   478                              <1> %if _ELDCALL_NEXT
   479                              <1> 	test byte [bp + ?optional], 3	; is it an optional relocation ?
   480                              <1> %else
   481 0000094F 807EFB00            <1> 	cmp byte [bp + ?optional], 0	; is it an optional relocation ?
   482                              <1> %endif
   483                              <1> %if _ELD_DEBUG
   484                              <1> 	jnz @F
   485                              <1>  %ifn _ELD_LINKER_PASSES
   486                              <1> 	mov si, 0			; (invalid link)
   487                              <1> linkdatarelocation internalflags6
   488                              <1> 	test si, si
   489                              <1> 	jz .codenotfound
   490                              <1> 	mov si, 0			; (invalid link)
   491                              <1> linkdatarelocation options7
   492                              <1> 	test si, si
   493                              <1> 	jz .codenotfound
   494                              <1>  %else
   495                              <1> 	cmp byte [bp + ?pass], 0
   496                              <1> 	je .codenotfound
   497                              <1>  %endif
   498                              <1> 	houdini				; (the above conditions are for this)
   499                              <1> 	jmp .codenotfound
   500                              <1> @@:
   501                              <1> %else
   502 00000953 7451                <1> 	jz .codenotfound		; no, handle as an error -->
   503                              <1> %endif
   504                              <1> 
   505                              <1> %if ELDCALL_PMREQUIRED_STATUS
   506                              <1>  %if _ELD_LINKER_PASSES
   507                              <1>   %assign ELDLINKER 0
   508                              <1>  %endif
   509 00000955 BE[0000]            <1> 	mov si, relocateddata
   510                              <1> linkdatarelocation build_option_PM
   511                              <1>  %if _ELD_LINKER_PASSES
   512                              <1>   %assign ELDLINKER 1
   513                              <1>  %endif
   514 00000958 85F6                <1> 	test si, si			; is it a PM build ?
   515 0000095A 7406                <1> 	jz @F				; no --> (treat PM required as optional)
   516 0000095C F646FB02            <1> 	test byte [bp + ?optional], 2	; optional status is PM required ?
   517 00000960 7544                <1> 	jnz .codenotfound		; yes, handle as an error -->
   518                              <1> @@:
   519                              <1> %endif
   520                              <1> 
   521                              <1> %if _ELD_LINKER_PASSES
   522                              <1> %if _ELDDATA_OPTIONAL || _ELDCALL_OPTIONAL
   523 00000962 D046E4              <1> 	rol byte [bp + ?optionalmissing], 1
   524 00000965 730B                <1> 	jnc .optionalcodemissingmsg
   525 00000967 8B76E6              <1> 	mov si, [bp + ?name]
   526 0000096A 800C80              <1> 	or byte [si], 80h
   527 0000096D F656E4              <1> 	not byte [bp + ?optionalmissing]
   528 00000970 EB15                <1> 	jmp @F
   529                              <1> .optionalcodemissingmsg:
   530                              <1> %endif
   531 00000972 36F606[0000]02      <1> 	testopt [ss:relocateddata], 2	; debug optional link ?
   532                              <1> linkdatarelocation options7, -3
   533 00000978 740D                <1> 	jz @F				; no -->
   534                              <1> %if _ELDDATA_OPTIONAL || _ELDCALL_OPTIONAL
   535 0000097A C646E5FF            <1> 	mov byte [bp + ?optionalmissing + 1], -1
   536                              <1> %endif
   537 0000097E BE[AE11]            <1> 	mov si, lmsg.warning_code_optional
   538                              <1> internalcoderelocation
   539 00000981 E83000              <1> 	call .notfound			; display a warning
   540                              <1> %if _ELDDATA_OPTIONAL || _ELDCALL_OPTIONAL
   541 00000984 F656E5              <1> 	not byte [bp + ?optionalmissing + 1]
   542                              <1> %endif
   543                              <1> @@:
   544                              <1> %endif
   545                              <1> %if _ELDCALL_NEXT
   546                              <1> 	test byte [bp + ?optional], 4	; is it a next relocation ?
   547                              <1> 	jnz .coderelocloop
   548                              <1> %endif
   549 00000987 C576EE              <1> 	lds si, [bp + ?entry]		; -> code site (must be in ELD cs)
   550 0000098A C7049090            <1> 	mov word [si], 9090h
   551 0000098E C6440290            <1> 	mov byte [si + 2], 90h		; indicate optional code link failed
   552                              <1> 					;  (NOP out the 3-byte call near imm)
   553 00000992 E9BA00              <1> 	jmp .coderelocloop
   554                              <1> %endif
   555                              <1> 
   556                              <1> 
   557                              <1> %if _ELD_LINKER_PASSES
   558                              <1> .datanotfound:
   559 00000995 BE[D011]            <1> 	mov si, lmsg.error_data
   560                              <1> internalcoderelocation
   561 00000998 E81900              <1> 	call .notfound			; display error
   562 0000099B 7306                <1> 	jnc .error_j3			; NC if in pass 0, error out now -->
   563 0000099D FF46E8              <1> 	inc word [bp + ?amounterrors]	; count the amount of errors
   564 000009A0 E92CFF              <1> 	jmp .datarelocloop		; go to next relocation entry -->
   565                              <1> 
   566                              <1> .error_j3:
   567 000009A3 E9BD01              <1> 	jmp .error
   568                              <1> 
   569                              <1> .codenotfound:
   570 000009A6 BE[E911]            <1> 	mov si, lmsg.error_code
   571                              <1> internalcoderelocation
   572 000009A9 E80800              <1> 	call .notfound			; display error
   573 000009AC 73F5                <1> 	jnc .error_j3			; NC if in pass 0 -->
   574 000009AE FF46E8              <1> 	inc word [bp + ?amounterrors]	; count the amount of errors
   575 000009B1 E99B00              <1> 	jmp .coderelocloop		; go to next -->
   576                              <1> 
   577                              <1> .notfound:
   578 000009B4 807EEA00            <1> 	cmp byte [bp + ?pass], 0	; pass 0 ?
   579 000009B8 7442                <1> 	je .notfound.retn		; yes, do not try displaying --> (NC)
   580 000009BA 16                  <1> 	 push ss
   581 000009BB 07                  <1> 	 pop es
   582 000009BC BF[0000]            <1> 	mov di, relocateddata
   583                              <1> linkdatarelocation line_out		; es:di -> line_out buffer
   584 000009BF E83B00              <1> 	call .copy			; copy prefix message
   585 000009C2 8B76E6              <1> 	mov si, word [bp + ?name]
   586 000009C5 AD                  <1> 	lodsw				; = hash
   587 000009C6 E8[0000]EB020000    <1> 	extcall hexword			; display the hash in hex
   588 000009CD 56                  <1> 	push si
   589 000009CE BE[0212]            <1> 	mov si, lmsg.error.2
   590                              <1> internalcoderelocation
   591 000009D1 E82900              <1> 	call .copy			; display message fragment
   592 000009D4 5E                  <1> 	pop si
   593                              <1> %if _ELD_LINKER_PASSES
   594 000009D5 56                  <1> 	push si
   595 000009D6 E82400              <1> 	call .copy			; copy over the full name
   596 000009D9 5E                  <1> 	pop si
   597                              <1>  %if _ELDDATA_OPTIONAL || _ELDCALL_OPTIONAL
   598 000009DA 800C80              <1> 	or byte [si], 80h		; mark as failed optional link
   599 000009DD D046E5              <1> 	rol byte [bp + ?optionalmissing + 1], 1
   600                              <1> 					; was it optional ?
   601 000009E0 7203                <1> 	jc @F				; yes -->
   602                              <1>  %endif
   603 000009E2 C60400              <1> 	mov byte [si], 0		; mark as failed (counter byte = 0)
   604                              <1> @@:
   605                              <1> %else
   606                              <1> 	call .copy
   607                              <1> %endif
   608 000009E5 B022                <1> 	mov al, '"'
   609 000009E7 AA                  <1> 	stosb				; end message with a closing quote mark
   610 000009E8 16                  <1> 	 push ss
   611 000009E9 1F                  <1> 	 pop ds
   612 000009EA E8[0000]EB020000    <1> 	extcall putsline_crlf		; display diagnostic line
   613 000009F1 B8350E              <1> 	mov ax, 0E35h
   614 000009F4 E8[0000]EB020000    <1> 	extcall setrc
   615 000009FB F9                  <1> 	stc				; CY, diagnostic displayed
   616                              <1> .notfound.retn:
   617 000009FC C3                  <1> 	retn
   618                              <1> 
   619                              <1> .copy:		; (cannot use extcallcall here)
   620 000009FD E8[0000]EB020000    <1> 	extcall copy_single_counted_string
   621 00000A04 C3                  <1> 	retn
   622                              <1> %else
   623                              <1> .datanotfound: equ .error
   624                              <1> .codenotfound: equ .error
   625                              <1> %endif
   626                              <1> 
   627                              <1> .build_match:
   628                              <1> %if _ELDDATA_OPTIONAL || _ELDCALL_OPTIONAL
   629 00000A05 C646E400            <1> 	mov byte [bp + ?optionalmissing], 0
   630                              <1> 		; This is needed for eldtestj.asm with debugoptlink.
   631                              <1> 		;  The optional data link sets flag 80h, then the
   632                              <1> 		;  required data link to the same symbol sets this
   633                              <1> 		;  flag but doesn't reset it. So the first optional
   634                              <1> 		;  code link still had this set. Reset here to fix.
   635                              <1> %endif
   636                              <1> %if _ELD_CODE_VSTART
   637 00000A09 2D[0000]            <1> 	sub ax, code			; revert adjustment (= displacement)
   638                              <1> %endif
   639 00000A0C 0346FC              <1> 	add ax, word [bp + ?instance]	; make displacement into -> name string
   640 00000A0F 96                  <1> 	xchg si, ax			; si -> hash word, counted name string
   641                              <1> %if _ELD_LINKER_PASSES || _ELDDATA_OPTIONAL || _ELDCALL_OPTIONAL
   642 00000A10 8976E6              <1> 	mov word [bp + ?name], si	; save away for diagnostics
   643                              <1> %endif
   644 00000A13 AD                  <1> 	lodsw			; = hash, si -> counted string
   645 00000A14 8A14                <1> 	mov dl, byte [si]	; dl = original start byte of match
   646                              <1> %if _ELD_LINKER_PASSES
   647 00000A16 84D2                <1> 	test dl, dl		; marked as already failed ?
   648                              <1> 				;  (80h = optional, 0 = required)
   649 00000A18 750A                <1> 	jnz @F			; no -->
   650 00000A1A 837EE800            <1> 	cmp word [bp + ?amounterrors], 0
   651                              <1> 				; validate error status
   652 00000A1E 7503E9B300          <1> 	je .error_j		; no error known ?! cancel quickly -->
   653 00000A23 C3                  <1> 	retn			; (NC)
   654                              <1> 
   655                              <1> @@:
   656                              <1> %else
   657                              <1> 	test dl, dl
   658                              <1> %endif
   659                              <1> %if _ELDDATA_OPTIONAL || _ELDCALL_OPTIONAL
   660 00000A24 7909                <1> 	jns @F
   661 00000A26 80E27F              <1> 	and dl, 7Fh
   662 00000A29 8814                <1> 	mov byte [si], dl
   663 00000A2B C646E4FF            <1> 	mov byte [bp + ?optionalmissing], -1
   664                              <1> @@:
   665                              <1> %endif
   666                              <1> %if ELDOTHER
   667                              <1> 	rol byte [bp + ?other], 1
   668                              <1> 	jnc @F
   669                              <1> 	rol byte [bp + ?use_hash_other], 1
   670                              <1> 	jmp @FF
   671                              <1> 
   672                              <1> @@:
   673                              <1> %endif
   674 00000A2F D046EC              <1> 	rol byte [bp + ?use_hash], 1
   675                              <1> @@:
   676                              <1> 		; If to use the hash, then ax = hash and si ->
   677                              <1> 		;  the entire symbol name as a counted string.
   678 00000A32 720A                <1> 	jc @F			; if to use hash, return now -->
   679 00000A34 AC                  <1> 	lodsb			; al = length
   680 00000A35 91                  <1> 	xchg cx, ax		; cl = length
   681 00000A36 AD                  <1> 	lodsw			; ax = prefix
   682 00000A37 49                  <1> 	dec cx
   683 00000A38 49                  <1> 	dec cx			; cl = adjusted length
   684 00000A39 4E                  <1> 	dec si			; -> second byte of prefix
   685 00000A3A 8A14                <1> 	mov dl, byte [si]	; dl = original start byte of match
   686 00000A3C 880C                <1> 	mov byte [si], cl	; si -> counted string suffix
   687                              <1> 		; (this name entry has been edited to provide the
   688                              <1> 		;  name suffix as a counted string, as required by
   689                              <1> 		;  the old-style non-hash link info tables.
   690                              <1> 		; it will be reset later by writing dl to si -> the
   691                              <1> 		;  first byte of the match string.)
   692                              <1> @@:
   693                              <1> %if _ELD_LINKER_PASSES
   694 00000A3E F9                  <1> 	stc			; CY
   695                              <1> %endif
   696 00000A3F C3                  <1> 	retn
   697                              <1> 
   698                              <1> 
   699                              <1> .donedatareloc:
   700                              <1> %if ELDOTHER
   701                              <1> 	rol byte [bp + ?other], 1
   702                              <1> 	jc .otherdone		; other link only has data links,
   703                              <1> 				;  so at this point we're done -->
   704                              <1> %endif
   705                              <1> 
   706 00000A40 8B56FC              <1> 	mov dx, word [bp + ?instance]
   707                              <1> %if _ELD_LINKER_PASSES
   708 00000A43 8B5EEA              <1> 	mov bx, word [bp + ?pass]
   709 00000A46 01D3                <1> 	add bx, dx
   710                              <1>  %if _ELD_IDENTICALISE
   711                              <1> 	add bx, word [bp + ?lt]
   712                              <1> 	add dx, word [ltLinkCode + bx]
   713                              <1>  %else
   714 00000A48 03978A0C            <1> 	add dx, word [linktable - code + ltLinkCode + bx]
   715                              <1>  %endif
   716                              <1> %else
   717                              <1> 	add dx, linkercoderelocations - code
   718                              <1> %endif
   719 00000A4C 8956F2              <1> 	mov word [bp + ?nextreloc], dx
   720                              <1> 
   721                              <1> .coderelocloop:
   722 00000A4F C576F2              <1> 	lds si, [bp + ?nextreloc]
   723 00000A52 AD                  <1> 	lodsw
   724                              <1> %if _ELDCALL_OPTIONAL || _ELDCALL_NEXT
   725 00000A53 48                  <1> 	dec ax				; optional word is 1-based, get 0-based
   726 00000A54 7903E98F00          <1> 	js .donecodereloc
   727 00000A59 8946FA              <1> 	mov word [bp + ?targetsection_low_optional_high], ax
   728 00000A5C AD                  <1> 	lodsw
   729                              <1> %endif
   730 00000A5D 0346FC              <1> 	add ax, word [bp + ?instance]
   731 00000A60 8946EE              <1> 	mov word [bp + ?entry], ax
   732 00000A63 AD                  <1> 	lodsw
   733 00000A64 8976F2              <1> 	mov word [bp + ?nextreloc], si
   734                              <1> %ifn _ELDCALL_OPTIONAL || _ELDCALL_NEXT
   735                              <1> 	test ax, ax			; if no optional word, check -> match
   736                              <1> 	jz .donecodereloc
   737                              <1> %endif
   738                              <1> %if _ELDCALL_NEXT
   739                              <1> 	rol byte [bp + ?skip_last], 1	; skipping ?
   740                              <1> 	jnc @F				; no -->
   741                              <1> 	test byte [bp + ?optional], 8	; is it a last relocation ?
   742                              <1> 	jz .coderelocloop		; no, leave skip_last set -->
   743                              <1> 	not byte [bp + ?skip_last]	; disable skip_last
   744                              <1> 	jmp .coderelocloop
   745                              <1> @@:
   746                              <1> %endif
   747 00000A67 E89BFF              <1> 	call .build_match
   748                              <1> %if _ELD_LINKER_PASSES
   749 00000A6A 73E3                <1> 	jnc .coderelocloop
   750                              <1> %endif
   751 00000A6C C45EF6              <1> 	les bx, [bp + ?linkinfo]
   752 00000A6F 268B4F10            <1> 	mov cx, word [es:bx + eldlCodeAmount]	; amount code link info
   753 00000A73 268B7F12            <1> 	mov di, word [es:bx + eldlCodePrefixes]	; -> prefixes or hashes
   754                              <1> .coderelocfind:
   755 00000A77 83F901              <1> 	cmp cx, 1			; NZ if cx == 0
   756 00000A7A F2AF                <1> 	repne scasw			; scan initial
   757                              <1> %if _ELDCALL_OPTIONAL
   758 00000A7C 7403E9CCFE          <1> 	jne .codenotfound_may_be_optional
   759                              <1> %else
   760                              <1>  %if _ELD_DEBUG
   761                              <1> 	je @F
   762                              <1> 	houdini
   763                              <1> 	jmp .codenotfound
   764                              <1> @@:
   765                              <1>  %else
   766                              <1> 	jne .codenotfound
   767                              <1>  %endif
   768                              <1> %endif
   769 00000A81 57                  <1> 	push di
   770 00000A82 51                  <1> 	push cx
   771 00000A83 56                  <1> 	push si
   772 00000A84 262B7F12            <1> 	sub di, word [es:bx + eldlCodePrefixes]	; = double index, 1-based
   773 00000A88 4F                  <1> 	dec di
   774 00000A89 4F                  <1> 	dec di				; 0-based
   775 00000A8A 26037F14            <1> 	add di, word [es:bx + eldlCodeEntries]	; -> entry
   776 00000A8E 268B3D              <1> 	mov di, [es:di]			; -> counted suffix/string
   777 00000A91 B500                <1> 	mov ch, 0
   778 00000A93 8A0C                <1> 	mov cl, byte [si]		; cx = length
   779 00000A95 41                  <1> 	inc cx
   780                              <1> 	; cmp al, al			; ZR if length is zero
   781 00000A96 F3A6                <1> 	repe cmpsb			; match ?
   782 00000A98 5E                  <1> 	pop si
   783 00000A99 59                  <1> 	pop cx
   784 00000A9A 5F                  <1> 	pop di
   785 00000A9B 75DA                <1> 	jne .coderelocfind
   786 00000A9D 8814                <1> 	mov byte [si], dl
   787 00000A9F 262B7F12            <1> 	sub di, word [es:bx + eldlCodePrefixes]	; = double index, 1-based
   788 00000AA3 4F                  <1> 	dec di
   789 00000AA4 4F                  <1> 	dec di				; 0-based
   790 00000AA5 01FF                <1> 	add di, di			; quadruple index
   791 00000AA7 26037F16            <1> 	add di, word [es:bx + eldlCodeAddresses]	; -> address (offset, segment)
   792 00000AAB 26FF35              <1> 	push word [es:di]
   793 00000AAE C576EE              <1> 	lds si, [bp + ?entry]
   794 00000AB1 8F4405              <1> 	pop word [si + 3 + 2]		; call near imm (3), jmp short (2)
   795                              <1> 					;  patch the destination address
   796 00000AB4 803CE8              <1> 	cmp byte [si], 0E8h		; is it as expected ?
   797 00000AB7 751D                <1> 	jne .error_j
   798 00000AB9 268B7D02            <1> 	mov di, word [es:di + 2]
   799 00000ABD BB[0000]            <1> 	mov bx, relocateddata
   800                              <1> linkdatarelocation linkcall_table	; ss:bx -> link call table
   801 00000AC0 36833F01            <1> 	cmp word [ss:bx], 1		; is it initialised to format 1 ?
   802 00000AC4 7510                <1> 	jne .error_j			; no -->
   803 00000AC6 368B4F02            <1> 	mov cx, word [ss:bx + 2]	; get amount of segments
   804 00000ACA E30A                <1> 	jcxz .error_j			; none -->
   805                              <1> @@:
   806 00000ACC 83C304              <1> 	add bx, 4			; -> next segment
   807 00000ACF 36393F              <1> 	cmp word [ss:bx], di		; value matches ?
   808 00000AD2 7405                <1> 	je @F				; yes, found -->
   809 00000AD4 E2F6                <1> 	loop @B				; try remaining segments
   810                              <1> .error_j:
   811 00000AD6 E98A00              <1> 	jmp .error
   812                              <1> 
   813                              <1> @@:
   814 00000AD9 368B5F02            <1> 	mov bx, word [ss:bx + 2]	; -> call destination offset
   815                              <1> 		; si + 3 + delta = bx
   816                              <1> 		; delta = bx - si - 3
   817 00000ADD 29F3                <1> 	sub bx, si
   818 00000ADF 83EB03              <1> 	sub bx, 3
   819 00000AE2 895C01              <1> 	mov word [si + 1], bx		; patch the call instruction
   820                              <1> %if _ELDCALL_NEXT
   821                              <1> 	test byte [bp + ?optional], 4	; is it a next relocation ?
   822                              <1> 	jz .coderelocloop
   823                              <1> 	mov byte [bp + ?skip_last], -1	; skip subsequent next/last relocs
   824                              <1> %endif
   825 00000AE5 E967FF              <1> 	jmp .coderelocloop
   826                              <1> 
   827                              <1> .donecodereloc:
   828                              <1> %if _ELD_LINKER_PASSES
   829 00000AE8 8B46E8              <1> 	mov ax, word [bp + ?amounterrors]
   830 00000AEB 85C0                <1> 	test ax, ax
   831 00000AED 75E7                <1> 	jnz .error_j
   832 00000AEF 8B5EEA              <1> 	mov bx, word [bp + ?pass]
   833 00000AF2 85DB                <1> 	test bx, bx
   834 00000AF4 750B                <1> 	jnz @F
   835 00000AF6 43                  <1> 	inc bx
   836 00000AF7 43                  <1> 	inc bx
   837 00000AF8 895EEA              <1> 	mov word [bp + ?pass], bx
   838 00000AFB 8B56FC              <1> 	mov dx, word [bp + ?instance]
   839 00000AFE E94AFD              <1> 	jmp .pass
   840                              <1> 
   841                              <1> @@:
   842                              <1> %endif
   843                              <1> 
   844                              <1> %ifnidni _LISTING, ""
   845                              <1> %assign ELDLINKER 0
   846                              <1> .hint:
   847 00000B01 16                  <1> 	push ss
   848 00000B02 1F                  <1> 	pop ds
   849 00000B03 B02D                <1> 	mov al, 2Dh
   850 00000B05 E8[0000]EB020000    <1> 	extcall intchk			; ZR if offset = -1 or segment = 0
   851                              <1> 					; CHG: ax, dx, bx
   852 00000B0C 7437                <1> 	jz .no_hint
   853                              <1> 
   854                              <1> %if ELDOTHER
   855                              <1> 	mov si, debuggeramissig	; ds:si -> our AMIS name strings
   856                              <1> internalcoderelocation
   857                              <1> %endif
   858                              <1> 
   859 00000B0E 8A26[0000]          <1> 	mov ah, byte [relocateddata]
   860                              <1> linkdatarelocation try_debugger_amis_multiplex_number
   861 00000B12 E85500              <1> 	call plex_check
   862 00000B15 7305                <1> 	jnc @F
   863                              <1> 
   864 00000B17 B4FF                <1> 	mov ah, 0FFh		; start with multiplex number 0FFh
   865                              <1> .loop_hint:
   866 00000B19 E84E00              <1> 	call plex_check
   867                              <1> @@:
   868 00000B1C 7307                <1> 	jnc .end_hint		; if found --> (NC)
   869 00000B1E 80EC01              <1> 	sub ah, 1		; search is backward (to find latest installed first), from 0FFh to 00h including
   870 00000B21 73F6                <1> 	jnc .loop_hint		; try next if we didn't check all yet -->
   871 00000B23 EB20                <1> 	jmp .no_hint
   872                              <1> 
   873                              <1> .end_hint:
   874 00000B25 50                  <1> 	push ax
   875 00000B26 C446FC              <1> 	les ax, [bp + ?instance]
   876 00000B29 BF[100F]            <1> 	mov di, listmsg.hint.offset
   877                              <1> internalcoderelocation
   878 00000B2C E8[0000]EB020000    <1> 	extcall hexword
   879 00000B33 BB[F00E]            <1> 	mov bx, listmsg.hint
   880                              <1> internalcoderelocation
   881 00000B36 368B16[0000]        <1> 	mov dx, [ss:relocateddata]
   882                              <1> linkdatarelocation extseg	; must be 86 Mode segment even in PM
   883 00000B3B 58                  <1> 	pop ax
   884 00000B3C B040                <1> 	mov al, 40h		; AMIS message display service
   885 00000B3E E8[0000]EB020000    <1> 	extcall call_int2D
   886                              <1> .no_hint:
   887                              <1> %endif
   888                              <1> 
   889                              <1> %if ELDOTHER
   890                              <1> %assign ELDLINKER 0
   891                              <1> 	not byte [bp + ?other]
   892                              <1> 
   893                              <1> 	push ss
   894                              <1> 	pop ds
   895                              <1> 	mov al, 2Dh
   896                              <1> 	extcall intchk			; ZR if offset = -1 or segment = 0
   897                              <1> 					; CHG: ax, dx, bx
   898                              <1> 	jz .no_other
   899                              <1> 
   900                              <1> 	mov si, debuggeramissig	; ds:si -> our AMIS name strings
   901                              <1> internalcoderelocation
   902                              <1> 
   903                              <1> 	mov ah, byte [relocateddata]
   904                              <1> linkdatarelocation try_debugger_amis_multiplex_number
   905                              <1> 	call plex_check
   906                              <1> 	jnc @F
   907                              <1> 
   908                              <1> 	mov ah, 0FFh		; start with multiplex number 0FFh
   909                              <1> .loop_other_debug:
   910                              <1> 	call plex_check
   911                              <1> @@:
   912                              <1> 	jnc .end_other		; if found --> (NC)
   913                              <1> 	sub ah, 1		; search is backward (to find latest installed first), from 0FFh to 00h including
   914                              <1> 	jnc .loop_other_debug	; try next if we didn't check all yet -->
   915                              <1> 
   916                              <1> 	mov si, loaderamissig	; ds:si -> our AMIS name strings
   917                              <1> internalcoderelocation
   918                              <1> 
   919                              <1> 	mov ah, byte [relocateddata]
   920                              <1> linkdatarelocation try_debugger_amis_multiplex_number
   921                              <1> 	call plex_check
   922                              <1> 	jnc @F
   923                              <1> 
   924                              <1> 	mov ah, 0FFh		; start with multiplex number 0FFh
   925                              <1> .loop_other_loader:
   926                              <1> 	call plex_check
   927                              <1> @@:
   928                              <1> 	jnc .end_other		; if found --> (NC)
   929                              <1> 	sub ah, 1		; search is backward (to find latest installed first), from 0FFh to 00h including
   930                              <1> 	jnc .loop_other_loader	; try next if we didn't check all yet -->
   931                              <1> 
   932                              <1> 	jmp .no_other
   933                              <1> 
   934                              <1> .end_other:
   935                              <1> 	mov al, 42h		; AMIS get other link info service
   936                              <1> 	extcall call_int2D
   937                              <1> 	cmp al, 0FFh
   938                              <1> 	jne .no_other
   939                              <1> 
   940                              <1> 	mov ax, si		; selector => PSP
   941                              <1> 	extcall ispm
   942                              <1> 	jz @F
   943                              <1> 	mov ax, dx		; segment => PSP
   944                              <1> @@:
   945                              <1> 	 push ss
   946                              <1> 	 pop ds
   947                              <1> 	mov word [otherds], ax
   948                              <1> internaldatarelocation		; current mode sel/seg
   949                              <1> 	mov word [otherseg], dx
   950                              <1> internaldatarelocation		; remember segment
   951                              <1> 
   952                              <1> 	mov ax, cx		; selector => link info
   953                              <1> 	extcall ispm
   954                              <1> 	jz @F
   955                              <1> 	mov ax, bx		; segment => link info
   956                              <1> @@:
   957                              <1> 	mov word [bp + ?linkinfo_other], di
   958                              <1> 	mov word [bp + ?linkinfo_other + 2], ax
   959                              <1> 
   960                              <1> 	mov ds, ax		; => link info
   961                              <1> 	xor ax, ax
   962                              <1> 	cmp word [di + eldlSignature], 0E1D1h
   963                              <1> 	jne .error_other
   964                              <1> 	cmp word [di + eldlUseLinkHash], 1
   965                              <1> 	ja .error_other
   966                              <1> 	jb @F
   967                              <1> 	dec ax
   968                              <1> @@:
   969                              <1> 	mov word [bp + ?use_hash_other], ax
   970                              <1> 
   971                              <1> 	mov dx, word [bp + ?instance]
   972                              <1> 	add dx, linkerotherdatarelocations - code
   973                              <1> 	jmp .otherloop
   974                              <1> 
   975                              <1> .error_other:
   976                              <1> 	push cs
   977                              <1> 	pop ds
   978                              <1> 	mov ax, 0E33h
   979                              <1> 	extcall setrc
   980                              <1> 	mov dx, lmsg.error_other
   981                              <1> internalcoderelocation
   982                              <1> 	jmp @F
   983                              <1> 
   984                              <1> .no_other:
   985                              <1> 	push cs
   986                              <1> 	pop ds
   987                              <1> 	mov ax, 0E34h
   988                              <1> 	extcall setrc
   989                              <1> 	mov dx, lmsg.no_other
   990                              <1> internalcoderelocation
   991                              <1> @@:
   992                              <1> 	extcall putsz
   993                              <1> .error_j2:
   994                              <1> 	jmp .error
   995                              <1> 
   996                              <1> .otherdone:
   997                              <1>  %if _ELD_LINKER_PASSES
   998                              <1> 	mov ax, word [bp + ?amounterrors]
   999                              <1> 	test ax, ax
  1000                              <1> 	jnz .error_j2
  1001                              <1>  %endif
  1002                              <1> %endif
  1003                              <1> 
  1004 00000B45 5B                  <1> 	pop bx				; -> our heap data
  1005 00000B46 5E                  <1> 	pop si				; -> our command line tail
  1006 00000B47 16                  <1> 	 push ss
  1007 00000B48 1F                  <1> 	 pop ds
  1008 00000B49 C47EFC              <1> 	les di, [bp + ?instance]
  1009 00000B4C 268B4502            <1> 	mov ax, word [es:di + eldiEndCode]
  1010                              <1> houdini
  1011 00000B50 2D[2008]            <1> 	sub ax, strict word endresident + code
  1012                              <1> internalcoderelocation
  1013 00000B53 26C74502[2008]      <1> 	mov word [es:di + eldiEndCode], endresident + code
  1014                              <1> internalcoderelocation
  1015 00000B59 2906[0000]          <1> 	sub word [relocateddata], ax
  1016                              <1> linkdatarelocation extseg_used
  1017                              <1> %if _DATA_SIZE == 0
  1018                              <1> 	xor ax, ax
  1019                              <1> 	mov word [es:di + eldiStartData], ax
  1020                              <1> 	mov word [es:di + eldiEndData], ax
  1021                              <1> %endif
  1022 00000B5D 89EC5D              <1> 	lleave code
  1023                              <1> 		; INP:	es => ELD code segment
  1024                              <1> 		;	ds:si -> command line tail
  1025                              <1> 		;	ds:bx -> ELD data block
  1026                              <1> 		;	ss:sp -> far return address for current mode
  1027                              <1> 		; STT:	ds = ss, UP, EI
  1028 00000B60 E9BFFB              <1> 	jmp start
  1029                              <1> 
  1030                              <1> .error:
  1031 00000B63 89EC5D              <1> 	lleave
  1032 00000B66 B8FFFF              <1> 	mov ax, -1
  1033 00000B69 CB                  <1> 	retf
  1034                              <1> 
  1035                              <1> 
  1036                              <1> %ifnidni _LISTING, ""
  1037                              <1>  %assign ELDHINT 1
  1038                              <1> %else
  1039                              <1>  %assign ELDHINT 0
  1040                              <1> %endif
  1041                              <1> 
  1042                              <1> %if ELDOTHER || ELDHINT
  1043                              <1> 		; INP:	ah = multiplex number to check
  1044                              <1> 		;	(if ELDOTHER:)
  1045                              <1> 		;	 cs:si -> 16-byte AMIS signature to check
  1046                              <1> 		; OUT:	CY if multiplex number unused or no signature match,
  1047                              <1> 		;	 bp, ah, ds unmodified
  1048                              <1> 		;	NC if match found,
  1049                              <1> 		;	 ah = multiplex number (unmodified)
  1050                              <1> 		; CHG:	di, es, cx, dx
  1051                              <1> 		;	(if ELDOTHER:) bx
  1052                              <1> 		;	(if not ELDOTHER:) si
  1053                              <1> plex_check:
  1054 00000B6A 16                  <1> 	push ss
  1055 00000B6B 1F                  <1> 	pop ds
  1056 00000B6C F606[0000]08        <1> 	testopt [relocateddata], 8
  1057                              <1> linkdatarelocation internalflags4, -3
  1058 00000B71 740B                <1> 	jz @F
  1059                              <1> %if ELDOTHER
  1060                              <1> 	mov bx, relocateddata
  1061                              <1> linkdatarelocation amis_multiplex_number, -2, optional
  1062                              <1> 	test bx, bx
  1063                              <1> 	jz @F
  1064                              <1> 	cmp ah, byte [bx]
  1065                              <1> 	je .notfound		; do not use our own multiplexer -->
  1066                              <1> %else
  1067 00000B73 BE[0000]            <1> 	mov si, relocateddata
  1068                              <1> linkdatarelocation amis_multiplex_number, -2, optional
  1069 00000B76 85F6                <1> 	test si, si
  1070 00000B78 7404                <1> 	jz @F
  1071 00000B7A 3A24                <1> 	cmp ah, byte [si]
  1072 00000B7C 7420                <1> 	je .notfound		; do not use our own multiplexer -->
  1073                              <1> %endif
  1074                              <1> @@:
  1075 00000B7E B000                <1> 	mov al, 00h		; AMIS installation check
  1076 00000B80 E8[0000]EB020000    <1> 	extcall call_int2D	; AMIS (or "DOS reserved" = iret if no AMIS present)
  1077 00000B87 3CFF                <1> 	cmp al, 0FFh
  1078 00000B89 7513                <1> 	jne .notfound
  1079 00000B8B 0E                  <1> 	push cs
  1080 00000B8C 1F                  <1> 	pop ds
  1081                              <1> %if ELDOTHER
  1082                              <1> 	push si
  1083                              <1> 	extcall setes2dx	; es:di -> name strings of AMIS multiplexer that just answered
  1084                              <1> 	mov cx, 8		; Ignore description, only compare vendor and program name
  1085                              <1> 	repe cmpsw
  1086                              <1> 	pop si
  1087                              <1> %else
  1088 00000B8D BE[E00E]            <1> 	mov si, debuggeramissig	; ds:si -> our AMIS name strings
  1089                              <1> internalcoderelocation
  1090 00000B90 E8[0000]EB020000    <1> 	extcall setes2dx	; es:di -> name strings of AMIS multiplexer that just answered
  1091 00000B97 B90800              <1> 	mov cx, 8		; Ignore description, only compare vendor and program name
  1092 00000B9A F3A7                <1> 	repe cmpsw
  1093                              <1> %endif
  1094 00000B9C 7401                <1> 	je .checkret		; ZR, NC = match -->
  1095                              <1> .notfound:
  1096 00000B9E F9                  <1> 	stc			; CY no match
  1097                              <1> .checkret:
  1098 00000B9F C3                  <1> 	retn
  1099                              <1> %endif
  1100                              <1> 
  1101                              <1> 
  1102                              <1> 	align 4, db 0
  1103                              <1> linkercoderelocations:
  1104                              <1> %if _ELDCALL_OPTIONAL || _ELDCALL_NEXT
  1105 00000BA0 01033B00[180F]0103- <1> 	dw ELDCALL_CODE_RELOCATIONS_OPTIONAL, 0
  1105 00000BA8 CF06[180F]0100F806- <1>
  1105 00000BB0 [300F]01006807-     <1>
  1105 00000BB6 [420F]01007007-     <1>
  1105 00000BBC [4A0F]01007807-     <1>
  1105 00000BC2 [5E0F]01008007-     <1>
  1105 00000BC8 [650F]01008807-     <1>
  1105 00000BCE [700F]01009007-     <1>
  1105 00000BD4 [800F]01009807-     <1>
  1105 00000BDA [8C0F]0100A007-     <1>
  1105 00000BE0 [970F]0100A807-     <1>
  1105 00000BE6 [9E0F]0100B007-     <1>
  1105 00000BEC [A60F]0100B807-     <1>
  1105 00000BF2 [AE0F]0100C007-     <1>
  1105 00000BF8 [CB0F]0100C807-     <1>
  1105 00000BFE [F40F]0100D007-     <1>
  1105 00000C04 [0910]0100D807-     <1>
  1105 00000C0A [1410]0100E007-     <1>
  1105 00000C10 [2410]0100E807-     <1>
  1105 00000C16 [3010]0100F007-     <1>
  1105 00000C1C [3910]0100F807-     <1>
  1105 00000C22 [4510]01000008-     <1>
  1105 00000C28 [4D10]01000808-     <1>
  1105 00000C2E [5610]01001008-     <1>
  1105 00000C34 [6010]01001808-     <1>
  1105 00000C3A [6A10]0100050B-     <1>
  1105 00000C40 [7610]01002C0B-     <1>
  1105 00000C46 [5610]01003E0B-     <1>
  1105 00000C4C [7F10]0100800B-     <1>
  1105 00000C52 [7F10]0100900B-     <1>
  1105 00000C58 [8C10]0000          <1>
  1106                              <1> %else
  1107                              <1> 	dw ELDCALL_CODE_RELOCATIONS, 0, 0
  1108                              <1> %endif
  1109                              <1> 
  1110                              <1> %if _ELD_LINKER_PASSES
  1111                              <1> linkerlinkercoderelocations:
  1112                              <1> %if _ELDCALL_OPTIONAL || _ELDCALL_NEXT
  1113 00000C5C 0100C609[5610]0100- <1> 	dw ELDCALL_LINKER_CODE_RELOCATIONS_OPTIONAL, 0
  1113 00000C64 EA09[1410]0100F409- <1>
  1113 00000C6C [9E0F]0100FD09-     <1>
  1113 00000C72 [AE0F]0000          <1>
  1114                              <1> %else
  1115                              <1> 	dw ELDCALL_LINKER_CODE_RELOCATIONS, 0, 0
  1116                              <1> %endif
  1117                              <1> 
  1118                              <1> 	align 2, db 0
  1119                              <1> linktable:
  1120                              <1> 	istruc LINKTABLE
  1121                              <1> at ltCodeToCode
  1122 00000C76 D00E                <1> 	dw internallinkercodetocoderelocations - code
  1123 00000C78 440D                <1> 	dw internalcodetocoderelocations - code
  1124                              <1> at ltCodeToData
  1125 00000C7A DA0E                <1> 	dw internallinkercodetodatarelocations - code
  1126 00000C7C 640D                <1> 	dw internalcodetodatarelocations - code
  1127                              <1> at ltDataToCode
  1128 00000C7E DC0E                <1> 	dw internallinkerdatatocoderelocations - code
  1129 00000C80 B60E                <1> 	dw internaldatatocoderelocations - code
  1130                              <1> at ltDataToData
  1131 00000C82 DE0E                <1> 	dw internallinkerdatatodatarelocations - code
  1132 00000C84 BA0E                <1> 	dw internaldatatodatarelocations - code
  1133                              <1> at ltLinkData
  1134 00000C86 BC0E                <1> 	dw linkerlinkerdatarelocations - code
  1135 00000C88 8E0C                <1> 	dw linkerdatarelocations - code
  1136                              <1> at ltLinkCode
  1137 00000C8A 5C0C                <1> 	dw linkerlinkercoderelocations - code
  1138 00000C8C A00B                <1> 	dw linkercoderelocations - code
  1139                              <1> 	iend
  1140                              <1> %endif
  1141                              <1> 
  1142                              <1> 	align 2, db 0
  1143                              <1> linkerdatarelocations:
  1144 00000C8E 01005300[9710]0100- <1> 	dw LINK_DATA_RELOCATIONS, 0
  1144 00000C96 5A00[9710]01007900- <1>
  1144 00000C9E [AC10]01007D00-     <1>
  1144 00000CA4 [BB10]01008100-     <1>
  1144 00000CAA [CA10]01008C00-     <1>
  1144 00000CB0 [E110]01009E00-     <1>
  1144 00000CB6 [BB10]0100B200-     <1>
  1144 00000CBC [F210]0100D300-     <1>
  1144 00000CC2 [0511]0100A802-     <1>
  1144 00000CC8 [0511]0100D603-     <1>
  1144 00000CCE [0511]01000004-     <1>
  1144 00000CD4 [0511]01003006-     <1>
  1144 00000CDA [0511]01004706-     <1>
  1144 00000CE0 [AC10]01004B06-     <1>
  1144 00000CE6 [BB10]01004F06-     <1>
  1144 00000CEC [CA10]01006F06-     <1>
  1144 00000CF2 [E110]01007806-     <1>
  1144 00000CF8 [F210]01008C06-     <1>
  1144 00000CFE [E110]01001607-     <1>
  1144 00000D04 [1011]01001F07-     <1>
  1144 00000D0A [1B11]01004207-     <1>
  1144 00000D10 [2411]01005207-     <1>
  1144 00000D16 [2F11]01005F07-     <1>
  1144 00000D1C [BB10]01005609-     <1>
  1144 00000D22 [3D11]0100100B-     <1>
  1144 00000D28 [6011]0100390B-     <1>
  1144 00000D2E [1B11]01005B0B-     <1>
  1144 00000D34 [2F11]01006E0B-     <1>
  1144 00000D3A [8511]0101740B-     <1>
  1144 00000D40 [9611]0000          <1>
  1145                              <1> 
  1146                              <1> 	align 2, db 0
  1147                              <1> internalcodetocoderelocations:
  1148 00000D44 5C0064009A00A200FA- <1> 	dw INTERNAL_CODE_TO_CODE_RELOCATIONS, 0
  1148 00000D4D 05EF0649074E075607- <1>
  1148 00000D56 5B072A0B340B510B57- <1>
  1148 00000D5F 0B8E0B0000          <1>
  1149                              <1> 
  1150                              <1> 	align 2, db 0
  1151                              <1> internalcodetodatarelocations:
  1152 00000D64 2D004C00500056006A- <1> 	dw INTERNAL_CODE_TO_DATA_RELOCATIONS, 0
  1152 00000D6D 007400A700B900BD00- <1>
  1152 00000D76 C100C500C800D700E8- <1>
  1152 00000D7F 00ED00030110011901- <1>
  1152 00000D88 220126012C0137013C- <1>
  1152 00000D91 014B01500159016201- <1>
  1152 00000D9A 6701700179018401A1- <1>
  1152 00000DA3 01AE01BD01C501D601- <1>
  1152 00000DAC DA01DE01E901EE01F3- <1>
  1152 00000DB5 01F801FF0104020802- <1>
  1152 00000DBE 12021902230227022E- <1>
  1152 00000DC7 023C02420248025302- <1>
  1152 00000DD0 62026A0272027E02A5- <1>
  1152 00000DD9 02AD02B102BC02C402- <1>
  1152 00000DE2 C802CE02D402FA02FD- <1>
  1152 00000DEB 0213031F0325032803- <1>
  1152 00000DF4 2B032E033103340337- <1>
  1152 00000DFD 033A033D0340034503- <1>
  1152 00000E06 48034C034F0358035C- <1>
  1152 00000E0F 03600368036B036E03- <1>
  1152 00000E18 710375037C03830387- <1>
  1152 00000E21 038B039803A003B503- <1>
  1152 00000E2A C303C903CD03DA03E4- <1>
  1152 00000E33 033304670470047604- <1>
  1152 00000E3C 7C0480048304930497- <1>
  1152 00000E45 0402050F0515052205- <1>
  1152 00000E4E 300534054B054F0555- <1>
  1152 00000E57 056E05740579057E05- <1>
  1152 00000E60 840589058F0594059D- <1>
  1152 00000E69 05A305AC05B205BB05- <1>
  1152 00000E72 C105CA05D005D905DF- <1>
  1152 00000E7B 05E805EF05F8050006- <1>
  1152 00000E84 09060F0618061E0633- <1>
  1152 00000E8D 06410652065E066406- <1>
  1152 00000E96 6B0675067F06880692- <1>
  1152 00000E9F 06A606B406C006CB06- <1>
  1152 00000EA8 DC06E706010705070B- <1>
  1152 00000EB1 0738070000          <1>
  1153                              <1> 
  1154                              <1> 	align 2, db 0
  1155                              <1> internaldatatocoderelocations:
  1156 00000EB6 0200FFFF            <1> 	dw INTERNAL_DATA_TO_CODE_RELOCATIONS, -1
  1157                              <1> 
  1158                              <1> 	align 2, db 0
  1159                              <1> internaldatatodatarelocations:
  1160 00000EBA FFFF                <1> 	dw INTERNAL_DATA_TO_DATA_RELOCATIONS, -1
  1161                              <1> 
  1162                              <1> %if _ELD_LINKER_PASSES
  1163                              <1> 	align 2, db 0
  1164                              <1> linkerlinkerdatarelocations:
  1165 00000EBC 01007509[2411]0100- <1> 	dw LINK_LINKER_DATA_RELOCATIONS, 0
  1165 00000EC4 BD09[0511]0100BE0A- <1>
  1165 00000ECC [4F11]0000          <1>
  1166                              <1> 
  1167                              <1> 	align 2, db 0
  1168                              <1> internallinkercodetocoderelocations:
  1169 00000ED0 7F099609A709CF0900- <1> 	dw INTERNAL_LINKER_CODE_TO_CODE_RELOCATIONS, 0
  1169 00000ED9 00                  <1>
  1170                              <1> 
  1171                              <1> 	align 2, db 0
  1172                              <1> internallinkercodetodatarelocations:
  1173 00000EDA 0000                <1> 	dw INTERNAL_LINKER_CODE_TO_DATA_RELOCATIONS, 0
  1174                              <1> 
  1175                              <1> 	align 2, db 0
  1176                              <1> internallinkerdatatocoderelocations:
  1177 00000EDC FFFF                <1> 	dw INTERNAL_LINKER_DATA_TO_CODE_RELOCATIONS, -1
  1178                              <1> 
  1179                              <1> 	align 2, db 0
  1180                              <1> internallinkerdatatodatarelocations:
  1181 00000EDE FFFF                <1> 	dw INTERNAL_LINKER_DATA_TO_DATA_RELOCATIONS, -1
  1182                              <1> %endif
  1183                              <1> 
  1184                              <1> %if ELDOTHER
  1185                              <1> 	align 2, db 0
  1186                              <1> linkerotherdatarelocations:
  1187                              <1> 	dw LINK_OTHER_DATA_RELOCATIONS, 0
  1188                              <1> 
  1189                              <1>  %ifnidn LINK_OTHER_LINKER_DATA_RELOCATIONS, ""
  1190                              <1>   %error Other linker data links not supported
  1191                              <1>  %endif
  1192                              <1> %endif
  1193                              <1> 
  1194                              <1> %if ELDOTHER || ELDHINT
  1195                              <1> 	align 2, db 0
  1196                              <1> debuggeramissig:
  1197 00000EE0 65636D20<rep 5h>    <1> 		fill 8, 32, db "ecm"
  1198 00000EE8 6C446562756720-     <1> 		fill 8, 32, db "lDebug"
  1198 00000EE8 <rep 2h>            <1>
  1199                              <1> %endif
  1200                              <1> 
  1201                              <1> %if ELDOTHER
  1202                              <1> 	align 2, db 0
  1203                              <1> loaderamissig:
  1204                              <1> 		fill 8, 32, db "ecm"
  1205                              <1> 		fill 8, 32, db "Loader"
  1206                              <1> %endif
  1207                              <1> 
  1208                              <1> %ifnidni _LISTING, ""
  1209                              <1> listmsg:
  1210 00000EF0 547261634C6973742D- <1> .hint:		db "TracList-add-offset=",_LISTING,"::"
  1210 00000EF9 6164642D6F66667365- <1>
  1210 00000F02 743D646F736469722E- <1>
  1210 00000F0B 6C73743A3A          <1>
  1211 00000F10 2D2D2D2D680D0A00    <1> .hint.offset:	asciz "----h",13,10
  1212                              <1> %endif
  1213                              <1> 
  1214 00000F18 2C9A15696E7463616C- <1> 	eldcall_dump_names ELDCALL_CODE_NAMES
  1214 00000F21 6C5F6578745F726574- <1>
  1214 00000F2A 75726E5F657322580F- <1>
  1214 00000F33 636D64335F6E6F745F- <1>
  1214 00000F3C 696E6A656374629605- <1>
  1214 00000F45 496E444F530C211179- <1>
  1214 00000F4E 795F646F735F706172- <1>
  1214 00000F57 73655F6E616D652890- <1>
  1214 00000F60 046973706D6831085F- <1>
  1214 00000F69 646F7363616C6C1CE3- <1>
  1214 00000F72 0D67756172645F6175- <1>
  1214 00000F7B 7862756666F1230975- <1>
  1214 00000F84 707065726361736567- <1>
  1214 00000F8D B1087472696D707574- <1>
  1214 00000F96 73BABD04636D6433B2- <1>
  1214 00000F9F 120573657472635512- <1>
  1214 00000FA8 05707574737AD0BB1A- <1>
  1214 00000FB1 636F70795F73696E67- <1>
  1214 00000FBA 6C655F636F756E7465- <1>
  1214 00000FC3 645F737472696E67AB- <1>
  1214 00000FCC FF26646973705F6478- <1>
  1214 00000FD5 61785F74696D65735F- <1>
  1214 00000FDE 63785F77696474685F- <1>
  1214 00000FE7 62785F73697A652E73- <1>
  1214 00000FF0 746F726503AA126465- <1>
  1214 00000FF9 635F64776F72645F6D- <1>
  1214 00001002 696E7769647468398C- <1>
  1214 0000100B 08707574736C696E65- <1>
  1214 00001014 6FA20D707574736C69- <1>
  1214 0000101D 6E655F63726C66A455- <1>
  1214 00001026 09736B6970636F6D6D- <1>
  1214 0000102F 30E83A066973656F6C- <1>
  1214 00001038 3F03C3096973737472- <1>
  1214 00001041 696E673FA7AA056572- <1>
  1214 0000104A 726F72DDB90663686B- <1>
  1214 00001053 656F6C848107686578- <1>
  1214 0000105C 776F7264EBA6076465- <1>
  1214 00001065 63776F7264D5550973- <1>
  1214 0000106E 6B6970636F6D6D6198- <1>
  1214 00001077 6906696E7463686B21- <1>
  1214 00001080 300A63616C6C5F696E- <1>
  1214 00001089 743244B77408736574- <1>
  1214 00001092 6573326478          <1>
  1215 00001097 3B26126578745F696E- <1> 	link_data_dump_names LINK_DATA_NAMES
  1215 000010A0 6A6563745F68616E64- <1>
  1215 000010A9 6C6572F6340C657874- <1>
  1215 000010B2 646174615F73697A65- <1>
  1215 000010BB B2400C657874646174- <1>
  1215 000010C4 615F75736564B0B214- <1>
  1215 000010CD 617578627566665F63- <1>
  1215 000010D6 757272656E745F7369- <1>
  1215 000010DF 7A65CA510E696E7465- <1>
  1215 000010E8 726E616C666C616773- <1>
  1215 000010F1 338B00106175786275- <1>
  1215 000010FA 66665F7365676F7273- <1>
  1215 00001103 656C84E3086C696E65- <1>
  1215 0000110C 5F6F7574EB42086578- <1>
  1215 00001115 74647373656CD52D06- <1>
  1215 0000111E 6578747365675ABC08- <1>
  1215 00001127 6F7074696F6E7337E7- <1>
  1215 00001130 D30B6578747365675F- <1>
  1215 00001139 7573656455030F6275- <1>
  1215 00001142 696C645F6F7074696F- <1>
  1215 0000114B 6E5F504D68440E6C69- <1>
  1215 00001154 6E6B63616C6C5F7461- <1>
  1215 0000115D 626C65F09E22747279- <1>
  1215 00001166 5F6465627567676572- <1>
  1215 0000116F 5F616D69735F6D756C- <1>
  1215 00001178 7469706C65785F6E75- <1>
  1215 00001181 6D626572CB510E696E- <1>
  1215 0000118A 7465726E616C666C61- <1>
  1215 00001193 677334688C15616D69- <1>
  1215 0000119C 735F6D756C7469706C- <1>
  1215 000011A5 65785F6E756D626572  <1>
  1216                              <1> %if ELDOTHER
  1217                              <1> 	link_data_dump_names LINK_OTHER_DATA_NAMES
  1218                              <1> %endif
  1219                              <1> 
  1220                              <1> lmsg:
  1221                              <1> %if _ELD_LINKER_PASSES
  1222                              <1> %if _ELDCALL_OPTIONAL
  1223 000011AE 214F7074696F6E616C- <1> .warning_code_optional:		counted "Optional code link missing, hash="
  1223 000011B7 20636F6465206C696E- <1>
  1223 000011C0 6B206D697373696E67- <1>
  1223 000011C9 2C20686173683D      <1>
  1224                              <1> %endif
  1225                              <1> %if _ELDDATA_OPTIONAL
  1226                              <1> .warning_data_optional:		counted "Optional data link missing, hash="
  1227                              <1> %endif
  1228 000011D0 1844617461206C696E- <1> .error_data:			counted "Data link missing, hash="
  1228 000011D9 6B206D697373696E67- <1>
  1228 000011E2 2C20686173683D      <1>
  1229 000011E9 18436F6465206C696E- <1> .error_code:			counted "Code link missing, hash="
  1229 000011F2 6B206D697373696E67- <1>
  1229 000011FB 2C20686173683D      <1>
  1230 00001202 0A682C206C6162656C- <1> .error.2:			counted "h, label ",'"'
  1230 0000120B 2022                <1>
  1231                              <1> %endif
  1232                              <1> %if ELDOTHER
  1233                              <1> .no_other:		asciz "ELD linker: No other link info found!",13,10
  1234                              <1> .error_other:		asciz "ELD linker: Other link info unknown format!",13,10
  1235                              <1> %endif
  1236                              <1> 
  1237 0000120D 00<rep 3h>          <1> 	align 16, db 0
  1995                                  
  1996                                  	align 16
  1997                                  code_size equ $ - code
